:100000000040002029710000697100006B71000040
:1000100000000000000000000000000000000000E0
:100020000000000000000000000000006D710000F2
:1000300000000000000000006F71000071710000FE
:1000400073710000A9520000A575000073710000D3
:1000500073710000000000007371000073710000F4
:100060007371000079790000B131000073710000F4
:1000700073710000737100007371000073710000F0
:100080007371000029760000737100007371000025
:1000900073710000737100007371000073710000D0
:1000A0007371000073710000000000000000000088
:1000B0000000000000000000000000000000000040
:1000C00010B5064C2378002B07D1054B002B02D02E
:1000D000044800E000BF0123237010BD6802002027
:1000E00000000000D0E40000044B10B5002B03D04A
:1000F0000349044800E000BF10BDC04600000000F6
:100100006C020020D0E40000164B002B00D1144BF1
:100110009D46402292029A1A924600218B460F4633
:100120001348144A121A0BF05BFA0F4B002B00D045
:1001300098470E4B002B00D0984700200021040068
:100140000D000D48002802D00C4800E000BF0BF065
:1001500007FA2000290007F077FA0BF0DBF9C04618
:100160000000080000400020000000000000000027
:1001700068020020C82F00200000000000000000DE
:1001800002000120104011D1042A0ED91368180969
:1001900080B2002809D001388000031D11180979A8
:1001A000002902D001309842F8D170470020FCE7C6
:1001B0000378002B03D05AB2002A01DB01307047CC
:1001C0003F229343C03B59424B41C01803789343AD
:1001D000802BF4D10130F9E710B500240378002B0F
:1001E00001D1200010BDFFF7E3FF0134F6E770B541
:1001F000002204000D00411C092003F003FB00282D
:1002000006D001236200134343600023A34200DBB6
:1002100070BD9A00A958821891600133F6E770B555
:10022000012803DC1C2001F045F870BD01230D6896
:1002300011201D42F7D04868184206D1042804D97D
:100240000F2302681340042B01D00E20EBE703F0CC
:1002500037F96D100400002D03DDFFF7BDFFA84244
:1002600006DA1220DFE72000FFF7A2FF0400013DBD
:10027000012DF8D120787F2809DDDF280BDCF82359
:100280003F22DB00800118406378134018430123AC
:1002900040001843C9E7EF280BDCFC226378120109
:1002A0009B0113403F220007000C0343A07810403D
:1002B000ECE7F72812DCFC22637892021B03134060
:1002C000E0228004520310403F221843E378134099
:1002D000FC220343A07812018001E8E7012040429C
:1002E000D5E7F8B54D680F00EB0706D4042D04D907
:1002F0000F232E683340092B03D00B2000F0DAFFC8
:10030000F8BD6B683609B6B25C10731EA3420FD8F5
:100310000321200009F020F86421642803DC010097
:10032000032800DA03212800891903F09DFA05004B
:100330002B6800201B099BB2013B9C42E0D23A682B
:10034000A31C9B005A510123013464001C436C60C0
:10035000D6E7F0B585B0012803DC1C2000F0AAFF29
:1003600012E001274B683A000093022806D08B6800
:100370003B4203D05F10002F00DC17000124009BDC
:10038000234203D00120404205B0F0BD009B042B66
:10039000F8D91B680D680F2619003140042921D1B6
:1003A000254205D1042D03D92B681E40042E01D00F
:1003B0000E20D3E70098FFF7E3FEB842E2DB009897
:1003C00003F07EF80600280003F07AF80100781E9A
:1003D00030180BF0BBFC0028D4D0801B013040004B
:1003E0002043D1E709293DD1009B5B685B10019355
:1003F0009F42C7DC25422CD1042D2AD92B683340DB
:10040000042B26D1280003F05BF8039602907E1C93
:10041000009AB300D058854201D17800E0E720422D
:100420000ED104280CD90368039A1340042B07D17A
:1004300003F046F8010002980BF052FC0028ECD0C3
:10044000019B37009E42E2DD9CE71F00019B9F421B
:1004500098DC7B1C00999A008A58AA42F5D1780052
:100460000124BDE7032900D08CE71A0992B25B0F83
:1004700092000B40D31A01939F4200DD82E7254290
:1004800029D1042D27D92A681640032E19D1100925
:1004900080B2520F800032402C1D801A019B26181A
:1004A0001B1A0193009B781E0433019A904200DDD1
:1004B00068E722001918B2420FD316D1013040006C
:1004C000CEE7042E07D1280002F0FAFF040028002E
:1004D000FFF756FEE2E70F2040E70D78AC461578AF
:1004E000AC4502D101310132E5E70130DDE710B55D
:1004F00002F0CAFF43000120184310BDC30711D406
:1005000004280FD90F2302681340032B0AD1194086
:100510000133591AC0234907DB051940024B1A4021
:10052000114301607047C046FFFFFF9FF7B507000A
:100530000E001C20012F06DD4C68012322001A400A
:10054000009203D10D2000F0B5FE53E0022F02D03F
:100550008A681A42F6D0012335681D4200D0A9E00E
:10056000042D00D8A6E01C41002C00DC1C000F204C
:1005700029680840092828D16B685B100093022F76
:1005800005D0B368009A5B109A4200DD0093009B8F
:1005900001221D1B0135EB43DB171D40691C09209F
:1005A00003F030F9071E09D001236D001D4303003D
:1005B0003268083345600099A14201DA3800FEBD77
:1005C0000134A100515802C3F5E7042845D12800A1
:1005D00002F076FFFFF700FE0190022F04D0B3680F
:1005E0005B10984200DD0193019BA34204DA0020D6
:1005F00003F07AF90700E1E7280002F061FF070045
:10060000009BA34221DB2800009702F059FF050060
:100610003800FFF7CDFD019B01340700A342F7DA54
:10062000009BC41A200003F05FF9071EC6D002F039
:1006300047FF0190306802F043FF2200009B591BE6
:10064000411801980AF0B0FFB8E73800FFF7B0FD95
:10065000009B070001330093D2E703282AD10B093E
:100660009BB2490F9B000140591A022F04D0B26877
:100670005210914200DD1100A14205DA0022032050
:10068000110003F0BFF8B5E703200E1B331DD91787
:100690000140C9188910002203F0B4F8071E00D1E8
:1006A0008CE7013631000334FFF728FF381D291984
:1006B0003200C7E7212046E7F8B5002805DC1C20FA
:1006C00000F0F8FD05002800F8BD01260C68264062
:1006D0000FD06410E343DB171C40E11C891000229B
:1006E000032003F08FF8051EEDD02100FFF706FF71
:1006F000E9E7042C01D80025E5E70F232268134021
:10070000042B1BD12000FFF73BFDC31C0700032077
:10071000D9170140C9188910320003F073F8051E7B
:10072000D1D03900FFF7EAFE200002F0C9FE2B1DF0
:1007300001003A0018000AF037FFC4E7092BDAD1AC
:100740000320636832005F10FB1CD9170140C918F1
:10075000891003F057F8051ECDD03900FFF7CEFE03
:10076000FF20BE42AFDA0122B300E3189B681342B8
:1007700008D01341FF2B00DD0300D943C917AA1984
:100780000B4013710136ECE710B57F2902DC0170D4
:10079000013010BD1A4B99420CDC40238A115B4298
:1007A000134303703F230B4080214942194341709A
:1007B0000230EEE7134B994210DC20230A135B4210
:1007C00013433F24802203708B1152422340214067
:1007D00013430A43437082700330DAE70A4B9942AD
:1007E000D7DCF0230370603B4370113B8A11FF3B61
:1007F0001A4382703F2211401943C1700430C8E788
:10080000FF070000FFFF0000FF0F0100F0B50D0023
:1008100085B0002803DC1C2000F04CFD0DE00968C9
:100820000122080010400AD002AC11412000FFF75D
:10083000ABFF011B200003F063F804001AE0042959
:100840003FD90F230C682340092B3AD14B685B102A
:10085000019303239C46019B9A420EDD03F044F86A
:10086000041E07D02E68012502F02AFE2F00019BEE
:100870009D421DDD200005B0F0BD01329300CC5833
:100880000123234001D10D20C6E764107F2C0DDD2C
:100890000D4E0223B44209DD0C4E6346B44205DD21
:1008A00000270B4EE30FA6427B419B00C018D2E706
:1008B0000135AB00F1583942E5D04910FFF764FF2C
:1008C000D5E72120A8E7C046FF070000FFFF000092
:1008D000FF0F010010B504000120084010D10429C9
:1008E0000DD90F230A681340042B08D1080002F029
:1008F000E7FD010020000BF0F3F94342584110BD21
:100900000020FCE7F7B50F00012803DC1C2000F0F5
:10091000D1FCFEBD01264D682E4006D1042D04D920
:100920000F222B681A40092A01D00B20EFE76A68D2
:100930001B099BB25410A34200D85C1E39681E48A4
:10094000FFF7C8FF01230190002813D139681B4825
:10095000FFF7C0FF002811D0002C0DD00123621C2E
:10096000013C9C409200535123436B6004E00136EC
:10097000B200AB50B442FADA0020CAE73B680D205F
:10098000DA07C4D55B10002B11DD9C420FDB9B0006
:10099000A200291DEB1889180433994209D10123BB
:1009A000013C9C40AA181C4353606C60E4E7122091
:1009B000ADE758681860EFE773CC000077CC000013
:1009C000002310B50C000B70C30705D50D4942106C
:1009D00020000BF049F908E00B49002802D0042858
:1009E00004D10A4920000BF05FF910BD0428FCD99E
:1009F0000F2302681340042BF7D102F061FD044974
:100A00000200E5E770D600007CCC000082CC00003C
:100A100087CC0000F0B593B0060002911C20012E97
:100A20001DDD029B01251B681C002C4000D0ADE0A1
:100A3000042B00D8E6E01A680F231A40092A4AD18D
:100A40000394039A029992008A5817002F4005D107
:100A5000042A03D910681840092806D0222000F083
:100A600029FC0190019813B0F0BD52685210A418EF
:100A7000039A013203929642E3D1611C012202F0F3
:100A8000C1FE0190002802D100230193EAE7019BF7
:100A90006400190025435D600831029ABB00D058FC
:100AA00002684368120992B25B109A4200D8531E42
:100AB0000022934209DCDA43D21713409B00C91885
:100AC000039B01379F42E8DBCCE794000519AD6832
:100AD00001320D51EDE72700032A59D10193029A03
:100AE000BB00D3582B42B9D1042BB7D91868019950
:100AF0000140032939D1020992B2430F92000B4001
:100B0000D31A1C190137BE42E9D10320E31CD917BF
:100B10000140C9188910002202F074FE01900028DB
:100B2000B2D000252100FFF7E9FC019B1E1D029AAF
:100B3000AB00D45801231C421FD1042C1DD90F2116
:100B400023681940032918D1180980B25B0F80006F
:100B50000B40C01A0023834213DBC343DB1718404A
:100B600001353618BD42E2DB7CE7042900D075E789
:100B70001800FFF705FB2418C4E72000FFF700FB6F
:100B8000E8E7E2181279F2540133E4E700273C0069
:100B90000F25029ABB00D3580122134234D1042BF3
:100BA00032D9186801002940042935D11800FFF70F
:100BB000E7FA24180137BE42EBD1200002F094FE80
:100BC0000190002800D15FE7029FB600BB19041D09
:100BD000029301233D681D4229D1042D27D90F26F8
:100BE0002B681E40042E37D12800FFF7C9FA0600F3
:100BF000280002F065FC0100200032000AF0D4FC5D
:100C0000A41922E02700C3E7180005A9FFF7D8FEC2
:100C100005A80BF06FF8CCE7032900D01EE7020906
:100C200092B2430F92000B40D31A1C19C2E705A9D8
:100C30002800FFF7C5FE05A80BF05CF805A9050024
:100C4000020020000AF0B0FC6419029B0437BB428A
:100C5000BFD10023237005E7032EF6D11A0992B203
:100C60005B0F92001E40961B291DC5E7F0B50D00D5
:100C700095B0002806DC1C2000F01CFB04002000BE
:100C800015B0F0BD0C68012123000B40009306D184
:100C9000042C04D922680F331A40092A01D00B20F2
:100CA000EAE7626852100392002A03DC009802F01F
:100CB0001BFEE3E73F4A019201280BD06868084217
:100CC00008D1042806D902681340042B02D102F08F
:100CD000F7FB019001980BF00DF806000F27039B1E
:100CE0000834013B04935E43039B02909B001B1955
:100CF000059301232068184251D104284FD9036875
:100D00003B40042B52D1FFF73BFA059B04343618C5
:100D1000A342EED1300002F0E7FD041EAFD02B68F5
:100D20000593029B002B03D0686802F0C9FB019079
:100D3000200002F0C5FB0500009B059A9B00D3181C
:100D40009F68380002F0BCFB012306001F4201D15E
:100D5000042F04D807A93800FFF732FE07AE300091
:100D60000AF0C8FF07000200310028000AF01CFC4E
:100D7000029BED19002B0AD0049B009A934206DDDA
:100D80002800029A01990AF00FFC029BED18009BC3
:100D900001330093009A039B9342CDD16FE707A9DB
:100DA000FFF70EFE07A80AF0A5FFAEE702F088FBEA
:100DB000F9E7C04614D1000010B50024A04207DDB9
:100DC0000B6801341C4003D05C10E343DB171C406C
:100DD000611C0122092002F015FD002803D0012327
:100DE00064001C43446010BD0A6870B51000012502
:100DF000284034D1042A32D90F24136849681C4092
:100E0000092C17D154681B099BB22C41A34200D86E
:100E10005C1E844205DC02200133984206DB002080
:100E20000FE085005519A9600130F2E784001151E7
:100E30000130F2E7032C12D1294203D1132000F034
:100E400039FA70BD4910FF29F8D81B099BB204324A
:100E50009B00D3189342E2D911700132FAE70B20BC
:100E600000F028FADBE700000123F7B500254E6803
:100E70000F0033400093AB420ED11D00042E0BD95E
:100E80000F2233681A40092A10D172681B099BB2DD
:100E90005510AB4200D85D1E3968CB0717D54C10F2
:100EA000002C01DDA5421DDA122032E0042A04D113
:100EB0003000FFF765F90500EEE7009D032AEBD14E
:100EC0001D09ADB25B0FAD001340ED1AE4E72E48EB
:100ED000FFF700FD002814D00AF062FE290008F098
:100EE00021FB4C1C009B002B4CD1042E4AD93268AC
:100EF0000F331340092B10D10134A400A459200052
:100F0000FEBD39682148FFF7E5FC2C000028E9D137
:100F1000113000F0CFF90400F1E7042B2AD13000A2
:100F200002F0CEFA0500FFF757F9A042BCDB012C16
:100F30001ADC300002F0C4FA00902800FFF738F9FC
:100F4000461B300002F0D0FC041ED8D002F0B8FAE4
:100F50000190786802F0B4FA009B3200E91A411857
:100F600001980AF021FBCAE72800FFF721F9013CAC
:100F70000500DCE7032B05D13419E478023B64005B
:100F80001C43BCE70B20C4E76CCC000077CC00000E
:100F9000F7B54D680F002A0001210A402FD1042D1A
:100FA0002DD90F242B68BE681C40092C14D1696808
:100FB0001B099BB24C100192A34200D85C1E3968F9
:100FC0002A48FFF787FC00282DD00F232A681340FA
:100FD000092B1DD1012317E0032C10D10E4203D1A0
:100FE000132000F067F9FEBD72100192FF2AF7D8B6
:100FF0001A0992B25B0F92001C40141BDFE70B2012
:10100000EFE701339A00AE509C42FADA0020EAE79B
:10101000032BFBD12B0001335A1BA242F6DC6A469C
:101020001279DA70F7E73968CB0706D5491000293D
:1010300001DD8C4209DA1220D3E70D48FFF74AFCA4
:101040002100002801D11130CBE70F232A6813407B
:10105000092B03D1013189004E51D7E7032BD5D19C
:101060006B461B796D18EB70D0E7C04673CC00005F
:1010700077CC000010B50124086820421AD104285A
:1010800018D90F2102681140092901D1406810BD0B
:10109000032908D113099BB2500F9B000840181A6E
:1010A00040002043F3E7042904D102F009FAFFF7D6
:1010B00093F8F5E70B2000F0FDF8E8E710B5034AD8
:1010C0000B21034804F0B2F910BDC04614CC000057
:1010D0000CCC0000002070470420704701207047AE
:1010E00010B5002002F000FC10BD00207047002069
:1010F0007047002070470020704700207047002094
:1011000070470020704700207047000010B5034A68
:101110000C21034804F08AF910BDC046FCCC000045
:101120005CCD000010B50124044002D04410200022
:1011300010BD042810D90F2302681340042B07D1D7
:1011400002F0BEF921000A220AF09CFE0400EEE73C
:10115000032B01D10430F5E70D22014B1A70E6E7AD
:10116000A8020020012210B5024018D1042802D99B
:1011700003681A0992B201230B4012D1042902D943
:101180000B681B099BB20024934206D104309B00DC
:101190000431C318984206D30124200010BD002258
:1011A000E9E70023EFE704780A78002C01D1002A50
:1011B000F2D0013001319442ECD00024EDE7000080
:1011C000F7B50700009101933049314B002A02D056
:1011D00002220A70013A00261A601B68CE54BE42F1
:1011E00000DBF7BD009AB300D058294B274D1C688F
:1011F000C8239B0065191C1B0123184206D0254AF1
:101200004310210028000AF0FDFC09E0224A0028D2
:1012100002D004281BD1214A210028000AF0F2FC48
:101220001A4C20000AF066FD194A019B1060002B41
:101230000BD07B1EB34208DD194B984205D8431CE6
:101240001360202222540022E2540136C7E704280A
:1012500019D90F2301680B40042B04D102F030F997
:10126000104A0300CDE7092B03D143680E4A5B10F7
:10127000C7E7032B08D10A0992B2490F92000B402D
:10128000D31A0A4ABDE70123094ABAE7A902002096
:10129000CC05002070D600007CCC000082CC000081
:1012A0001F0300009BDC0000CCCF0000DBCF000060
:1012B000E6CF0000014B187000207047A802002004
:1012C00070B501F063FE094C0100251D1F222800A6
:1012D0000AF028FD28000AF00DFD042304308008E0
:1012E000000118432060200070BDC0468402002029
:1012F000C368F0B59D00836889B05D190300183399
:1013000006930369069A9F00069B0290DF194369C2
:1013100001939B00D3180393CD4B1B78002B26D150
:101320007F222B68CB491C1213409B005B5804356D
:1013300001929F46029B587804F0A4FC0023029A75
:10134000137027E0C24B1B78002B10D12B68019A39
:101350001C121340BF4A9B009B580435E9E7069BCB
:101360003A1DD11ABA4BD82928DD1A221A70029BCD
:10137000B74C9B6821780193EA1A029B92109B78E4
:1013800012021A43029B587804F084FC0023029A4C
:1013900023701370029B069A9B680193ED1A029BBF
:1013A000AD10DD60069BFE1A029BB6101E61039B0A
:1013B0009B1A029A9B10536109B0F0BD1B783C60E8
:1013C000002B01D01700D2E72B6801991C120B40AB
:1013D000A0499B005B5817000435AAE7069B3A1DFD
:1013E000D11A9B4BD82902DD1A221A70BFE7286850
:1013F0001B78291D3860002B02D017000D00B6E7BE
:101400006B6801991C120B4092499B005B581700B6
:1014100008358EE7069B3A1DD11A8D4BD82902DD7F
:101420001A221A70A3E7A4001B782C193C60002B29
:1014300001D017009BE72B6801991C120B408549CE
:101440009B005B581700043573E7069B3A1DD11AC1
:101450007F4BD82902DD1A221A7088E77E49A40042
:1014600061581B783960002B01D017007FE72B688B
:1014700001991C120B4077499B005B5817000435FB
:1014800057E7043F744B3A68A400E250704B1B7856
:10149000002B00D06BE72B68019A1C1213406D4A99
:1014A0009B009B58043544E76B4BA400E058FFF7C2
:1014B00039FE043F06003868FFF734FE3618012075
:1014C000654B76000643E650614B1B78002B00D03D
:1014D0004DE72B68019A1C1213405E4A9B009B58F3
:1014E000043526E7069B3A1DD11A594BD82902DD4F
:1014F0001A221A703BE70698039C0121A04202D2EF
:1015000021000C3909681B783960002B01D01700C5
:101510002DE72B6801991C120B404E499B005B582C
:101520001700043505E7069B3A1DD11A484BD82908
:1015300002DD1A221A701AE70699039881420FD227
:1015400003000C3B1B6845495B106418E41AA400B7
:1015500023583B603E4B1B78002B05D0170006E755
:10156000182119700023F4E72B6801991C120B4015
:1015700038499B005B5817000435DAE6069B039A4E
:10158000934219D213000C3B1B68344A043FA41841
:101590005B10E31A039A39689B0099502C4B1B7817
:1015A000002B00D0E3E62B68019A1C121340294A55
:1015B0009B009B580435BCE61822254B1A70EDE7BA
:1015C000069B039A93422DD2244B3E1FE31814002E
:1015D0000C3C04932368049A5B10D31A039A9B0073
:1015E0009858FFF79FFD07903068FFF79BFD246830
:1015F000049B64101C1B079BA4001F1801207F0084
:10160000039B0743E7503700114B1B78002B00D09A
:10161000ADE62B68019A1C1213400E4A9B009B58A2
:10162000043586E618220A4B1A70EDE7069B3A1D30
:10163000D11A074BD82902DD1A221A7097E60399AE
:10164000A40061581B783960002B09D017008EE682
:10165000A8020020CCCD0000942D0020FDFFFF3F0C
:101660002B6801991C120B40D9499B005B5817004D
:1016700004355EE6043F039B3A68A400E250D54B74
:101680001B78002B00D072E62B68019A1C121340C5
:10169000CF4A9B009B5804354BE6039BA4001C19C2
:1016A0002368043F38685E10FFF73CFD36180120C0
:1016B000C84B76001B7806432660002B00D056E608
:1016C0002B68019A1C121340C14A9B009B58043599
:1016D0002FE6069BA4003F1BBE4CBB420CD82378D0
:1016E000002B00D043E62B68019A1C121340B84A25
:1016F0009B009B5804351CE6B74801F0D1FE2378C7
:10170000002B00D033E62B68019A1C121340B04A1C
:101710009B009B5804350CE6A300ED18002C00DA62
:1017200038E6AC4B1B78002B00D020E62B68019AE2
:101730001C121340A64A9B009B580435F9E5043F50
:101740003B68042B04D1A300ED18002C00DA21E63D
:10175000A04B1B78002B00D009E62B68019A1C12C5
:1017600013409B4A9B009B580435E2E5043F3B68CD
:10177000042B04D0A300ED18002C00DA0AE6954BE8
:101780001B78002B00D0F2E52B68019A1C12134045
:101790008F4A9B009B580435CBE53E1F3068FFF70E
:1017A000C1FC013806D401234000A40018432D19C0
:1017B0003060EFE5874B37001B78002B00D0D6E573
:1017C0002B68019A1C121340814A9B009B580435D8
:1017D000AFE53A00069B0C32D31AD82B03DD1A2250
:1017E0007C4B1A70C3E5FF2361005B001940FE3B90
:1017F000FF3B1943396002990698896824120491C5
:101800006D1A0299AD1089782D020D4303999D4000
:10181000091A891099401D430B43BB60029B7D60F0
:101820009C70E4B26D4BE4000392E358029A93601B
:10183000684A1278002A03D008331D00039F96E5FA
:101840001D00019A9B680C351C121340604A9B00D6
:101850009B58039F6DE53B1F1C68039A069B9342B0
:101860002DD10A20E3070CD4042C13D90F232268AE
:101870001340042B11D1200001F022FE0AF03AFAA5
:101880000630643003F00CFE00280FD1043D069BA7
:1018900003937FE50720042CF3D02000431E9841DA
:1018A000FA234042FF3318400730EAE7029B210049
:1018B000587804F001FA0023029A1370E7E7039BBB
:1018C000039A0C3B1B6802995B109B00D31A0C3BDC
:1018D0001C601F1D1300083B1B685A108A70D2B28F
:1018E0003E49D2005B0055589B0A029A9B009560C6
:1018F000ED18039B069A043B1B685B109B00D318F2
:101900000393344B1B78002B00D030E52B68019AF1
:101910001C1213402E4A9B009B58043509E53B1FBF
:101920001868FFF7FFFBA40006003F1B1E2827DCFA
:1019300000280DDC274B1B78002B00D017E52B6807
:10194000019A1C121340224A9B009B580435F0E474
:1019500001F00AFB033E361801F006FB204B801B0A
:101960009842F9D81B4B1B78002B00D0FFE42B6862
:10197000019A1C121340164A9B009B580435D8E468
:101980000123029A137001F0EFFA029B0A388619BC
:101990005E60FFE43B1F1868FFF7C4FBA40006006D
:1019A0003F1B00280DDC0B4B1B78002B00D0DEE426
:1019B0002B68019A1C121340054A9B009B58043562
:1019C000B7E4084B98420FDD1D22024B1A70CEE49B
:1019D000CCCD0000A8020020F8CF00009C250020FC
:1019E0003F420F0080EE36000123029A137001F08F
:1019F000BBFAFA239B005E43029B0A3E30185860F4
:101A0000C8E4A300FF1A002320001A003900FFF7E2
:101A1000D7FBD44ED44C3168200001F071FFD34B7A
:101A200031681860200003F0EBFF3168200004F0FB
:101A30004AF9CF4B1B78002B00D098E42B68019A11
:101A40001C121340CB4A9B009B58043571E4C84BD1
:101A5000A4001B783F1B002B00D088E42B68019A60
:101A60001C121340C34A9B009B58043561E4029842
:101A700003F07AFDBE4B1B78002B00D077E42B6877
:101A8000019A1C121340BB4A9B009B58043550E43A
:101A90003B1F1B68002B3ED13B000C3B1B68DA0749
:101AA0002CD5390001225B105800083902430A6026
:101AB000002B44DD012259001143381F0160390019
:101AC000083909681141CB1A39000C3909681142EB
:101AD00024D09B189340A4001343039AA350A44B13
:101AE0001B78002B00D042E42B68019A1C12134093
:101AF000A04A9B009B580435FFF71BFC042B06D91A
:101B00000F211A680A40092A01D15B68C9E7192226
:101B1000974B1A702BE45B10013BC9E7042909D9E4
:101B20000F200A680240092A04D102339B005B5847
:101B3000A400D2E719228E4B1A70FFF718FC043567
:101B4000CDE7A300069AFB189B1AD82B13DC0122C1
:101B5000631E002C14DC864B1B78002B01D0FFF792
:101B600006FC2B68019A1C121340824A9B009B586A
:101B70000435FFF7DEFB1A227D4B1A70FFF7F7FBE7
:101B80003A601C000437E3E7069A3B1D9B1A784E27
:101B9000D82B03DD1A233370FFF7E9FB069B039A6A
:101BA000A40093422AD23B1F1868FFF7BBFA011E1C
:101BB00021DD039B0C3B1A68521082421BDB90070D
:101BC000801A6D4B4018C018039B8000C2583B1B05
:101BD0001A60674B3F1B1B780437002B01D0FFF7BF
:101BE000C6FB2B68019A1C121340624A9B009B584B
:101BF0000435FFF79EFB20233370EAE71823FBE749
:101C00005A4BA4001A683B1B1F001A60584B04373C
:101C10001B78002B01D0FFF7AAFB2B68019A1C123E
:101C20001340544A9B009B580435FFF782FB3B1F2F
:101C30001A68042A11D1A4002D194D4B1B78002BD2
:101C400001D0FFF794FB2B68019A1C121340494AFC
:101C50009B009B580435FFF76CFB1F00EDE73A1F14
:101C60001368042B04D0002313603A00A4002D193C
:101C70003F4B1B78002B02D01700FFF778FB2B6837
:101C800001991C120B403B499B005B58170004351F
:101C9000FFF74FFBA3009C46FE1A002C17DC1C220A
:101CA000334B1A70002333606346FF1A304B0437FE
:101CB0001B78002B01D0FFF75AFB2B68019A1C12EE
:101CC00013402C4A9B009B580435FFF732FB002041
:101CD00033685A108300F15801230B4003D10D21C2
:101CE000234A1170DFE749108A4200DD0A00013003
:101CF0008442EFDC012352001343D4E7A3009C4647
:101D0000FE1A002C17DC1C22194B1A7000233360BA
:101D10006346FF1A164B04371B78002B01D0FFF7E0
:101D200026FB2B68019A1C121340124A9B009B58F9
:101D30000435FFF7FEFA002033685A108300F1588B
:101D400001230B4003D10D21094A1170DFE749102F
:101D50008A4200DA0A0001308442EFDC012352009B
:101D60001343D4E7CC050020A9020020080000207E
:101D7000A8020020CCCD0000FCFFFF3F3B00083B49
:101D80001868FFF7CFF93B1F06001868FFF7CAF97C
:101D90000023864200DA0433A4003A1B17001360C4
:101DA000E54B04371B78002B01D0FFF7E0FA2B68D6
:101DB000019A1C121340E14A9B009B580435FFF71F
:101DC000B8FA3B00083B1868FFF7ACF93B1F060068
:101DD0001868FFF7A7F9F30FC217B0425341A400E8
:101DE0003A1B17009B001360D34B04371B78002B62
:101DF00001D0FFF7BCFA2B68019A1C121340CF4A9E
:101E00009B009B580435FFF794FA3B00083B186889
:101E10003B1F1968A600BE1B0423814202D0042880
:101E200002D80023336018E001239C461842F8D101
:101E30000F2302681A40042AF3D163461942F0D1F5
:101E40000429EED90B680B321340042BE9D1FFF7BC
:101E500089F9431E984180003060B74BA4001B787D
:101E60003F1B0437002B01D0FFF781FA2B68019A42
:101E70001C121340B14A9B009B580435FFF759FAD6
:101E80003B00083B18683B1F1968A600BE1B0023D7
:101E9000814202D0042802D80423336018E00123D1
:101EA0009C461842F8D10F2302681A40042AF3D145
:101EB00063461942F0D10429EED90B680B32134066
:101EC000042BE9D1FFF74EF94342584180003060BE
:101ED000994BA4001B783F1B0437002B01D0FFF760
:101EE00046FA2B68019A1C121340944A9B009B5897
:101EF0000435FFF71EFA3B00083B1868FFF712F99C
:101F00003B1F06001868FFF70DF9F317C20F864252
:101F10005341A4003A1B17009B001360864B043703
:101F20001B78002B01D0FFF722FA2B68019A1C12B4
:101F30001340824A9B009B580435FFF7FAF93B0097
:101F4000083B1868FFF7EEF83B1F06001868FFF71C
:101F5000E9F80023864200DD0433A4003A1B170091
:101F60001360754B04371B78002B01D0FFF7FFF986
:101F70002B68019A1C121340704A9B009B58043531
:101F8000FFF7D7F93B1F1B68A400043B5A1E93417F
:101F90003A1B17009B001360674B04371B78002B1C
:101FA00001D0FFF7E4F92B68019A1C121340634A31
:101FB0009B009B580435FFF7BCF93B00083B1868B1
:101FC000FFF7B0F83B1F06001868FFF7ABF83218B0
:101FD0000120A4003B1B1F00520002431A60564B15
:101FE00004371B78002B01D0FFF7C1F92B68019A49
:101FF0001C121340514A9B009B580435FFF799F976
:102000003B00083B1868FFF78DF83B1F0600186877
:10201000FFF788F8321A0120A4003B1B1F00520072
:1020200002431A60444B04371B78002B01D0FFF7A2
:102030009EF92B68019A1C121340404A9B009B5842
:102040000435FFF776F93B00083B1868FFF76AF89C
:102050003B1F06001868FFF765F802000120A40086
:102060003B1B1F007243520002431A60324B04377D
:102070001B78002B01D0FFF77AF92B68019A1C120C
:1020800013402E4A9B009B580435FFF752F93B1F23
:102090001868FFF747F8061E17D11F23264A13704A
:1020A000A4003B1B1F001E60234B04371B78002B32
:1020B00001D0FFF75CF92B68019A1C1213401F4AEC
:1020C0009B009B580435FFF734F93B00083B186828
:1020D000FFF728F8310007F03FF9012640000643DA
:1020E000DEE73B1F1868FFF71DF8061E17D11F23F8
:1020F000114A1370A4003B1B1F001E600E4B0437D7
:102100001B78002B01D0FFF732F92B68019A1C12C3
:1021100013400A4A9B009B580435FFF70AF93B001D
:10212000083B1868FEF7FEFF310007F0FBF90126B7
:1021300049000E43DEE7C046A8020020CCCD0000D7
:102140003B1F1868FEF7EEFFC217801850400122AF
:10215000A4003B1B1F00400010431860F14B0437E4
:102160001B78002B01D0FFF702F92B68019A1C1293
:102170001340ED4A9B009B580435FFF7DAF8A300A3
:10218000FE1A3068012C24D1FEF7CCFF049407908E
:1021900009F006FD0799002900DC012107F0C2F9CA
:1021A000049BA400C918012349001943DD4B3F1BC0
:1021B0001B7831600437002B01D0FFF7D8F82B686B
:1021C000019A1C121340D84A9B009B580435FFF714
:1021D000B0F8FEF7A7FF04907068FEF7A3FF049B1A
:1021E0000130C31A0793D3E7A300FE1A3100200081
:1021F000049301F00BFD049B3060FF1AC94B0437B8
:102200001B78002B01D0FFF7B2F82B68019A1C1243
:102210001340C54A9B009B580435FFF78AF83B00E2
:10222000083B1868FEF77EFF3B1F06001868FEF7A4
:1022300079FF02000120A4003B1B1F003240520026
:1022400002431A60B74B04371B78002B01D0FFF70D
:102250008EF82B68019A1C121340B34A9B009B58BE
:102260000435FFF766F83B00083B1868FEF75AFF95
:1022700006003B1F1868FEF755FF3200024301209D
:10228000A4003B1B1F00520002431A60A54B0437F9
:102290001B78002B01D0FFF76AF82B68019A1C12FB
:1022A0001340A14A9B009B580435FFF742F83B00BE
:1022B000083B1868FEF736FF06003B1F1868FEF75C
:1022C00031FF320042400120A4003B1B1F0052009E
:1022D00002431A60934B04371B78002B01D0FFF7A1
:1022E00046F82B68019A1C1213408F4A9B009B589A
:1022F0000435FFF71EF83B1F1868FEF713FFC043B5
:102300000122A4003B1B1F00400010431860854BB6
:1023100004371B78002B01D0FFF729F82B68019AAE
:102320001C121340804A9B009B580435FFF701F8AC
:102330003B00083B1868FEF7F5FE06003B1F1868D7
:10234000FEF7F0FE3200824051000122A4003B1B48
:102350001F000A431A60734B04371B78002B01D00F
:10236000FFF705F82B68019A1C1213406E4A9B0078
:102370009B580435FEF7DDFF3B00083B1868FEF76D
:10238000D1FE06003B1F1868FEF7CCFE320002416A
:1023900051000122A4003B1B1F000A431A60614B3D
:1023A00004371B78002B01D0FEF7E1FF2B68019A60
:1023B0001C1213405C4A9B009B580435FEF7B9FF82
:1023C0003B000C3B1868FEF7ADFE3B00083B0600E7
:1023D0001868FEF7A7FEF1170200C317300007F0D8
:1023E000F3F83B1F049005911868FEF79BFE02006E
:1023F0000498059907F09CF843000120A4003E1BB7
:1024000037001843474B30601B780437002B01D04E
:10241000FEF7ADFF2B68019A1C121340424A9B0045
:102420009B580435FEF785FFA300FE1A31002000FB
:102430000493FEF7C1FC049B3060FF1A394B04374C
:102440001B78002B01D0FEF792FF2B68019A1C121B
:102450001340354A9B009B580435FEF76AFFA300E2
:10246000FF1A39002000FEF7BFFC2E4B1B78002B13
:1024700001D0FEF77CFF2B68019A1C1213402A4AF8
:102480009B009B580435FEF754FFA300FE1A310051
:1024900020000493FEF7E8FC049B3060FF1A214BF8
:1024A00004371B78002B01D0FEF761FF2B68019ADF
:1024B0001C1213401C4A9B009B580435FEF739FF41
:1024C000A300FF1A39002000FEF762FD154B1B78B0
:1024D000002B01D0FEF74BFF2B68019A1C12134012
:1024E000114A9B009B580435FEF723FFA300FE1AF8
:1024F000310020000493FEF7BDFD049B3060FF1AFD
:10250000084B04371B78002B01D0FEF730FF2B68F7
:10251000019A1C121340044A9B009B580435FEF795
:1025200008FFC046A8020020CCCD00003B1F186861
:1025300000F0C6FF3A00083A12680300A400D10771
:1025400029D4042A0CD910680F2210400138082819
:102550000FD806F06DFE052026220E0E0E0E24006A
:10256000EC49180009F0BCFB434258413B1B80007A
:102570001860E94B3F1B1B780437002B01D0FEF796
:10258000F6FE2B68019A1C121340E44A9B009B58EC
:102590000435FEF7CEFEE249E3E7E249E1E7E2492E
:1025A000DFE7E249DDE7069B3E1DF31ADA4CD82B44
:1025B00003DD1A232370FEF7DAFE00F0DFFC430090
:1025C0000120184323783860002B02D03700FEF733
:1025D000CEFE2B68019A1C121340D04A9B009B58D8
:1025E00037000435FEF7A5FE069B3E1DF31ACA4CC4
:1025F000D82B03DD1A232370FEF7B9FE00F0B4FCDC
:10260000CB4B400018400123184323783860002B3F
:1026100002D03700FEF7ABFE2B68019A1C12134064
:10262000BE4A9B009B5837000435FEF782FE069B8E
:102630003E1DF31AB84CD82B03DD1A232370FEF786
:1026400096FE00F09BFCBB4B1A68831A904201D2A5
:10265000B94A9B1801205B0003433B602378002BA1
:1026600002D03700FEF783FE2B68019A1C1213403C
:10267000AA4A9B009B5837000435FEF75AFE00F02B
:102680007DFCAC4BA4001860A34B3F1B1B78002BB8
:1026900001D0FEF76CFE2B68019A1C1213409F4A72
:1026A0009B009B580435FEF744FE0123A600BE1B89
:1026B00020001A003100FEF783FDA04C2068643032
:1026C00002F0EEFE002802D1043DFEF763FE029BFD
:1026D00021685A789A4803F004FB0123029A3700D4
:1026E000137000F041FC974B22681B68063253437D
:1026F0001818029B5860FEF74DFEA600BE1B200076
:10270000012300223100FEF75BFD8C4C2068643011
:1027100002F0C6FE0028D7D0894803F061F8DCE754
:10272000A4003E1BFEF7CCFD37007B4B30601B78CE
:102730000437002B01D0FEF71AFE2B68019A1C12F9
:102740001340764A9B009B580435FEF7F2FD724B0E
:10275000A4001B783F1B002B01D0FEF708FE2B685E
:10276000019A1C1213406D4A9B009B580435FEF7DA
:10277000E0FDA4003E1B300000F02FFC3700664B4C
:1027800030601B780437002B01D0FEF7F0FD2B687A
:10279000019A1C121340614A9B009B580435FEF7B6
:1027A000C8FDA4003E1B300000F019FC37005A4B56
:1027B00030601B780437002B01D0FEF7D8FD2B6862
:1027C000019A1C121340554A9B009B580435FEF792
:1027D000B0FDA300FE1A31002000049300F002FCBB
:1027E000049B3060FF1A4C4B04371B78002B01D040
:1027F000FEF7BDFD2B68019A1C121340474A9B004F
:102800009B580435FEF795FDA4003F1B380000F0EF
:102810001BFC414B1B78002B01D0FEF7A8FD2B6859
:10282000019A1C1213403D4A9B009B580435FEF749
:1028300080FDA300FE1A31002000049300F02CFC60
:10284000049B3060FF1A344B04371B78002B01D0F7
:10285000FEF78DFD2B68019A1C1213402F4A9B0036
:102860009B580435FEF765FDA4003F1B380000F0BF
:1028700055FC294B1B78002B01D0FEF778FD2B6807
:10288000019A1C121340254A9B009B580435FEF701
:1028900050FD0121200000F029FC1F4B1B78002B6C
:1028A00001D0FEF764FD2B68019A1C1213401B4AED
:1028B0009B009B580435FEF73CFD0021200000F0F2
:1028C00015FC154B1B78002B01D0FEF750FD2B6833
:1028D000019A1C121340114A9B009B580435FEF7C5
:1028E00028FDA4003E1B300000F03AFC37000A4BE4
:1028F00030601B780437002B01D0FEF738FD2B68C1
:10290000019A1C121340054A9B009B580435FEF7A0
:1029100010FDC04608D00000A8020020CCCD000069
:1029200010D0000017D000001ED0000023D00000FF
:10293000FEFFFF7FD405002037894100CC05002031
:10294000A902002004000020A4003E1B300000F07B
:102950001BFC3700EE4B30601B780437002B01D096
:10296000FEF705FD2B68019A1C121340E94A9B00F3
:102970009B580435FEF7DDFCA4003F1B380000F037
:10298000DDFBE34B1B78002B01D0FEF7F0FC2B683E
:10299000019A1C121340DF4A9B009B580435FEF736
:1029A000C8FCA4003F1B380003F0E0FCD84B1B78A8
:1029B000002B01D0FEF7DBFC2B68019A1C121340A0
:1029C000D44A9B009B580435FEF7B3FCA4003E1B81
:1029D000300003F065FD3700CD4B30601B780437C5
:1029E000002B01D0FEF7C3FC2B68019A1C12134088
:1029F000C84A9B009B580435FEF79BFCA4003F1B74
:102A0000380003F063FCC24B1B78002B01D0FEF7AB
:102A1000AEFC2B68019A1C121340BE4A9B009B58C7
:102A20000435FEF786FCA4003E1B300003F064FC76
:102A30003700B74B30601B780437002B01D0FEF70E
:102A400096FC2B68019A1C121340B24A9B009B58BB
:102A50000435FEF76EFCA300FF1A3900200001F0D8
:102A600015FCAB4B1B78002B01D0FEF780FC2B68CC
:102A7000019A1C121340A74A9B009B580435FEF78D
:102A800058FCA300FF1A3900200001F013FAA04BF4
:102A90001B78002B01D0FEF76AFC2B68019A1C12F0
:102AA00013409C4A9B009B580435FEF742FCA30050
:102AB000FF1A3900200001F021FB954B1B78002BF9
:102AC00001D0FEF754FC2B68019A1C121340914A66
:102AD0009B009B580435FEF72CFCA300FF1A39001D
:102AE000200001F033FB8A4B1B78002B01D0FEF74E
:102AF0003EFC2B68019A1C121340864A9B009B588F
:102B00000435FEF716FCA300FE1A310020000493E2
:102B100003F05EFD049B3060FF1A7D4B04371B7889
:102B2000002B01D0FEF723FC2B68019A1C121340E6
:102B3000784A9B009B580435FEF7FBFBA300FE1A66
:102B400031002000049303F04BFD049B3060FF1A1A
:102B50006F4B04371B78002B01D0FEF708FC2B6865
:102B6000019A1C1213406B4A9B009B580435FEF7D8
:102B7000E0FBA300FE1A31002000049303F038FDAF
:102B8000049B3060FF1A624B04371B78002B01D086
:102B9000FEF7EDFB2B68019A1C1213405D4A9B0067
:102BA0009B580435FEF7C5FBA300FE1A3100200038
:102BB000049303F0F7FA049B3060FF1A544B043778
:102BC0001B78002B01D0FEF7D2FB2B68019A1C1258
:102BD0001340504A9B009B580435FEF7AAFBA30004
:102BE000FF1A3900200001F09DF9494B1B78002B9A
:102BF00001D0FEF7BCFB2B68019A1C121340454A1A
:102C00009B009B580435FEF794FBA300FF1A390084
:102C1000200001F0C3FA3E4B1B78002B01D0FEF7D9
:102C2000A6FB2B68019A1C1213403A4A9B009B5842
:102C30000435FEF77EFBA300FE1A3100200004934A
:102C400001F028FA049B3060FF1A314B04371B78DF
:102C5000002B01D0FEF78BFB2B68019A1C1213404E
:102C60002C4A9B009B580435FEF763FBA300FF1A18
:102C70003900200001F0D6F9254B1B78002B01D03C
:102C8000FEF775FB2B68019A1C121340214A9B002A
:102C90009B580435FEF74DFB069B029AFB1A9B10CE
:102CA0001361A300FF1A3900200002F0D7FD184B72
:102CB0001B78002B01D0FEF75AFB2B68019A1C12DF
:102CC0001340144A9B009B580435FEF732FB069BC9
:102CD000029AFB1A9B101361A300FE1A3100200018
:102CE000049302F0BBFD049B3060FF1A084B0437CD
:102CF0001B78002B01D0FEF73AFB2B68019A1C12BF
:102D00001340044A9B009B580435FEF712FBC04653
:102D1000A8020020CCCD00000023F7B55A1E019276
:102D2000002B07DA01F0C8FA02F0C8FE03F038F809
:102D30001923019300263000194B1968B14212DDA6
:102D4000184B1A6801328A420FDAF0241A601D68A3
:102D5000154F6C43E35D002B1FD0E419022B06D105
:102D60002000FEF7C5FA019BD8E70022EDE7012B12
:102D70000DD1002801D100F0F7F8F0226A43BB180A
:102D80005B680A49C31A8B4201D80223BB54F02363
:102D90005D43054BEB5C022BE2D00136CCE7C0462D
:102DA000D0050020000000203C1C00203F420F0006
:102DB000012200210A4B0B481A61195004301950A6
:102DC000A2210420C9005850C121C02089008002DE
:102DD00058501A60044BFC311960044B1A7070474C
:102DE00000A000400405000000E100E0FB05002019
:102DF00004207047F8B550C9012322001A40101E64
:102E00002DD03340181E2AD0641000201C2C26D848
:102E10001D4B761035009E4200DD1D001B4F3B5DB3
:102E2000012B05D00121200004F0F2FD01233B55C8
:102E3000174B1B78002B01D1FFF7BAFF0023154A6F
:102E40009E420DDCFF2514491448D65CB44202D1E1
:102E50005E007052D5540133042BF6D10420F8BD26
:102E6000D15C8C4203D10C4A5B009D52F6E70133E2
:102E7000042BF5D10023D15CFF2901D1D454F2E712
:102E80000133042BF7D1E9E788130000DC050020AB
:102E9000FB0500201C0000200E000020DC050000C7
:102EA00070B530C9012322001A40101E1BD02B40E0
:102EB000181E18D064101C2C00D90024174E335D46
:102EC000012B05D00121200004F0A2FD0123335580
:102ED00069100800124A1038124B904204D901229E
:102EE00052421A60042070BD1C600F4806F034FA8C
:102EF0000E4B18800E4B1B78002B02D1FFF758FFAA
:102F0000F0E701220B4B9A64A922D2009A5880184C
:102F1000A82280B2D2009850E4E7C046DC05002029
:102F2000908601001800002020A107000C0000205E
:102F3000FB05002000A00040030010B50120002B7D
:102F400002DC1B30FEF7B6F910BD0420704710B547
:102F5000002803DC1C20FEF7ADF910BD0B68002033
:102F6000DB07FAD40D30F6E70122034B1A64A822DE
:102F7000D20098587047C0460080004010B5FFF757
:102F8000F3FFFA21890006F05DF910BD0048704793
:102F900080D000001D20704770B5054E0400335CE2
:102FA0000D008B4202D004F033FD355570BDC04694
:102FB000DC05002070B50024064D635D012B05D1B2
:102FC0000021200004F024FD0023635501341D2C52
:102FD000F2D170BDDC05002070470D2070473B200A
:102FE00070470000F8B501240B6806000D0023426D
:102FF00004D10D20FEF75EF92000F8BD5B10200023
:10300000052BFAD80E4A9B009C580E4F3B5D002BB7
:1030100005D00021200004F0FBFC00233B55012ECD
:1030200006DD6B68042B03D10221200004F0F0FCC4
:10303000200004F09BFB012440002043DDE7C04654
:1030400068D00000DC050020F8B50126056835428F
:1030500002D04468344203D10D20FEF72BF9F8BDAD
:103060006D101C2DFBD80A4F7B5D012B04D0310065
:10307000280004F0CDFC7E55064964108C4202DC29
:10308000E143C9172140280004F0F6FBE7E7C046FA
:10309000DC050020FF03000070B501240D68254207
:1030A00004D10D20FEF706F9200070BD6D101C2D17
:1030B00017D80024012804DD4C68043C63425C41BD
:1030C0006400094E735DA34204D02100280004F07F
:1030D0009FFC7455280004F0CFFC03000420012B52
:1030E000E3D00020E1E7C046DC05002070B5040015
:1030F0000D001C280ED8084E335C012B04D0012192
:1031000004F086FC01233355290020004D1EA941FF
:1031100004F09CFC70BDC046DC050020036810B5BF
:10312000DA0703D40D20FEF7C5F810BD416858102A
:1031300004394A425141FFF7D9FFF6E737B56946EE
:103140000A00064B30CB30C203680220042B02D1A8
:1031500000F0D4FF37BD00F0F9FFFBE730D00000EE
:1031600010B5084C6379002B05D00021052004F030
:103170004FFC00236371052004F07EFC434258415C
:10318000800010BDDC05002010B5084CE37A002B50
:1031900005D000210B2004F03BFC0023E3720B2040
:1031A00004F06AFC43425841800010BDDC05002059
:1031B000F7B5304D304E6B6C002B15D0A824002392
:1031C000E40037596B642D4B186800280CDB2C4B3E
:1031D00019784A425141C9B2197004F037FC294BA1
:1031E0001B88DF19BFB23751AB6C002B39D00021DF
:1031F000254B264FF458A9643A780C340193244D9A
:103200008A4206D02B68032B03D8224AD05C04F0F4
:103210001DFC2B68204A0133134004D50422013BD6
:103220005242134301331B4900228C462B60042B6E
:1032300018D06046C05C591CFF2802D10B00012247
:10324000F5E7002A00D02B60012104F0FFFB0123E9
:103250003B702B68114A5B009B5AE418019BA4B297
:10326000F450F7BD01235B422B6000233B700C4BF5
:10327000F3E7C046FCA0004000A00040180000207A
:10328000FA0500200C00002044050000F90500208C
:10329000D80500201C000020030000800E00002044
:1032A00050460000084B094AFF201A805A809A8035
:1032B000DA800023064A07491370074A08704870ED
:1032C0008870C870136070470E000020DC05000095
:1032D000F90500201C000020D80500200122024B27
:1032E00052421A607047C0461800002010B5034AC9
:1032F0000621034802F09AF810BDC04638D00000FD
:10330000A2D70000E12170B54902194803F0A4FFDB
:10331000002401220320174B17491A615C50043125
:1033200058508018083158501A60063004F018FAC6
:10333000FF21124AA15401341D2CFBD1012200208F
:103340000F4B01001A6004230E4A0F4D1468002C25
:10335000FCD02C680002013B20431160002BF5D10A
:1033600001220A4B1A6004F033F901F0F1F870BD44
:10337000C41B00200080004004050000DC05002084
:1033800000D0004000D1004008D5004004D00040EB
:10339000F8B50B4E070030000D0003F0A5FF040048
:1033A000A84200DD2C003D00EB1B9C4205DD3000F7
:1033B00003F0A4FF28700135F6E72000F8BDC046F1
:1033C000C41B002010B50100014803F04DFF10BDE3
:1033D000C41B002010B5054C200003F053FFE12171
:1033E0002000490203F038FF10BDC046C41B002076
:1033F000C3070CD4064B1B68834208D8054B1B68D7
:10340000984204D8031F1B68002B00D01800704797
:1034100004060020000600200023012210B50A48FF
:10342000990001334250642BFAD1084C084B00211B
:103430001A602000074A08F0D3F8074B074A636078
:10344000074B1A6010BDC046942D002008060020CE
:1034500008000020D4090000302700000C060020DE
:10346000FC05002010B5044B044A1A60044B054AC1
:103470001A60FFF7D1FF10BD0406002008060020E7
:1034800000060020DC0F0020044B1B6818680009B0
:1034900080B20238C343DB1718407047FC05002098
:1034A00000B59BB00200054901A808F0DDFB01A8AA
:1034B00002F0B2F902F074FCFCE7C04604D100004F
:1034C0000B4BC20704D4042804D80A4B00D00A4B83
:1034D000180070470F2203681A40031D042AF7D012
:1034E000064B092AF4D0064B032AF1D0054BEFE72F
:1034F000DED0000082CC00007CCC0000E8D00000D0
:10350000F8D00000EFD000000020064A0649131F43
:10351000186013681B099BB202339B00D2188A42C1
:10352000F5D370470C060020DC0F0020F7B50F2400
:103530000126314B314A1968314B324D18681368F6
:103540001F002740072F26D813681B099BB20233A0
:103550009B00D218AA42F2D300242B4EA500AD192D
:103560002868FFF745FF01342860642CF6D1274C0A
:103570002068FFF73DFF2060254C2068002802D01E
:10358000FFF736FF20600025224B1B680093009B4D
:103590009D4214DBF7BD1B099BB29B00D3189A42D6
:1035A000D2D01F68374208D1B94206D2B84204D3FC
:1035B000043F3F68002F00D01F60043BEFE7F0237B
:1035C0006B43154A9B181A78002A01D10135DEE7B2
:1035D0001F693C2300266B43DB199B0001930136D6
:1035E000BB1BF3D4019BB4001C1B0B4B1C19A06923
:1035F000FFF7FEFEA061F2E7040600200C060020A3
:1036000000060020DC0F0020942D00200800002080
:10361000DC0F0020D00500203C1C0020F7B5012461
:10362000204246D1234B1B689C46984241D3224BF3
:103630001B68019398423CD8031F1B68002B38D1AC
:103640000200036800941B099BB2002B0FD1009964
:10365000131F196090422CD015682B1F1B6899000E
:1036600069180C68013B14600A602A00EDE79D00B0
:1036700055192968009C214219D18C4517D8019C05
:103680008C4214D30E1F3468002C10D10F680F34F5
:103690003C40072C08D92F60151F2B600B680A606F
:1036A0001B099BB20A00D0E700993160CDE7013BCE
:1036B000CBE7F7BD04060020000600200D4970B5D9
:1036C0000A000D4D1368141F1B0926689BB2981C35
:1036D000002E0BD000238A4200D00B002360830011
:1036E000C91880001218AA42ECD370BD1B011360E8
:1036F000F7E7C0460C060020DC0F0020F8B5124C9E
:1037000027000F223B681D09ADB213420DD06E1C7D
:10371000B600A74204D032003900200007F04DFF68
:103720000022A3190436A4191A600235AD00074B14
:103730007F199F42E5D31B1B9B10013B1B0123609C
:10374000034B1C60F8BDC0460C060020DC0F0020B7
:10375000FC050020F0B59BB0FFF706FC0024070035
:10376000214AA300D0580134FFF758FF642CF7D149
:103770001E4B1868FFF752FF1D4B1868002801D038
:10378000FFF74CFF00261B4B1B689E4217DBFFF721
:1037900095FFFFF7CBFEFFF7B1FFFFF7E5FB164BF9
:1037A000C21B1B6815491B6801A81B099BB2023B81
:1037B00008F05AFA01A802F02FF81BB0F0BDF0256E
:1037C00075430F4BED182B78002B01D10136DAE74A
:1037D0002B695C1E002CF9DBA300EB189869FFF73E
:1037E0001DFF013CF6E7C046942D00200800002094
:1037F000DC0F0020D0050020FC050020BED000001A
:103800003C1C0020F7B5174D4F1C2B6806001B68A9
:103810000C001B099BB201929F420BDBFFF79AFF42
:103820002B681B681B099BB29F4203DB0A20FDF734
:1038300041FDFEBD2868A71CBA00DB1B81181B01D7
:103840000B6029600021031F19600F231E40030035
:103850002401264340C3083A9A189A42E9D90199AB
:1038600002C3FAE7FC050020F7B50300012213406C
:1038700004000D000193002B2BD1174B1B688342D2
:1038800027D8164B1B68834223D90F23144F386067
:1038900000681840FFF7B6FF019B3C68061E3B60BE
:1038A00017D0236804301B099BB29D4200DD1D0028
:1038B000AA00211D251F07F077FEFFF725FE2E60C9
:1038C000FFF734FE00232B602268064B1340236071
:1038D00034002000FEBDC046040600200006002083
:1038E000DC0F0020F0FF0F000323043010B5C117D8
:1038F00019400918891000220420FFF783FF10BD2A
:1039000070B5050008000C00FFF7EEFF002300284B
:1039100004D170BDE95CC21811710133A342F9DB17
:10392000E343DB171C40002304192371F1E7F0B5D2
:103930000C009BB0022804DC1C20FDF7BBFC1BB074
:10394000F0BD01230868184206D1042804D90F26C7
:1039500001683140042901D00E20EEE761680D00B6
:103960001D40F9D10429F7D90A683240042AF3D15D
:10397000A2681A4201D10D20DFE7FFF7A1FD060082
:103980006068FFF79DFDA768010001AC7F10300063
:10399000257003F00CF839006423220003F06CF862
:1039A000200008F0A7F901002000FFF7A9FFC6E7F3
:1039B00010B51C4CA544041E02D1FFF795FF0BE087
:1039C00002F00EFF0138062828D805F031FC09095D
:1039D00011182904240000208023DB009D4410BD21
:1039E000200002F079FF011B2000FFF789FFF3E7B9
:1039F000200002F01FFF430001201843ECE7802263
:103A00006946D200200002F02CFF684608F072F9E7
:103A100001006846E9E704210348E6E70020CCE717
:103A20000420D9E700FCFFFF4CD1000070B50C006A
:103A3000022803DC1C20FDF73DFC70BD0123086853
:103A4000184206D1042804D90F2501682940042909
:103A500001D00E20EFE761681942FAD10429F8D9A4
:103A60000A682A40042AF4D1A2681A4201D10D2022
:103A7000E1E7FFF725FD05006068FFF721FDA46879
:103A800001006410280002F092FF210002F0CFFF35
:103A9000FFF78EFFD1E770B50D00012803DC1C2075
:103AA000FDF708FC70BD01240868204206D10428F7
:103AB00004D90F2102680A40042A01D00E20EFE742
:103AC0006A682242FAD1042AF8D913680B40042B01
:103AD000F4D1FFF7F5FC06006868FFF7F1FC010080
:103AE000300002F064FF02F0E6FF40002043D9E717
:103AF000F8B507000C001C20012F0BDD012508681C
:103B0000284206D1042804D90F2102680A40042A59
:103B100003D00E20FDF7CEFBF8BD62682A42F8D133
:103B2000042AF6D913680B40042BF2D1FFF7C8FC26
:103B300006006068FFF7C4FC0100022F14D0A468DF
:103B40002C4211D06410300002F031FF050002F069
:103B500047FE012811D1002C02DD0135012C06D1D0
:103B60002800FFF725FFD7E701246442EBE7280090
:103B700002F0BEFE013C0500F0E70228F0D1002C67
:103B8000EEDD0135012CEBD000222800110002F0FF
:103B9000E1FE02F0ADFE013C0500F3E710B50124A3
:103BA0000868044016D04410200005F069FE15494D
:103BB00005F034FD07F01AFC04F06CF80022124BFB
:103BC00006F0CEFD04F00EF807F0A0FB4300012044
:103BD000184310BD042810D90F2302681340042B8A
:103BE00007D1FFF76DFC21000A2208F04BF9040011
:103BF000DAE7032B01D10430F5E70D20FDF75AFB7E
:103C0000D2E7C046D30237390000D040086870B50B
:103C100001240500254006D1042804D90F23026899
:103C20001340042B03D00E20FDF744FB70BDFFF7BB
:103C300047FC03782900233B5A4253411022C01805
:103C400008F020F980239B05C218044B9A4201D941
:103C50001420E9E740002043E8E7C046FFFFFF3FAC
:103C600010B5034A0621034801F0E0FB10BDC04631
:103C70001CD1000015D100000020704710B51E2097
:103C8000FDF718FB10BD10B51E20FDF713FB10BD8E
:103C900010B51E20FDF70EFB10BD10B51E20FDF760
:103CA00009FB10BD10B51E20FDF704FB10BD10B5BB
:103CB0001E20FDF7FFFA10BD10B51E20FDF7FAFA21
:103CC00010BD10B51E20FDF7F5FA10BD10B51E2071
:103CD000FDF7F0FA10BD10B51E20FDF7EBFA10BD90
:103CE00010B5034A0B21034801F0A0FB10BDC046EC
:103CF00088D10000E0D100000120034B1860034B85
:103D00001B6883401843704700100020E00F00201C
:103D1000F0B5EFF310810123194083F31088134CA1
:103D2000134AA4461268134E013A9340124F134AA5
:103D3000002B17D0146803420FD03D682C60C0469A
:103D4000C046C046C046C046C046C046C0460C4CF1
:103D50001568246825605B08EAE765462C601468EE
:103D60003460F8E781F31088F0BDC04608050050C4
:103D7000200000200C050050EC0F0020F40F002064
:103D8000E80F002030B585B001AD0C2206492800AF
:103D900007F00AFC0024285D01210134FFF7FCF83C
:103DA0000C2CF8D105B030BD75D20000F7B56A46CD
:103DB000394B01AD13801C239370384B2B800A23A1
:103DC000AB70FFF7D1F8364B364CC01823689842D9
:103DD00001D2002323602668002E3DD16B469F5DF3
:103DE00001213800FFF7D8F801360021380003F030
:103DF0002DFE032EF2D10026AF5D01213800FFF722
:103E0000CBF801360121380003F020FE032EF3D158
:103E1000C8200138C046C046C046C046C046C0465D
:103E2000C046C046C046C046C046C046F1D100218B
:103E30002878FFF7B1F868780021FFF7ADF8A87887
:103E40000021FFF7A9F8FFF78FF8FA2300251B01DF
:103E5000C01820602800FEBDFFF786F82368002503
:103E60009842F7D3032003F081FC0600042003F0FE
:103E70007DFC36180A2003F079FC0B4B9B1B181AAB
:103E80000A4BA84206DB18600023094A236013602E
:103E90000125DFE71D60F7E71A1B0000030400009F
:103EA00010270000F80F0020E3030000E00F0020BF
:103EB000001000200022054B10B51A60044B1B684F
:103EC000934201D002F02CFC002010BDFC0F00201A
:103ED000E81A002010B5041E10DA00240A4BA400D2
:103EE000E25801239340094A09491360094A1160C5
:103EF000094A0A4911600A4A136010BDFFF74AF8DF
:103F0000A042EADDEAE7C04688DF0000F40F0020A7
:103F100008050050EC0F0020E80F00200C050050B1
:103F200018050050F0B53B4B85B01B680C00002B0A
:103F300003D101204042FFF7CDFF24680122270072
:103F4000174028D0FF2360121840334967146610C9
:103F500040431F401E4005F0FFF9050438002E497C
:103F6000784305F0F9F90002054330002A4970430F
:103F700005F0F2F9294B28431B68202B06D1640079
:103F8000A40E274BA400E35800021843FFF7C0FE1D
:103F9000002005B0F0BD042CFAD90F2321680B4096
:103FA000092BF5D1636803925B100193019B9F423B
:103FB000EEDABB00E3189E68039B1E4228D0FF2365
:103FC0007012184072101A401349751440431D4076
:103FD000009205F0C1F9030428000F4968430293D9
:103FE00005F0BAF9029D0002054300980A494043D2
:103FF00005F0B2F9094B28431B68202B06D1760047
:10400000B60E074BB600F55800022843FFF780FEB6
:104010000137CBE7F40F00205906000020000020F4
:104020005CD400000200086810B5C3070FD540102B
:104030001823012A03DD4A68042A00D10833054AFF
:104040001360FEF7C9FFFFF745FF002010BD0120F8
:104050004042EDE72000002010B50124044002D0CA
:104060004410200010BD042810D90F23026813400B
:10407000042B07D1FFF724FA21000A2207F002FFE0
:104080000400EEE7032B01D10430F5E70D20FDF726
:1040900011F9E6E70868F8B5C3071AD5FFF7DCFFA2
:1040A0000300203B5E2B25D80520434301221D1829
:1040B0000020114E9D4219D005211024F75C3C428E
:1040C00000D080180139520064100029F7D1013363
:1040D000F0E704280ED90F2203681A40042A09D1F8
:1040E0001B099BB2002B05D00379DAE701234000BE
:1040F0001843F8BD0120FCE781D2000070B50868C4
:104100000D00FFF7A9FF04006868FFF7A5FF621E16
:104110000100042A14D8451E042D11D805236B4331
:104120009B18012215009D402B00064805682B4373
:104130000360054B1B68002B02D0200002F0F1FA4F
:10414000002070BDFC0F0020E81A002070B5086840
:104150000D00FFF781FF04006868FFF77DFF621E16
:104160000100042A13D8451E042D10D805236B43E3
:104170009B1801229A400748036893430360064B4B
:104180001B68002B03D00022200002F0CAFA002096
:1041900070BDC046FC0F0020E81A0020F0B50500F5
:1041A00089B008680C00FFF757FF0690022D36DD36
:1041B0006068FFF751FF0190A068FFF74DFF040012
:1041C0000127231D661E0793731C0293079B9E42C3
:1041D00035D0052373430593019B019D053304935B
:1041E000049BAB421ED0042E16D86B1E042B13D892
:1041F0000122059B2349013B5B199A409446224AC0
:104200000B681068069A3A4003920DD062461A4332
:104210000A60012200280DD17F000135E0E701246A
:104220000194CDE7029ECFE7624693430B600028DE
:10423000F2D0039A0299280002F073FAECE7019B8E
:104240001E1D042E1AD8012C18D1002505273B006D
:1042500021006B439B1999400B000A4A01351168F4
:104260009943094B11601B68002B05D0019B00226C
:10427000581D290002F055FA052DE8D1002009B09B
:10428000F0BDC046FC0F0020E81A0020086810B5F9
:10429000C30703D5FFF7E0FE054B1860054B1B680D
:1042A000002B03D0024B186802F03CFA002010BD2E
:1042B000FC0F0020E81A00207FB5A04C2368002BDB
:1042C0000AD19F4A1268002A06D19E4B1B68002B18
:1042D00001D0FFF76BFD7FBD9B4D2A68002A26D1D8
:1042E000984A1268002A1BD0FFF760FD0028F2D020
:1042F000FFF748FD924B24681A681C60002A16D00C
:10430000002C14D101AD0C229049280007F04CF983
:10431000285D00210134FEF73FFE0C2CF8D1DAE7CE
:10432000874A1268002AE5D1002BE3D0E0E700219C
:104330001A2003F08BFB00211B2003F087FB0021D8
:104340001C2003F083FB2E68012E5CD0022E00D1CE
:10435000A2E0002E50D101363100794C03202368B1
:10436000994303F073FB0420216801404B425941FB
:1043700003F06CFB102123680A2019404B4259417D
:1043800003F064FB80212368090119404B42594125
:10439000062003F05BFB80212368090219404B4291
:1043A0005941072003F052FB80212368490219403C
:1043B0004B425941092003F049FB802123688902BF
:1043C00019404B425941192003F040FB80212368DA
:1043D000C90219404B425941182003F037FB802392
:1043E00021681B0319404B425941172003F02EFB53
:1043F00031001A2003F02AFB2B680321581C05F01A
:1044000091F8296067E702214D4C17202368194075
:104410004B42594103F01AFB082123681820194028
:104420004B42594103F012FB80212368C900194017
:104430004B425941042003F009FB802123684901C4
:1044400019404B4259410A2003F000FB80212368A8
:10445000C90119404B425941032003F0F7FA80216A
:104460002368890319404B425941092003F0EEFAB1
:10447000802321681B0419404B425941192003F045
:10448000E5FA3100062003F0E1FA3100072003F0DD
:10449000DDFA31001B20ADE72021294C17202368CD
:1044A00019404B42594103F0D1FA402123681820AA
:1044B00019404B42594103F0C9FA80212368192061
:1044C00019404B42594103F0C1FA80212368490049
:1044D00019404B425941092003F0B8FA8021236862
:1044E000890019404B425941072003F0AFFA80215F
:1044F0002368890119404B425941062003F0A6FA6E
:1045000080212368490319404B4259410A2003F096
:104510009DFA80212368C90319404B425941032069
:1045200003F094FA802321685B0419404B425941FF
:10453000042003F08BFA01211C205BE7FC0F002014
:10454000F00F002000100020E40F002075D20000C2
:10455000012010B54042FFF7BDFC10BD10B5034A65
:104560000921034800F062FF10BDC0465CD5000081
:10457000A4D500008023F0B502255B051A690A4C1A
:104580000A4BA1261D5103278025F600ED00BA43F2
:10459000884202D300221A51F0BD5F59002FFCD08F
:1045A00098518018F4E7C0460405000000E001407F
:1045B00010B5002806D1C020B02140028902FFF7C3
:1045C000D9FF10BDB02080218002C902F7E70000AA
:1045D00043425841064B40421840B0239B02C0184A
:1045E000036800201A0E532A01D11B02180A7047D3
:1045F00000C0FEFF30B501248025054B054AED00C3
:104600009C505C59002CFCD001600021995030BDB9
:1046100000E001400405000043425841074B40427E
:104620001840B0239B02C018A62310B50902DB0571
:10463000090A1943FFF7DEFF10BDC04600C0FEFFA8
:10464000F0B5012480260D4B0D4DF6005C5100297C
:1046500002DC00225A51F0BD577814783F022743FC
:10466000947824042743D478043224063C439F5989
:10467000002FFCD010C00139E9E7C04600E001403E
:104680000405000070B505004B680A009C1C210061
:10469000A400FFF7D5FF281970BD0000134B1B685D
:1046A000002B0CD08022B023D2029B0200280BD119
:1046B0001A1D5B681B0E522B00D110007047B022F0
:1046C000C02392025B02F1E782420DD903681B0E00
:1046D000522B09D1436802339B00C018824203D990
:1046E00003681B0E522BE9D00020E7E704110020DD
:1046F000F0B50020B7B00024FFF7D0FF2700050079
:104700002600002D2ED1284D2868FFF761FF3200CA
:104710003B0001900094254904A807F0A5FA04A8DD
:1047200001F07AF8224B64201C682B68A0215A42C1
:104730005341204A5B421340B02292029B18E41A74
:104740006043490204F008FEA022520203000092D6
:104750001949220004A807F087FA04A801F05CF8C0
:1047600037B0F0BDFF226B6829689C460233FF1802
:104770000B12013613409C4200DA1C00FF200A1481
:10478000024003926246014001920091039A0B4954
:1047900004A807F069FA04A801F03EF82800FFF722
:1047A0007DFF0500ADE7C04604110020AED6000035
:1047B0000811002000C0FEFF58D600009AD6000065
:1047C00070B50020FFF704FF04000120FFF700FF91
:1047D000844200DA04000A4B1D686A4255412800F1
:1047E0001D60FFF7E5FEA0226B4252021340054A0E
:1047F00028009B18044A611C1360FFF70DFF70BD71
:10480000041100200480010008110020F8B50020E8
:10481000FFF7DEFE07000120FFF7DAFE3E00204D25
:104820000643204C0DD18021C020C9024002FFF771
:10483000A1FE01213000FFF7EFFE1B4B2E6023602D
:104840001DE0874209DD0023B0212B60164B890251
:10485000236023680020012517E0012380212B60BD
:10486000124BC9022360F4E7120E522A08D0002826
:1048700000D023600E4800F0CFFFFFF7A1FFF8BD86
:1048800028005A68023292009B188B4205D21A689F
:10489000561CE9D10028F2D0D1E72160EFE7C046ED
:1048A00004110020081100200480010004C002004F
:1048B00073D6000070B50020FFF7F0FEFF2605005C
:1048C000002801D1280070BD03681C143440FFF794
:1048D000E5FEDA2CF4D10500F2E700008022F0B505
:1048E0005200A1B00021674806F07AFE8022002124
:1048F0005200654806F074FE644BFF271B681A00DF
:10490000049353425A4110000592FFF751FE049C54
:104910000020631E9C415E4B64421C405D4BE418CA
:10492000FFF7C8FF0600002E2DD10498FFF750FEB8
:10493000411C0598FFF770FE059A574D534B2C60AC
:104940001A60FEF747FD514B64201B68A0215A42B4
:1049500053414F4A5B421340B0222C6892029B188D
:10496000E41A6043490204F0F7FCA022520203005B
:1049700000924A49220007A807F076F907A800F03C
:104980004BFF21B0F0BD3268131412123A403B4085
:1049900003921A000A3A092A49D83A4B039A995CB9
:1049A000002931D110223E4806F01AFE35002B684E
:1049B00003991A123A40914209D11A143A400B2A2B
:1049C00027D0132A2DD00A2A01D1354B1D6028008B
:1049D000FFF764FE051EEAD1314B196800290FD09C
:1049E0002000FFF74FFE04002D4B5B19596800298A
:1049F00003D02000FFF746FE040004350C2DF3D150
:104A0000204B0121039A99543000FFF747FE06001E
:104A100089E73B40022BDADC214A9B00D3185D601A
:104A2000D5E7102200211E4806F0DAFDCFE71A0074
:104A3000153A082AE8D8144A0399525C002AE3D1AF
:104A40003500152B00D01500300003681A143A40C9
:104A5000152A0FD01D2A00D10025FFF71FFE0028C0
:104A6000F3D1002D04D020002900FFF70BFE040035
:104A7000054BC6E7039A1B123B409A42EDD1050055
:104A8000EBE7C046041000200C11002004110020A8
:104A900000C0FEFF04C00200081100203DD6000047
:104AA000242F002010B5FFF719FF10BDF0B585B019
:104AB000039203220333DC17294D1440E4182B68BA
:104AC000284F5A42534180225B42D202A4103B40FD
:104AD0009B18A21C0291244E910000910190316814
:104AE00000980A18934215D2FFF7F8FE2B685A4235
:104AF000534180225B421F40D202BF183368009AA4
:104B00009B189F4206D2194800F086FE0025280017
:104B100005B0F0BD029B356819066B461A7BA423CD
:104B2000DB051343FF222F00090C1943019B1204DC
:104B30001B04134019432800FFF75CFD0837281DAC
:104B400021003760FFF756FD002C04D00A9A21009F
:104B50003800FFF775FD009B083BFF183760D6E76C
:104B60000411002000C0FEFF0811002017D600002D
:104B700070B59AB0FFF74AFEFF221E4CD20000210A
:104B8000200006F02DFDFF25FFF794FE00260028EB
:104B900014D10200C300E3580130591E8B41D218D2
:104BA000FF28F7D1144901A807F05EF801A800F02A
:104BB00033FE124800F030FE1AB070BD03681A14BC
:104BC0002A400A2A0AD11A122A40FF2A03D0D20008
:104BD000A1180B71A050FFF761FDD8E7132AFAD195
:104BE0001B122B40FF2BF6D0DB00E2181671E650AB
:104BF000F1E7C0469C250020E3D60000F7D6000070
:104C00000021094B094A5960013151605968002956
:104C1000FCD000211961012393600222044B8131F1
:104C2000FF315A501A607047FC10004000100040DD
:104C300000E100E00222064B0121DA670022054B69
:104C40005A61054A11615A69002AFCD07047C04672
:104C500004E100E0FC1000400010004010B5044CDE
:104C60002378002B01D0FFF7E5FF0020207010BD56
:104C70000D120020802301205B055B6E5B00184352
:104C8000704700000120024B1B685B00184370470F
:104C9000901200200120024B1B685B0018437047F4
:104CA000240000200120024B1B685B001843704762
:104CB0009412002070B504000D001600FEF75EF996
:104CC000802301215B055A6E267000265300617017
:104CD000E1706272010A5A0A6071A171A272010C3C
:104CE0005A0C000E5B0EA6702571E1712072E27203
:104CF000237370BD10B5044C200006F0FBFF0100CB
:104D00002000FEF7FDFD10BD991200200E4B10B5DE
:104D10001B680E4C5A1C0FD00D4C002B0CD00D4CA8
:104D2000012B09D00C4C022B06D0094C042B03D0CC
:104D30000A4C052B00D1074C200006F0DBFF0100D8
:104D40002000FEF7DDFD10BD2800002088D7000000
:104D500010D0000093D7000017D000008DD70000BE
:104D600070B5214C2278002A3DD1204B01215A6098
:104D70008022D20511605A68002AFCD00022072048
:104D80001B4B1C4901255A500439585008315A50C0
:104D900019481A4958501A491A485A501A495A502B
:104DA000A622D2009D50082218495A50043158506A
:104DB00002201749585017491748585017480439C6
:104DC0005850182016495850C12189005A500539A9
:104DD000FF395858921802435A501249124A9950B2
:104DE000FFF70EFF257070BD0D120020FC00004083
:104DF000001000400C050000746962751C0500007D
:104E000024050000200004022C0500001405000009
:104E1000340500003C050000FFFF000021100100E8
:104E2000540500000E1200200405000070B50E4B62
:104E300006001B78002B01D1FFF792FF00200B4DDD
:104E40002C7884420ED00A4B202219780323091BA8
:104E50001940084B4901C918300006F0A5FB012094
:104E6000013C2C7070BDC0460D120020981200202D
:104E70000C1200200E120020002370B588B098425A
:104E800035DD0D6801262C0034409C422FD12300D3
:104E9000042D2CD90F222B681A402300092A26D171
:104EA0006A683F2A23DD6846FFF7C0FF2300002819
:104EB0001DD06B4619783300A14203DB6B461B5DA6
:104EC0005B003343A200AA1801349360202CF2D176
:104ED000092169444A780B7812021A438B781B0423
:104EE0001A43CB781B061343024A136004231800AD
:104EF00008B070BD9412002070B5454B8AB01B7885
:104F0000002B01D1FFF72CFF02AC2000FFF78EFF32
:104F1000002802D100200AB070BD23780B2BF9D9EC
:104F20006378012BF6D1E378012BF3D10023112014
:104F3000384E394D33602B7068442379374A4178B5
:104F40001360027809021143827812041143C27877
:104F500012060A4332490A60002B0ED1152169441A
:104F60004A780B7812021A438B781B041A43CB78C9
:104F70001B0613433360002318E0012B1AD11521BF
:104F800069444A780B7812021A438B781B041A433F
:104F9000CB781A211B06134333600E23627C6944CD
:104FA000934200DD130000229A422CD100220420FB
:104FB000EA54B0E7022B03D1627B10331621EEE7EF
:104FC000042B0DD1152108226944684606F0ECFA3D
:104FD0000098019902F076FD06F098F93060CAE772
:104FE000052BC8D1152108226944684606F0DCFA71
:104FF0000098019902F066FD06F088F93060627D44
:105000000A231E21CBE7885CA8540132CCE7C046B6
:105010000D1200209012002099120020280000207C
:105020009412002010B5134B04001B78002B01D103
:10503000FFF796FEFFF7FEFD00200F4A0F49104BC9
:10504000545058600130106058680028FCD000208F
:1050500018610130906018690028FCD0094B0A489B
:105060001B785B011B185350FFF7E4FDFFF7C8FDE9
:1050700010BDC0460D1200200010004004050000C5
:10508000FC1000400C1200200E12002010B588B059
:1050900000281DDD0A68012113000B4018D1042AE5
:1050A00016D90F2014682040092811D150683F28D4
:1050B0000EDD9800101880680024084201D04010CE
:1050C000C4B26846C4540133202BF2D1FFF7AAFFC3
:1050D000002008B010BD000010B5002813DD0C68DA
:1050E000E30710D56410532C0DD8084B1B78002B08
:1050F00001D1FFF735FEFFF79DFDA123044ADB0038
:10510000D450FFF77DFD002010BDC0460D120020D9
:105110000010004010B500280EDD0C68E3070BD529
:105120006410FF2C08D8054B1B78002B01D1FFF72A
:1051300017FE034A034BD450002010BD0D1200206F
:10514000001000402405000013B5002814DD0C6891
:10515000E30711D5094B64100093094B0193072C09
:105160000AD8084B1B78002B01D1FFF7F9FD6B46DD
:10517000054A1957054BD150002016BDE2ECF0F45A
:10518000F8FC00040D120020001000400C05000087
:1051900070B588B0002820DD0124086804401CD1C7
:1051A00004281AD90F2302681340042B15D1FEF7E7
:1051B00087F9060006F09EFD0500122800D9122589
:1051C0002A0002210D326846FFF774FD6B465D73BD
:1051D000A54205DC6846FFF725FF002008B070BD3A
:1051E0002300325D6B449A730134F1E7F0B50D0092
:1051F0008BB0012832DD08680122040014402DD153
:1052000004282BD90F2301680B40042B26D16B688F
:10521000134223D0FEF754F96E6807007310019310
:1052200006F068FD05000E2800D90E252A00012190
:10523000113202A8FFF73EFD6A46127902AB5A739B
:1052400002AA73129373019B76141B0ED673137408
:105250005574A54205DC02A8FFF7E4FE00200BB060
:10526000F0BD3A5D02A963189A740134F1E730B5D4
:1052700089B0002814DD0C68E30711D510226846B8
:105280000021FFF717FD6B466A4665105D7368469F
:1052900063122D0E64149373D4731574FFF7C2FE5A
:1052A000002009B030BD0000174B184A596800298A
:1052B00003D00021596001319160196900291FD084
:1052C000002018618023DB00D3581149012B18D12D
:1052D000A923DB00D3585B420B600E490B78032BEC
:1052E00001D801330B7003200B490B7801330340C5
:1052F0000B700A495B015B18094953500123936005
:1053000070470860FAE7C046FC10004000100040FB
:1053100024000020981200200C1200200E12002001
:105320000405000010B5034A1021034800F07EF880
:1053300010BDC04608D70000FFD60000044A05494A
:105340001368C85401339B059B0D13607047C0461A
:10535000C8160020C812002070B5114C114A2368ED
:10536000834202DC0023236016E0155C411C2E0002
:10537000FA3E012E05D899420FDA555C013D1F2DEA
:1053800001D90800ECE70100151A565C6E54013192
:105390008B42FADC181A206070BD1570FAE7C0461F
:1053A000D41A0020D416002010B5FDF7DDFD064B01
:1053B0001A68824201D900221A601B68C31A034886
:1053C00098428041404210BDC4120020204E00008F
:1053D00010B5094C094A23681268934200D110BDE8
:1053E000074AD05CFDF7EEFF0028F8D023680133B0
:1053F0009B059B0D2360ECE7CC160020C81600200F
:10540000C812002010B50400064B074A1B6812683A
:105410009B1ADB439B059B0DA34200DB10BDFFF7EE
:10542000D7FFF1E7C8160020CC16002070B5074E54
:1054300033680B2B08DC0C255D43054C01332851E8
:1054400064196160A260336070BDC046D016002050
:10545000342F002010B5FBF731FEFFF77FF8FBF784
:1054600055FEFDF743FFFEF7FBFBFEF739FCFFF7A8
:1054700059FF00F04FFF01F057F901F0A1FB10BDFB
:10548000962210B512010021034806F0A9F8002267
:10549000024B1A6010BDC0463C1C0020D005002005
:1054A000064B074A1B6812689B1ADB439B059B0D42
:1054B0000122834200DC002210007047C816002041
:1054C000CC160020F8B505000C0016001F1E0ED1EA
:1054D0000320FFF7E5FF002808D0FA20FFF72EFF92
:1054E000E8B2FFF72BFFE0B2FFF728FFF8BD501D31
:1054F000FFF7D6FF0028F9D0FB20FFF71FFFE8B227
:10550000FFF71CFFE0B2FFF719FFF0B2FFF716FF3D
:105510003012C0B2FFF712FF3C00E31B9E42E5DDF4
:105520002078FFF70BFF0134F7E7000070B5002487
:10553000F0250B4B1B68A34202DCFFF7A1FF70BDF7
:105540002B006343074A9B181A78002A05D0597824
:10555000002311201A00FFF7B5FF0134E9E7C04628
:10556000D00500203C1C0020F8B507000024F025E1
:105570002B0063430C4A01349E18B74211D0317896
:1055800000290BD00133D15C002311201A00FFF752
:1055900099FF2A000021300006F022F80A2CE7D1FA
:1055A000F8BD024B1C60F9E73C1C0020D005002030
:1055B000F0B5150001222F00754C1740A54401904D
:1055C0000291002F11D005AB1A706A105A70120E9A
:1055D0001A710522691299706D140299DD70FFF736
:1055E00071FFCF239B009D44F0BD042D1ED90F20D9
:1055F0002A681040042826D1022304AA2800137127
:10560000FDF75EFF040006F075FB624B984200D97F
:105610001800B84204DC421C05AB02990198DEE791
:1056200001377B1EE35C05AAD355F2E7042D00D0B9
:10563000A9E0032304AA043D13716B425D4105AB4D
:1056400055710222E9E709287ED1042205AB1A70C0
:105650006A68511000916946521209789A70009A4E
:1056600059701F2A01DD202200926A46127806AC8A
:10567000DA70009BBB4202DC05ABE21ACDE70126E3
:10568000BB00EB189868064006D1042837D90F21D3
:105690000368194002290CD1012323704310637061
:1056A00042121B0E4014A270E070237105340137C2
:1056B000DFE7042921D102232370FDF701FF0390C6
:1056C00006F018FBA31C0C2809D86070864201D193
:1056D0009C19ECE7039A925D9A550136F6E70C2285
:1056E0006270039A925D9A550136092EF9D12E23E4
:1056F000E372237363730E34D9E7012907D10323BF
:10570000043823704342584160700234CFE70929BE
:1057100009D10423237043685A1062705B12A3708E
:10572000E6700434C3E703290BD105232370006816
:10573000020992B2430F92000B40D31A63701B12FE
:10574000EDE726700134B2E7032800D049E70521D0
:1057500005AB1970110989B2520F890002408A1AEB
:10576000111299705A701100642A00DD642104201E
:10577000D970C9B2041FA14201DC04324DE72C5C90
:105780001C540130F6E7002D00D02AE751E7C0464F
:10579000C4FCFFFF2303000070B502000024F021C9
:1057A0000D4E0800604380194578954203D00134BE
:1057B0000A2CF6D170BDF022002105F011FF074A36
:1057C0001368013BA34200D11460002329001A0092
:1057D0001120FFF777FEEDE73C1C0020D0050020EC
:1057E00010B5B2B002236A460400137006F082FAC4
:1057F000C72800D9C7200023984207DC421C6B460B
:10580000FE211420FFF75EFE32B010BD6946013361
:105810005A1EA25CCA54EFE730B5B3B002236A4601
:105820000500137006F066FA0400C72800D9C724E3
:1058300000239C420BDC20003230FFF7E3FD621CAA
:105840006B46FF211420FFF73DFE33B030BD6946A3
:1058500001335A1EAA5CCA54EBE70000F0B5BBB096
:1058600004900C00012803DC1B20FBF723FD51E012
:105870002A4B08680293C30709D4042807D90F23C9
:1058800002681340042B02D1FDF71AFE0290234B4D
:1058900060680393C30709D4042807D90F2302685B
:1058A0001340042B02D1FDF70BFE039000271C4B85
:1058B0001B680693069BBB420BDC039B194A0093B3
:1058C000C821029B08A806F09DF908A8FFF7A4FFCD
:1058D000CAE70C267E43144B0299F618306806F08E
:1058E000FFF9051E05D17368B6680793079B9D42B3
:1058F00001DB0137DEE730680399059606F0F0F921
:105900000836002808D121000498059B0831023888
:105910005B6898473BB0F0BD0135E7E714D1000064
:10592000D016002064D80000342F0020F7B5234B98
:1059300006001B68F02100930023009A9A4211DCB4
:105940000024F0231A006243019201991C4A551861
:105950002F78002F12D001340A2CF3D11948FFF709
:105960005BFF29E00A005A43154882185078B0427C
:1059700002D11278002A1FD10133DEE7F02239006C
:10598000280005F02DFE02230D4A0199EB605354C7
:105990000D4AF1008A58009B6E70AE70AA602F61AC
:1059A0006F61A34202DC054B01341C60002331000F
:1059B0001A001020FFF786FDF7BDC046D005002075
:1059C0003C1C0020ADDC00009C25002010B5FFF73A
:1059D000ADFDFF24084AE3005B429B18074AD35CF5
:1059E000043B012B03D8E043C0B2FFF79FFF013C0B
:1059F000002CEFD110BDC046FC0700009C25002004
:105A0000F7B50F00FF247F2501901E4AE300D31A4B
:105A10001D4A9A181278062A01D0032A20D1FF22A3
:105A2000D2009B18186883682B401C2B18D1C368C0
:105A30001A002A40042A13D102692A40192A0FD1D8
:105A40001B0A01339B000C30C018FDF739FD0378A9
:105A50000600002B10D006F04DF90023B84209D003
:105A6000013C002CD1D1F7BD019AF15CD25C91428E
:105A7000F6D101339F42F7DCE043C0B2FFF756FF97
:105A8000EEE7C0469C250020FC07000070B505002D
:105A9000FF24084AE3005B429B18074AD35CAB42F1
:105AA00003D1E043C0B2FFF741FF013C002CF0D12D
:105AB00070BDC046FC0700009C250020F7B5FDF72F
:105AC00053FA574B1A68824201D900221A601A68A9
:105AD0005449821A8A420DD9FF2253491860D300D3
:105AE0005248CB1A1B181B78073B022B0CD9013AE2
:105AF000002AF4D1F7BD0720FFF7C8FF4C4B27E081
:105B00000820FFF7C3FF38E0FDF738FA071E00D181
:105B100001270020FDF724FB01900020FDF734FB56
:105B2000019B0090434C444D002B12D02368002B66
:105B30006ED12B682760002B6ED0404B01261B785E
:105B4000002BD8D10920FFF7A1FF394B1E703B4B2A
:105B50001E70009B002B12D02B68002B0FD12368E6
:105B60002F60002B1ED0324B01261B78002BC7D193
:105B70000920FFF78BFF2E4B1E70304B1E702368E1
:105B8000002B0FD02A4E3278002A0BD19F4200D230
:105B900027602368FB1A312B04D90720FFF776FF13
:105BA000012333702B68002B0FD0244E3278002A4B
:105BB0000BD1BB4200D92F602B68FF1A312F04D9BB
:105BC0000820FFF763FF012333702368002B0CD0FC
:105BD000019B002B09D1164E3378002B02D10720F0
:105BE000FFF754FF0023236033702B68002B00D194
:105BF00080E7009B002B00D07CE7104C2378002B23
:105C000002D10820FFF742FF00232B60237071E7C9
:105C1000009A002AA0D1B5E7009B002B9FD1AEE7E8
:105C2000C01200200F2700009C250020FC07000068
:105C3000B4120020B0120020B8120020BC120020C4
:105C400037B500240500FFF771FC01A80194FDF7AA
:105C500075FA21002000FEF72DF9FEF72DFBFDF768
:105C600021FBFDF73BFBFEF773FCFDF7A3F9A54213
:105C700004D0FDF7D1FB0248FFF7CEFD37BDC0468B
:105C80009EDC0000002310B501001A001120FFF770
:105C900019FC10BD07B56B46197069465A7013128E
:105CA0008B701314120ECB700A716B460100052223
:105CB0001320FFF707FC07BD10B50A0001001220F2
:105CC000FFF776FC10BD70B5050008000C003230FF
:105CD000FFF798FB2B00220000211B20FFF7F2FBAF
:105CE00070BD10B50C000300110014202200FFF756
:105CF000E9FB10BD012370B5FF24084A41185B423F
:105D0000884201D3D84370BD06781D0A23407340F2
:105D10009B009B5801306B40F2E7C04680D80000E2
:105D200013B50400FE2813D80A4BC200D05800282F
:105D30000ED0436808309900FFF7DCFF019009207E
:105D4000FFF760FB01AB042221001720FFF7BAFB2D
:105D500013BDC0469C250020F7B50190FEF7AAFDB3
:105D600001250400FF276D42002C01D12800FEBD53
:105D7000266833143B40152B0DD1210001980831C2
:105D800005F0AEFF002801D135123D402000FEF79E
:105D900085FC0400E8E71D2BF8D101256D42F5E7ED
:105DA000F0B580279FB0FFF713FBB24CB24D2068CF
:105DB000FF00391A4019FDF7EBFA23680600C318F3
:105DC0002360002B0ED11FB0F0BD2068391A2818AF
:105DD000FDF7DEFA236806001B182360FDF7C4F800
:105DE000A64B1860002EF0DC2B78FA2B00D002E1D5
:105DF0002368022B07DCFFF7D7FA0028E3D0012045
:105E0000FFF7AAFADFE76878AC78023818281FD8BD
:105E100003F00EFA0D2024282B341E3E707A7E9457
:105E2000CDDE1E1E1E1E1E1E1E1E1E1EEC00FF2C84
:105E30000ED02000FFF7B0FC0022914BE100CA50C9
:105E40005B181A712100009213001320FEF72EFE3A
:105E50000320D5E72000FFF769FDF9E72000FFF7F1
:105E60009BFCF5E7FFF7B2FDF2E7FFF75FFB0020D1
:105E7000FFF7E6FE8348FFF7CFFCE9E7632CE7D89E
:105E8000814BA200D25821001520FFF791FBDFE7DC
:105E9000FEF710FDFF270400002CD9D025682B1435
:105EA0003B40152B04D02000FEF7F8FB0400F3E77D
:105EB0002000083005F01EFF06000530FFF7A2FAAB
:105EC000FB20FFF73BFA2D121D20FFF737FAE8B24F
:105ED000FFF734FAF0B2FFF731FA3012C0B2FFF731
:105EE0002DFA25002B1B9E42DDDD287AFFF726FACE
:105EF0000135F7E700211D2000910B000A00FEF795
:105F0000D5FDFDF789FAA3E72000FFF709FF9FE71A
:105F1000FDF73CF805AC5D4A642100905C4B200025
:105F200005F070FE02232000237005F0E3FE23003D
:105F3000020000211620FFF7C5FA89E70026504A23
:105F4000F3009B181C68002C28D01B79039363680E
:105F500008349F00B81D0293FFF754FAFB20FFF7A7
:105F6000EDF901207D1CFFF7E9F9F0B2FFF7E6F942
:105F7000E8B22D12FFF7E2F9E8B2FFF7DFF9039874
:105F8000FFF7DCF9E719A7420CD8FFF721FA052340
:105F90000298584301F03AFBFFF71AFA0136FF2E38
:105FA000CDD155E72078FFF7C9F90134EBE700249C
:105FB000FFF7BCFA2200210000942300DA20FEF74C
:105FC00075FDFF222100D2002D4805F009FB98E75E
:105FD000012C02D1FEF78CFB3AE7022C02D1FEF72E
:105FE00061FD35E70120FFF72BFE31E7002321009B
:105FF0001A001A209FE7FB2B00D000E72268042A32
:1060000000DCF8E62E79E878224B360206439E4201
:1060100000DDF4E6331D9A4200DCECE6EB5CFE2B7F
:1060200000D0ECE66B78AC78771E1B2B76D019D8B5
:10603000072B5CD0082B31D0012B19D1FF2C17D0A6
:106040002000FFF7A9FB6D79134AB31E00922100CF
:106050002A000A20FEF72AFD094BE400E0501B1934
:106060001D7105E01D2B6BD05DD31E2B00D17EE092
:10607000701DC5E6D41A0020D4160020C4120020DA
:106080009C25002080DC0000942D002097DC00007F
:1060900092DC0000F6030000DA160020632CE7D83B
:1060A0006A79022A13D0032A1BD0012AE0D1E979A8
:1060B000AB79090219432B7AA4001B0419436B7AAC
:1060C0001B060B435B001343324AA350D0E7002F5B
:1060D000CEDDB11E3048FDF713FC2E4BA400E0507E
:1060E000C6E7AB79A4005A1E93419B00ECE7632FEF
:1060F000BEDC05AD3A002949280005F055FA002319
:106100002800EB55FFF728FE0028B1DB214B80006B
:10611000C25821001520FFF74BFAA9E739001F48A4
:10612000FFF76EFCA4E7FF2CA2D06A79022A9FD861
:1061300019490B2000912100B31EFEF7B7FC97E729
:10614000632F00DD6327002305A9BB420ADBFB4365
:106150000022DB173B40CB181A70152000917B1CE6
:106160002100EAE7EA185279CA540133EDE7012C1D
:1061700000D07DE7002F00DC7AE76B79002B03D09D
:106180001C00322B00DD322464235C43044B1C6072
:106190006EE7C046942D0020DA160020D9160020A4
:1061A000040000200122094B1A60094A1368002BE1
:1061B000FCD00322074B1B68D8171040C0180123DE
:1061C00080100638400018437047C04600C00040A9
:1061D00000C1004008C500400120704710B5064CC2
:1061E000200000F023FE0549200000F047FE0122B8
:1061F000034B1A6010BDC0460C1B0020801A06001D
:10620000D81A002010B501210D20FCF7C5FE012190
:106210000E20FCF7C1FE00210F20FCF7BDFE044C50
:10622000200000F03FFD1021200000F057FD10BDC0
:10623000EC1A0020F8B501250C682C4203D10D2082
:10624000FBF738F8F8BD64102DD4FCF7A3FEA0428C
:1062500029DB00212000FCF79FFEFA222900D20052
:10626000200001F005FA00281DD000250027072690
:10627000FA2201219200200001F0FAF9002812D040
:10628000282802DD0123B3401F43013EF0D20E4E09
:10629000AF550135052DE9D1012206210920FDF771
:1062A000B1FA002801D10020CCE70B230124436080
:1062B0000023F25C990052004118224301338A60A6
:1062C000052BF6D1BEE7C046DC1A002010B50468E5
:1062D0000D20E30703D56410FF2C03D91720FAF72C
:1062E000E9FF10BDFFF78EFFE1B2024800F018FD94
:1062F0000020F6E7EC1A002010B5FFF783FF00211D
:10630000034800F00DFD43000120184310BDC046B6
:10631000EC1A002010B5034A09210348FFF786F85C
:1063200010BDC046C4DC00000CDD00000D4B70B594
:106330001B6804000E001500002B01D1FFF74EFF73
:10634000E1B2094C200000F030FEF1B2200000F074
:1063500033FDE9B2200000F02FFD200000F090FE98
:1063600070BDC046D81A00200C1B002010B50124B7
:106370000368234205D04168214202D0826822424C
:1063800003D10D20FAF796FF10BD5810802801D9CF
:106390001520F7E74910FF2901D91620F2E752101E
:1063A000FF2A01D91720EDE7FFF7C0FF0020EBE738
:1063B000F7B501221400904222DD0D682A421FD059
:1063C0001D4B15411B684C68002B01D1FFF706FFE0
:1063D000E9B201272500194E3D40300000F0E5FDEF
:1063E000002D0FD03C413000E1B200F0E5FC300060
:1063F00000F046FE0024A04202D02320FAF75AFF04
:106400002000FEBD042CF2D90F2322681340092B73
:10641000EDD163685B100193019BAB42E7DDAB00FC
:10642000E3189968394204D04910C9B2300000F02D
:10643000C3FC0135F0E7C046D81A00200C1B002031
:10644000154B70B51B6805000E00002B01D1FFF73E
:10645000C5FE124CEDB22900200000F0A6FDF1B2FD
:10646000200000F0A9FC0021200000F0A9FD002878
:1064700001D0404270BD72B601222900200000F018
:106480008FFD62B6200000F088FC0028F2D02000CA
:1064900000F088FCEEE7C046D81A00200C1B002054
:1064A00010B501240368234202D04168214203D180
:1064B0000D20FAF7FFFE10BD5810802801D91520D5
:1064C000F7E74910FF2901D91620F2E7FFF7B8FFD7
:1064D00040002043EFE7000010B50D211D20FFF71D
:1064E000AFFF164C5A2809D101222A2122703D38CB
:1064F000FFF71CFF0122124B1A6010BD0F2119205B
:10650000FFF79EFF332805D102235F22237020214D
:106510001A38EDE70D211E20FFF792FFC7280AD198
:10652000032300222A21A9382370FFF7FFFE1B2234
:106530002A211E20DCE700232370DBE72C0000204B
:10654000E41A0020204B10B51B680400002B01D179
:10655000FFF7C2FF1D4B1B785BB2022B0AD0032B47
:1065600029D0012B2CD121001D200124FFF768FF29
:10657000644205E0012C13D129211920FFF760FFA7
:106580007F2801DD0138FF3803007F3301DA7F20E7
:106590004042C8237F21584302F0DEFE604310BD15
:1065A000032C0BD12B211920FFF74AFF043CE7E70E
:1065B0002D211920D9E721001E20D6E7052CF7D080
:1065C000012400206442E4E7E41A00202C000020AB
:1065D00010B50120FFF7B6FF43000120184310BD9E
:1065E00010B50320FFF7AEFF43000120184310BD94
:1065F00010B50520FFF7A6FF43000120184310BD8A
:10660000144B70B51B68002B02D10120FFF79AFFD5
:10661000114B1B785BB2013301D1FFF75DFF012005
:10662000FFF790FF04000320FFF78CFF0500052013
:10663000FFF788FF6D43644340436419201804F05A
:106640009BFE01F06FFB04F061FE43000120184344
:1066500070BDC046E41A00202C000020F8B50123CC
:106660001C0098422BDD0F683B4228D04E68350055
:106670001D4024D1042E22D90F2231680A40092A54
:106680001DD173685C10202C00DD2024144B1B6886
:10669000002B01D1FFF7A2FD72B67F10F9B2114FA6
:1066A0002200380000F07CFC62B6A54214DA380003
:1066B00000F073FB002804D101246D002C4320005E
:1066C000F8BD380000F06EFB0122AB004000F3186B
:1066D00010439860AD18E8E764000125EEE7C04676
:1066E000D81A00200C1B00200020704701207047A2
:1066F000002070470020704701207047002070473D
:10670000002070470020704700207047002070472D
:10671000002070470020704700207047002070471D
:10672000704770477047000010B5034A0E210348B8
:10673000FEF77CFE10BDC04664DD0000D4DD000025
:106740000378013B1F2B00D970470130F8E710B5E3
:10675000FFF7F6FF0378002B0BD00130222B11D16D
:106760000378002B03D0421C222B03D11000FFF72B
:10677000E7FF10BD5C2B03D14378002B00D0821CB7
:106780001000EDE73A2BF2D02C2BF0D07B2B0BD165
:10679000FFF7D6FF0378002BE9D07D2B01D1013024
:1067A000E5E7FFF7D4FFF5E720225B2B14D1FFF7D5
:1067B000C7FF0378002BDAD05D2BF0D0FFF7C7FFBF
:1067C000F7E7202BD3DD2C2BD3D0190091435D2983
:1067D000CFD0222BCDD001300378002BF1D1C6E7EA
:1067E000002210B5904216D0FFF7AAFF03780422CA
:1067F000222B10D0023A7B2B0DD0013A5B2B0AD012
:10680000190030390232092905D92D2B05D14178DB
:10681000303909290AD8100010BD0522742BFAD08E
:106820000132662BF7D001326E2BF4D0581E834113
:106830005A42F0E770B5FFF783FF037801222D2B52
:1068400001D18018023A00230A2502E06B4301308F
:10685000CB1801783039CCB2092CF7D95A43100043
:1068600070BDF8B50C001500FFF76AFF0378222B06
:1068700002D000232370F8BD0D236A1E21000825D5
:106880000C260A279C4601300378222B02D10023D4
:106890000B70F0E7002BFAD0441C5C2B0BD1437833
:1068A000841C622B0ED0662B0ED06E2B0ED0722B5A
:1068B0000ED0742B0ED0002AE9DD0B70013A0131A5
:1068C0002000E1E72B00F6E73300F4E73B00F2E7B6
:1068D0006346F0E70923EEE710B50400FFF737FF42
:1068E000A04202D90378202B00D910BD0138F7E768
:1068F00010B5002815D00378002B13D0FFF720FF28
:106900002021037802008B4300205D2B09D010006A
:10691000FFF71DFF03782C3B5A425341C018FFF785
:106920000FFF10BD1800FCE70300002070B50C003D
:1069300081420EDD1A785B2A0BD1581CFFF700FF4D
:106940000125AC4205D0FFF7D3FF002801D0013567
:10695000F7E770BD70B50C001500002901D00023C9
:106960000B70002820D00378002B1ED0FFF7E8FE24
:10697000037806002C2B03D10130FFF7E1FE06005F
:10698000337800207D2B0FD0844204D02A002100D0
:106990003000FFF766FF3000FFF7D9FE03783A2B8F
:1069A00002D10130FFF7CCFE70BD1800FCE7F0B556
:1069B0000D0004009DB02E78002E35D02E21280029
:1069C00005F080F9071E14D0431B0193303E092EB9
:1069D00014D82800FFF72EFF01002000FFF7A4FFC6
:1069E0000400002C20D0002F1ED0019B0133ED1895
:1069F000E1E7280005F07EF90190E7E723787B2B9B
:106A000011D1601C642203A9FFF7A4FF041E0BD060
:106A1000019A290003A805F074F90028E1D02000AC
:106A2000FFF795FEEEE7002420001DB0F0BD70B525
:106A3000050000200C0081421DDD2800FFF7D0FE7C
:106A40000300681C012B14D00020022B13D100225C
:106A5000681C1100FFF77EFF012C0CD0FFF748FFE8
:106A600000221100FFF776FF013CF5E7FFF740FF3A
:106A7000013C012CFAD170BDF8B5050000200C00D6
:106A800016001F0081420DDD2800FFF7A9FE03005C
:106A90000020022B06D1681C3A003100FFF75AFF94
:106AA000012C00D1F8BDFFF723FF3A003100FFF7BA
:106AB00051FF013CF4E710B50024A04218D0FFF7C5
:106AC0003FFE03787B2B0AD1013000221100FFF733
:106AD00041FF00280CD0FFF73AFE0134F5E75B2BAD
:106AE00006D10130FFF704FF002801D00134F9E797
:106AF000200010BDF8B5002816DD0D68EB0713D592
:106B00006D10013D0124FDF7D5FE0026FF276442EC
:106B100000280CD1002E21D0300005F0EBF8010048
:106B20003000FCF7EDFEF8BD01256D42EAE7036891
:106B30001A143A40152A0BD11B123B409C4200DA32
:106B40001C009D4201D106000836FDF7A7FDDFE7D6
:106B50001D2AFAD1012400266442F6E701200134FF
:106B600064002043DFE7000010B508680C00FCF764
:106B7000A7FCFFF7F1F8002803DB6268024B8000F6
:106B8000C250002010BDC046942D002010B50868EA
:106B9000FCF796FCFFF7E0F80123002802DB024B2C
:106BA0008000C358180010BD942D002010B508684F
:106BB000FCF786FCFFF7D0F8C043C00F800010BD83
:106BC00010B5034A04210348FEF730FC10BDC0464F
:106BD00064DE00005DDE000010B5FCF793FBFCF7FF
:106BE00041FCFEF737FC0448FEF716FEFDF7C0FF38
:106BF000FEF7ECFE10BDC046B3DE000010B5FCF79A
:106C00008BF810BD70B5002504AC24780573A9423B
:106C100005D10A4B0A4A23210A4804F057FC0160B7
:106C20000949920052589B0002715B58A40083717D
:106C30006358856043710223C37170BDCBDE0000D1
:106C40002ADF0000D9DE000088DF0000037B002B74
:106C500004D14373837303610133037370470000EE
:106C60001FB50191A02100240068C900D2B2445090
:106C7000012A10D0A24209D0032A0AD0074A835021
:106C8000074B019AC250012343501FBD02221343F8
:106C9000F4E70422FBE70622F9E7C04654050000AA
:106CA0002405000010B50400FFF7D0FFA1222368DF
:106CB000A179D20099506179064A20009950217932
:106CC00004329950044B19685A689B68FFF7C8FF53
:106CD00010BDC0460C050000001B00204BB2002B6D
:106CE0000FDB80233F290FD81F290FD80F290FD87A
:106CF00007290FD803290FD81B060168074A8B50B4
:106D0000704780239B04F8E7DB04F6E71B05F4E7F4
:106D10005B05F2E79B05F0E7DB05EEE724050000E5
:106D20000368074A99501A00FC32D1680029FCD048
:106D3000A321C90058580023C0B2D3607047C04691
:106D40001C05000007B58022074BD2051A600022FF
:106D50009A6002321A710F230C3200930349023BEE
:106D60000348FFF74FFF07BD001B00200030004025
:106D7000EC1A0020F8B505000E0017000024BC42F4
:106D800008D02B68315D1B6828009847002801D087
:106D90000134F4E72000F8BD704710B51C3000F056
:106DA000A9F910BD10B51C3000F096F910BD10B552
:106DB0001C3000F0A5F910BD70B5437E0D00002B0E
:106DC00001D1002070BD6430040000F0A2F9002859
:106DD000F7D12000290000F070F90120F2E700004F
:106DE000F7B50193FA23002504009B0083600D4B47
:106DF0004560083303601C300F00160000F052F9A4
:106E00002000643000F04EF9074A2761B600B358FD
:106E100020006375019B9B009B586576A576A37542
:106E2000FEBDC04668DF000088DF00000123A0220D
:106E3000C375837D0E49C133FF33D2059B00995042
:106E4000437DC133FF339B009950CC220169094B2C
:106E50005204CA5005220169243BCA50827D01694F
:106E60000833CA500269417D034BD1507047C04678
:106E70000C060000240500000C050000A0220023E1
:106E800010B50469D200A3500A4CA1420FD90A4C94
:106E90008C425B4109495B420B40CD21C9045B1820
:106EA00004690749635005210369995010BDCC233B
:106EB0005B04F5E7A086010090D00300000098FD78
:106EC00024050000F7B5040000200D000193824264
:106ED00065D01600402A00D9402627001C3738000C
:106EE00000F0F6F8B1232269DB00D550802201239F
:106EF000216992008B50A27E002A03D1226913627D
:106F0000226913600025731EAB4207D1019B002B41
:106F100004D0802202212369920099500122236922
:106F20001A622369FC33DA68002A02D19A6A002ABD
:106F3000F9D09A6A002A0BD1DA60A3232269DB0018
:106F4000D1583800C9B2013500F0B7F8B542DAD3EC
:106F5000019B2269002B0FD11300FC339B6A002B8D
:106F60000AD10133A376D3612369FC33DA6C002A9A
:106F7000FCD00022DA640AE000230121A3765161EB
:106F80001A002369FC3399680029FCD09A602369B0
:106F9000FC339A6A002A01D000229A62E8B2FEBD50
:106FA00010B50123FFF78EFF10BD0300AC3310B501
:106FB00004001970643000F08BF80123637610BD73
:106FC0000023020070B5AC3243760D001178B12277
:106FD00004000069D20081508022216992008B5008
:106FE00022690133136222699360260064363000FF
:106FF00000F080F8002812D0300000F06DF81E4B31
:107000002269D0502369FC331A6A002A02D19A6A95
:10701000002AF9D09A6A002A01D11A62E5E72369A9
:107020000122002D0DD11900FC31896A002908D1F7
:10703000DA612369FC33DA6C002AFCD00022DA64BE
:1070400007E05A612369FC339A68002AFCD00022C9
:107050009A6000202369FC339A6A82420BD09862BE
:107060002169064A8B588B501800022B03D0181F39
:10707000431E9841033070BD1C050000C40400008D
:1070800010B50121FFF79CFF10BD000010B51323C0
:10709000142202490248FFF7A3FE10BD0040004041
:1070A0000C1B002010B540220021040004F098FAC7
:1070B000002320002364636410BD10B53F24026CDC
:1070C000531C2340446C9C4201D08154036410BD86
:1070D0000023036443647047436C026C934206D000
:1070E0003F21C25C01330B40436410007047012014
:1070F0004042FBE7036C406C181A00D540307047E3
:10710000436C026C934201D0C05C70470120404246
:10711000FBE73F22036C406C01331340181A4342D3
:107120005841C0B27047000003210A4802680A4370
:107130000260094802680A4302600849084A094B8C
:107140009B1A03DD043BC858D050FBDC00F012F85A
:10715000F8F7DAFF2405004054050040DCE40000A5
:107160000000002068020020FEE7FEE7FEE7FEE7E1
:10717000FEE7FEE72D4B10B51A68D2B2012A0FD1F7
:107180002B4A126812070BD12A4AE0241168F02218
:107190000800104021422DD12749096811422CD006
:1071A0001A68D2B2012A12D12149096809070ED101
:1071B000F020204909680140402908D11E4909688A
:1071C000014204D18020C121C005C90042501B6882
:1071D000DBB2012B0DD1164B1B681B0709D1154BD8
:1071E0001A68F0231A40A02A0FD1134A12681A42D3
:1071F0000ED010BD3028CFD0D2E7104A1049116010
:107200008021104A09021160CAE7D02AF1D1ECE7C7
:107210000D4B1A68012A04D00C4A1A601A68012A18
:10722000FCD1C0220A4B1A60E3E7C046E00F00F031
:10723000E40F00F0E80F00F0EC0F00F00405004050
:10724000DFFF07C0186C004000EC0640759300009B
:1072500014EC06400120704710B503681322DB6967
:10726000984710BD70470000054B0269D150036973
:10727000FC331A6A002AFCD0002201201A627047EF
:107280001C050000030010B55C331A781F231A4058
:107290001E3B19009140114AD167C22204210469A2
:1072A0009200A150026953600269D360A0230022BA
:1072B0000169DB00CA5001230169094A5B428B5016
:1072C0000169084A8B5001690C3A8B5001690832F8
:1072D0008B501430FFF7FCFE10BDC04604E100E007
:1072E0000C0500001405000010B51430FFF702FF74
:1072F00010BD10B51430FFF703FF10BD10B51430EA
:10730000FFF7EAFE10BD0000030070B55E331A7887
:107310000469724BE25003005D331A780469704BC4
:10732000E250030061331C7802696E4B012C00D0DF
:107330009EE005005F352E78A225ED005651020033
:1073400060321578A1220669D200B5500269D45086
:107350009623DB00994200D88CE096231B019942CA
:1073600000D88AE096235B01994200D888E09623F2
:107370009B01994200D885E0E1239B01994200D806
:1073800082E09623DB01994200D880E0E123DB0113
:10739000994200D87DE096231B02994200D87AE0FA
:1073A000E1231B02994200D877E096235B029942C1
:1073B00000D874E0E1235B02994200D871E0E12338
:1073C0009B02994200D86EE0474B994200D86CE08E
:1073D000E123DB02994200D86AE0E1220023120394
:1073E0008A425B41414A5B421340802252059B180E
:1073F00001693F4A8B50A02304220169DB00CA5077
:1074000000210369FC33D9600369FC33196201234D
:1074100001690B6001698B60C121046989006250B8
:107420001F215C3002780A4093406231314AFF31BB
:1074300053500021415600293CDA0F230B40083BF2
:107440002D4C9B089B001B1903242140A140FC34B8
:107450008C40DD69A5432C00C0258D4029002143C7
:10746000D9611F23017819401E3B8B40136070BD0A
:1074700000246CE79E23DB02BAE79D231B03B7E7DA
:107480001E4BB5E71E4BB3E7EC239B03B0E71D4B48
:10749000AEE71D4BACE71D4BAAE71D4BA8E71D4B04
:1074A000A6E71D4BA4E71D4BA2E78023DB049FE763
:1074B0001B4B9DE78C080F4BA400E41803230B40E3
:1074C000FF21C025DB009940AD0066598E43310095
:1074D000C0269E4033000B436351C2E70C050000F9
:1074E000140500006C05000090D0030000D0BEFE23
:1074F0002405000000E100E000ED00E000B0130012
:107500000050270000A04E0000F0750000509D00C4
:1075100000F0EB0000903A0100E0D70100B0AF03AB
:1075200000705F07F7B5009308AB1B780025019347
:10753000FA2304009B0083600E4B45600833036010
:1075400014300F001600FFF7ADFD23005C332761F8
:107550001E70009B084A9B00995823005D331970E8
:10756000019B20009B009A5823005E33DD701A7047
:10757000FEBDC0460CE0000088DF0000036910B5C6
:107580001A00FC32D2680400002A0AD0A322D200DA
:1075900099581430C9B2FFF790FD00222369FC33DB
:1075A000DA6010BD10B50248FFF7E8FF10BDC04615
:1075B000C41B0020162307B5022200930249013B99
:1075C0000248FFF7AFFF07BD00200040C41B0020AA
:1075D00010B5002801D004F0BFFA10BD0849094ACF
:1075E000094B10B51B688858FA22190A1B06184364
:1075F0009200002301F0E8FF4904C00B084310BDCE
:107600000010014004050000281C002070B5041E75
:1076100009D0FFF7E3FF050000F014F8FFF7DEFFE5
:10762000401BA042F8D370BD0022044B9A60044A6C
:1076300013680133DBB213607047C046FC10014091
:10764000281C00207047704710B500F05FF8FFF766
:10765000FAFF0120FFF7DAFFFFF7BEFAFFF7CEFAD5
:10766000024B002BFAD000E000BFF7E7000000005B
:10767000F8B54C1EA1410126114D86404C422868A8
:107680001049170001F0DEFD0D21784301F0DAFD0D
:1076900034400300220031000B4800F019F80028A4
:1076A0000DD0FA23FA21094C9B0144438900286834
:1076B000E41801F0C7FD0100200001F0C3FDF8BD92
:1076C0003000002040420F0010050050C83200007A
:1076D00030B504680C40944206D1013B002BF8D130
:1076E00012E0013B002B0FD004680C409442F8D10B
:1076F000002405680D40954204D101349C42F8D124
:10770000002002E0201C00E0181C30BDC420114BFA
:1077100080001A5810491140C02212020A431A5020
:10772000C0218022490092025A501A608023A3226D
:107730000021DB05D20099500122F9309A60074BF5
:10774000FF301950C12002318000195040301950CB
:107750001A60704700E100E0FF00FFFF00100140E9
:10776000014B18607047C0467C000020F7B500232D
:1077700020285AD8384B8000C258042A5BD007D83A
:10778000022A54D055D80423012A09D000234CE002
:10779000062A54D051D31A2A53D002231B2AF5D1DA
:1077A0002E4A116808294ED909294FD00A240226E9
:1077B000A02001252A4AC00015502A482A4D0768F2
:1077C0001C20BF00074029480197006857590090C6
:1077D00027481B0207401F43C02300989B02034019
:1077E000FF2057515759000207401F43019B1F4379
:1077F000009B58016023184007433E435651012522
:107800001C4B156058680028FCD000205860A1234C
:107810000125DB00D3585560A025ED0050511BB267
:10782000A14202D015D2611ACB401800FEBD082338
:10783000B6E71023B4E72023B2E74023B0E7802364
:10784000AEE70123ACE708240026B1E70C000126CF
:10785000AEE7091B8B40E8E788DF000078000020D6
:1078600000700040340000200405000038000020B3
:10787000FF00FFFFFC700040F0B520285BD8364BBE
:107880008000C258354B1E68002E30D1C227344BC1
:10789000BF00D859334C03250440C02000022043C8
:1078A000D851C02480206400800018512E4F1860E9
:1078B0002E4B803CD859FF3CA043D8510437D859AF
:1078C000A8432043D8510837D8590C35A8438446DB
:1078D000072065462843D851A820C0001E50C1206B
:1078E0008026800076021E501C601C4B1C601425F4
:1078F00000202B001E4C2E0046433659771C1BD10E
:107900004343E250A0230325C132FF329200DB053E
:10791000D550184B1A68082A14D114234343E3188E
:107920009A6812485132FF32920059601150DA6859
:10793000C1239B00C250F0BD9642E1D00130032824
:10794000D9D1F8E7082A02D9083AD140E5E7082357
:107950009A1A9140E1E7C04688DF00002C1C002005
:1079600000E100E0FF00FFFF040500000090004080
:107970003C0000207C0000202149F0B54A6C2148E1
:10798000002A14D0A025A12600230124ED05F6002D
:10799000C258571C06D0C7187F68002F02D0270096
:1079A0009740AF5114333C2BF2D100234B64A023FA
:1079B0000121DB0500260F009C4614234B43C3180E
:1079C0001A1F1268104C0E4D920014195219526C65
:1079D000002A10D01A00143A1268551C09D0103B26
:1079E0001B68FF2B05D03B00934065461A00074BF0
:1079F000EA50FC34666401310429DED1F0BDC04692
:107A0000FC9000403C000020009000400C0500006D
:107A100000B5202810D80C4A8000835803290BD8C1
:107A2000A0220800C133FF33D2059B0001F000FC07
:107A3000020905070021D15000BD0C21FBE70421FC
:107A4000F9E70321F7E7C04688DF000020280AD8BD
:107A5000074B8000C25801239340A022D205002981
:107A600002D1044953507047A121C900FAE7C0462A
:107A700088DF00000C05000003000020202B0AD83E
:107A8000A021A222C905D2008858034A9B009B5816
:107A9000D84001231840704788DF0000F7B5060082
:107AA0000D000C008B180193019B671B9C4207D0B3
:107AB000336821781B683000984701340028F3D1DF
:107AC0003800FEBDF0B5C64600B5CB0F9846404A1B
:107AD0004B005B0D9A1882B00D000400132A2FDCB6
:107AE000002A49DB3B4F17413E000E40064323D09E
:107AF0007F08390029400C430AD03749BD438C46E2
:107B000063445C425C418023DB021341E4071D4374
:107B10004146CE0031492B008E1922003468756829
:107B20002000290001F0F6FE0090019100980199D3
:107B300022002B0003F086F802B004BC9046F0BD92
:107B4000332A08DD8023DB009A42F5D102000B00C6
:107B500001F0E0FEF0E7224A9446012263445242DB
:107B6000DA400242E8D052080242D1D09443802247
:107B7000D2051A411443CBE74B005B080343DBD02B
:107B80000B031B0B1C436342234380244D0C240333
:107B90001B0B23406D042B4319004346DA000F4BA7
:107BA0009B181C685D6802000B002000290001F092
:107BB000B1FE009001910098019922002B0003F082
:107BC00041F842464B005B08D60733431900B3E740
:107BD00001FCFFFFFFFF0F00EEFBFFFF40E0000096
:107BE000EDFBFFFFF8B5274A4B005B0D9A180C0020
:107BF0000700132A10DC002A36DB234B13410B420B
:107C00003AD0802424031441002064189C430600C9
:107C1000250030002900F8BD332A0EDD8023060040
:107C2000DB000D009A42F4D102000B003800210065
:107C300001F070FE06000D00EBE7144D0600AC46A7
:107C4000012563446D42DD40AC4663460D000342AE
:107C5000DFD033239A1A323B93401818874200D959
:107C60004C1C63469843D2E7C90FCC070020531C35
:107C7000CDD1074B1C43CAE706000D000028C0D138
:107C8000C7E7C04601FCFFFFFFFF0F00EDFBFFFF52
:107C90000000F03F30B5214A4B0087B05B089342AB
:107CA0001EDD1F4A934205DD02000B0002F0CAFFF1
:107CB00007B030BD02AA00F095F803231840049ADB
:107CC000059B012813D002281DD0002814D002984B
:107CD000039900F06FFB80231B069C466144E7E795
:107CE000002300220093002301F0DEF8E0E7029871
:107CF000039900F05FFBDBE70124029803990094ED
:107D000001F0D2F8D4E7012402980399009401F01D
:107D1000CBF880231B069C466144C9E7FB21E93F61
:107D2000FFFFEF7FF0B54746CE4680B58DB004002B
:107D30000D0000F067FA294B06001B780F005BB2BC
:107D40009846013310D022002B002000290003F0B8
:107D5000C1FA8146002807D1002200232000290013
:107D600001F00AFC002806D1300039000DB00CBC2F
:107D700090469946F0BD01230293194B069407954E
:107D800003934B460A93434604940595002B15D064
:107D9000002300221900100002F0D8F84346089092
:107DA0000991022B0ED103F0AFFB212303600A9B44
:107DB0000193002B0CD1089E099FD5E700230024D6
:107DC0000893099402A801F0C1F90028EFD1EAE76D
:107DD00003F09AFB0A9B01930360ECE7800000200C
:107DE00050E00000F0B54E464546DE465746E0B549
:107DF000E14B4C008FB09046894664089C4200DC01
:107E000087E0DE4B9C4222DCDD4A002900DC92E068
:107E1000DC4B02F017FFDB4B06000F009C4200D149
:107E20007EE1D94AD94B02F00DFF02000B0041461A
:107E300030000A604B60390002F004FFD34BD24A95
:107E400002F000FF434601259860D9606BE0D04BFB
:107E50009C4200DC8FE0CF4B9C4200DD55E1CE4AD6
:107E6000231592469A4451460905631A19001D00CC
:107E7000040003F04BFA03F07FFA02000B0020002D
:107E800029000892099302F0DDFE0022C34B02F0A4
:107E900067FC0F00060003F039FA03F06DFA0400E6
:107EA0000D0002000B00300039000A940B9502F01F
:107EB000C9FE0022B94B02F053FC002200230C90B3
:107EC0000D9101F053FB002800D192E10023002224
:107ED0002000290001F04AFB434243410133B04AEC
:107EE00041460192022208A80092524600F07CFB13
:107EF0004B460500002B16DA8022434612069446B4
:107F000042465B68454263445360D3686344D36030
:107F100009E00B00020041460A604B60002200238A
:107F200000258A60CB6028000FB03CBC9046994683
:107F3000A246AB46F0BD934B01F0ECFC914B060022
:107F40000F009C4200D13DE18F4A904B01F0E2FCD2
:107F500002000B00414630000A604B60390002F01D
:107F600071FE894A894B01F0D5FC012543466D42DB
:107F70009860D960D7E701F049F88A4A8A4B060031
:107F80000F0002F0EDFB0022884B01F0C3FC03F070
:107F9000BDF9050003F0F0F9794A7A4B0490059198
:107FA00002F0DEFB02000B003000390002F04AFE56
:107FB000754A06000F0004980599744B02F0D0FB37
:107FC000029003911F2D00DCC7E0029A039B300052
:107FD000390002F037FE83468A4653465B0024157B
:107FE0005B0DE31A102B6CDD04980599D322674BC7
:107FF000520502F0B5FB02000B003000390002927E
:10800000039302F01FFE0A0001001300069107927D
:1080100002003900300002F015FE029A039B02F0C4
:1080200011FE06000F0004980599614A614B02F0A9
:1080300097FB32003B0002F005FE069E079F0B00F7
:108040000200390030000292039302F0FBFD4B0066
:108050005B0D83468A46E41A312C32DD049805997B
:10806000B822544B920502F07BFB03000C00020087
:10807000029303940B000698079902F0E3FD0200B7
:108080000B0006000F000698079902F0DBFD029A2C
:10809000039B02F0D7FD484A02900391049805998A
:1080A000464B02F05DFB029A039B02F0CBFD0200FF
:1080B0000B00300039000292039302F0C3FD8346A7
:1080C0008A465A465346414630000A604B603900A2
:1080D00002F0B8FD029A039B02F0B4FD44460B0087
:1080E0000200A260E3604B46002B00DB1BE75B460F
:1080F000236080231B065344636080231B069C4639
:108100006144A060E1606D420DE70B00020002F0E7
:1081100099FD434600259860D9601860596002E7D0
:10812000D3221A4B520502F08DFD214A214B0D003E
:10813000040002F087FD02000B00414620000A60A7
:108140004B60290002F07EFD1A4B194A02F07AFDBD
:10815000434601259860D960E5E602000B00300037
:10816000390002F06FFD6B1E154A9B009B58834639
:108170008A46A342A5D130E7FB21E93F7BD90240E3
:1081800000004054FB21F93F3163621A61B4D03DD5
:10819000FB213941FFFFEF7FEAFBFFFF0000704149
:1081A000D8E0000083C8C96D305FE43F0000E03FC5
:1081B0007370032E8A19A33BC14920259A837B390A
:1081C00058E00000D3220C4B520501F0A3FB0B4AF0
:1081D0000B4B04000D0001F09DFB02000B0041461B
:1081E00020000A604B60290002F02CFD034A044B7A
:1081F000B9E6032373E6C04661B4D03D7370032E25
:108200008A19A33BF8B54746CE46674B80B50A00AE
:108210000F00190005003940994200D19BE004008D
:108220000100002F69DD3F1500D1B4E05F4B120360
:108230009C468023120B5B0313435B00CA0F674409
:108240009B184A00F80703D5D20F5B009B188A00E1
:1082500079108C46002180201624894680030D1851
:108260009D4202DC29185B1B8144D50F5B00013C59
:108270005B1952004008002CF1D10020804680207C
:1082800020250027000609E08B425CD0D40F5B005C
:10829000013DE31852004008002D16D0C4198B424E
:1082A000F2DD27180E00002C49DB5B1AA24289413F
:1082B00049425B1A121BD40F5B00013D8044310020
:1082C000E31852004008002DE8D113434ED1434635
:1082D0005B0837494A468846494652104244C90716
:1082E00002D5802109060B4361460F05BD18180011
:1082F00029000CBC90469946F8BD7B005B080343FF
:108300003900002BF5D0002F3CD1E30A153A640563
:10831000002BFAD08020400303423FD1002700E029
:108320000F005B00791C0342FAD0250020208D400D
:10833000401A2900D71B2200C2401A4376E7FE43A9
:10834000F60F8E19B1E79442A0D82718002CF6DB5F
:108350001E000023AEE702003B002800390002F0B7
:10836000FFF92A003B0001F0D5FAC2E7434601338A
:1083700003D0434601335B08ABE701239846002353
:10838000C144A6E73B00020002F05CFC02000B00C7
:1083900001F0DCFDADE713000022BBE7012721005F
:1083A00020207F42C6E7C0460000F07F01FCFFFFAF
:1083B0000000E03FF0B54746CE4680B587B000925A
:1083C0000193754B4F00814688467F089F4263DCCE
:1083D00002F09CFF002800D1D4E04A4643464846BC
:1083E000414602F0BDF904000D006C4A6C4B02F0EE
:1083F000B7F96C4A6C4B01F08DFA22002B0002F0A9
:10840000AFF96A4A6A4B02F01DFC22002B0002F011
:10841000A7F9684A684B01F07DFA22002B0002F0B0
:108420009FF9664A664B02F00DFC22002B0002F019
:1084300097F9644A644B01F06DFA22002B0002F0B8
:108440008FF9029003910022604B2000290002F076
:1084500087F9029A039B06000F002000290002F012
:108460007FF9009A019B04000D004846414602F046
:1084700077F902000B002000290002F0E3FB020064
:108480000B003000390002F0DDFB02000B00002081
:108490004F4902F0D7FB70E002000B0002F060F9D8
:1084A00004000D003D4A3E4B02F05AF93D4A3E4B56
:1084B00001F030FA22002B0002F052F93B4A3C4B0B
:1084C00002F0C0FB22002B0002F04AF9394A3A4B75
:1084D00001F020FA22002B0002F042F9374A384B13
:1084E00002F0B0FB22002B0002F03AF9354A364B7D
:1084F00001F010FA2B00220002F032F9354B029005
:1085000003919F429FDD344B00229F423DDC334963
:1085100000207B182E4916001F0002F093FB0490E8
:1085200005910022294B2000290002F019F93200A0
:108530003B0002F087FB029A039B06000F0020001D
:10854000290002F00DF9009A019B04000D00484635
:10855000414602F005F902000B002000290002F05C
:1085600071FB02000B003000390002F06BFB0200CF
:108570000B000498059902F065FB07B00CBC90460F
:108580009946F0BD00201249F7E7154B00260492EA
:108590000593144FC5E7C046FFFF3F3ED43888BE61
:1085A000E9FAA8BDC4B1B4BD9EEE213EAD529C8097
:1085B0004F7E923E9015CB19A001FA3E7751C1161D
:1085C0006CC1563F4C5555555555A53F0000E03FF1
:1085D0000000F03F3233D33F0000E93F0000E0FFEE
:1085E0000000E73F0000D23FF0B5DE464E4645466C
:1085F0005746E0B5DC4CA5440D9114001900A49A2F
:108600000993DA4B9200D6584D1E03901821E01EB4
:108610000696029500F0A0FEC3430100DB17194047
:108620004B1C9A009B1ADB001B190B9105934C1BEA
:10863000771918D4A59BA5009C463F1922AE654426
:10864000013707E0286802F097FE013403C60435BD
:10865000BC4208D0002CF5DA00200021013403C60A
:108660000435BC42F6D1069B002B01DA00F0FDFB7D
:10867000069B03990133DB009A46099BDA00944676
:1086800000920022914672AA0492B94A614493462C
:1086900088469AAB63449B44029B002B00DABCE102
:1086A0005D4600260027039C4D442A686B6803CC76
:1086B00002F056F802000B003000390001F02AF9F0
:1086C000083D06000F004445EFD1049B4B441E605B
:1086D0005F6008239C46E144D145DDD10EA804210A
:1086E0008446494261448C46069A93009C44614604
:1086F00084460A910399083B63448C460C93009B83
:10870000009263449B46009A0498D10003008C4673
:10871000634408911E685F68002A33DD95498046EE
:108720008C466244D300984470AB9A460EAB99468F
:108730000022914B3000390002F012F802F0E6FD01
:1087400002F01AFE00228D4B04000D0002F008F822
:1087500002000B003000390002F074FA02F0D6FD7E
:108760004B4601C39946434620001A685B682900BE
:1087700001F0D0F808235B429C46E04406000F005D
:10878000D045D5D1059B30001A003900984600F03D
:10879000DFFCFF2300229B0504000D0001F0E0FF39
:1087A00000F038FC0022764B01F0DAFF02000B00EB
:1087B0002000290002F046FA0D00040002F0A6FD98
:1087C000814602F0D9FD02000B002000290002F0D2
:1087D00039FA060040460F00002800DCEEE0009B5E
:1087E00018215A1E92000EAB9B58091A1D000D410C
:1087F000A9448D405D1B0EAB9D5017231B1A1D41D4
:10880000002D2DDD01239C46009BE144002B00DC64
:108810001CE20E9C0123002C00D0B5E0009A012A36
:1088200009D099000EAA54580133002C00D0ACE0B6
:10883000009A9A42F5D1059B002B0EDD012B00D149
:10884000A8E1022B09D1009B0EA95A1E92000EAB83
:108850009B5807939B029B0A8B50022D00D1C1E0CD
:10886000002300223000390000F080FE009B002829
:1088700000D194E2069A591E8A4210DC414A0A98B5
:1088800094460EAA6344944600229B0063441C68ED
:10889000043B22438342FAD1002A00D0C0E0069B69
:1088A0000EAA013B9B00D358002B00D0B3E001225D
:1088B0000C9B043B596801320029FAD0009B9C466E
:1088C0006244110007921A0001338B4246DC0B9878
:1088D00063468046A59C4344A046099C9B00A14654
:1088E0004A449844D30022AA9146049A9944944653
:1088F000089BA59A63448446614494469A468B003B
:10890000634400934346586802F036FD4B461860B6
:108910005960029B002B24DB4D46039C0026002758
:1089200001E0286869680CCC01F01AFF02000B0016
:108930003000390000F0EEFF083D06000F005C45F6
:10894000EFD153469E60DF6004239C460433E0442D
:108950009C46009BE144E2449845D3D1079B009399
:10896000D1E600260027ECE794FDFFFF20E200009F
:1089700018FEFFFFFFFFFF1F0000703E0000704168
:1089800000002040FFFFFF3F002180225204141B03
:108990000EAA5450009999420EDD0EA884469B0001
:1089A0000EAA8900D25861446344CF4800E01A6897
:1089B000821A04C38B42FAD101243CE7059B002BA9
:1089C00006D1009B0EAA013B9B00D558ED1517E779
:1089D0000022C64B300000F0EDFD002800D024E15D
:1089E00000253DE732003B000020C14902F02AF992
:1089F00006000F00002C00D132E7059A0020BC4988
:108A000000F0A6FB02000B003000390002F01AF95A
:108A100006000F0024E7012250E70026002754E655
:108A20004B46059A079388468B000EA9CB58183AF7
:108A300008950592002B0DD18C464146AD4B434421
:108A40009B006344043B58680139183A0028F9D068
:108A500088460592059A0020A54900F079FB434617
:108A600004000D00002B00DA05E29E000EAB9C46D0
:108A70004346DB0066449C46059370AB9946049FD1
:108A800067440097306802F077FC22002B0001F069
:108A900067FE002238607960974B2000290001F0C2
:108AA0005FFE083F04000D00043EB945EAD14AAB21
:108AB00003939B4600239A46069B424699464346AB
:108AC0000132029204934B46002B00DAAAE0802088
:108AD0008A4B009D9846C00589490026002700243E
:108AE00008E008239C460835E044544511DC434621
:108AF000186859682A686B6801F032FE02000B00A2
:108B00003000390000F006FF013406000F00A145D7
:108B1000E7DA5B46C0C39B4601239C46009BE244C8
:108B2000083B0093029B9A45CDD1049B9846A49B99
:108B3000022B00DD8EE0002B37DC1FD1059B0027C8
:108B40001D00039B00249C461E006544083E2A68C5
:108B50006B683800210000F0DDFE083D07000C00C6
:108B6000AE42F4D1089B002B03D080231B069C4609
:108B700064443A0023000D990A604B600720079B6C
:108B800018409B239B009D443CBC90469946A246BE
:108B9000AB46F0BD009B0EA95A1E92000EAB9B582F
:108BA00007935B025B0A8B5057E64346002B00DAC3
:108BB00070E100200021DB004AAAD61848AF3268D5
:108BC0007368083E00F0A6FEB742F8D1089B002B60
:108BD00000D025E10B0002004A984B990D9C2260C1
:108BE000636002F02FF8434607000C00002B13DDF2
:108BF00001254CAEB14638002E0021004C4601360E
:108C00000CCC00F087FEA146B045F7DA089B0700C0
:108C10000C00002B00D015E13A0023000D998A606A
:108C2000CB60ABE70026002773E701239C46009B3F
:108C3000E1440225002B00DDEBE532003B00002083
:108C40002B4901F0FFFF06000F0009E60024F2E5C2
:108C50004AAB0393A49B032B00D08FE74346002B22
:108C600000DC14E1039ADB009B46130091465B4451
:108C70001E685F68234B43440293DB00994448AB72
:108C80009A464B465C681B681800210032003B0086
:108C90000090019100F03EFE04000D0002000B0068
:108CA0000098019901F0CEFF3B00320000F032FE47
:108CB0004B469860D9601C605D6008235B429C460F
:108CC000E14426002F00CA45DBD14346012B00DCDE
:108CD000E3E0039A13005B441E685F68029BDB00BD
:108CE00099464A44904610E0FFFFFF000000E03F35
:108CF0000000F03FFFFFFF3F0000703EE0E100009A
:108D0000FB21F93FFFFFFF1F984643465C681B6845
:108D10001800210032003B000090019100F0FAFDA4
:108D200004000D0002000B000098019901F08AFF79
:108D300032003B0000F0EEFD4346039A9860D96094
:108D40001C605D60083B26002F009A42DCD14D4636
:108D50009446002600244746083565442A686B6817
:108D60003000210000F0D6FD083D06000C00AF42A7
:108D7000F4D1039B4A9F5D689968D868089B002BD3
:108D800065D08022120694460D9B6544604464447D
:108D90001F605D609960D8601E615C61EEE69A4676
:108DA0004B460793059B30005A423900089500F066
:108DB000CFF900223A4B06000F0000F0FBFB002821
:108DC00024D0384B00223000390001F0C9FC02F0F9
:108DD0009DFA52460400950002F0CEFA0022304B74
:108DE00001F0BEFC02000B003000390001F02AFF48
:108DF00002F08CFA0EAA50510122059B52441833FE
:108E00009046059393000EAAD45023E653463000B3
:108E100039009C0002F07AFA0EAB1851D04619E6E0
:108E200080230D9A1B06CB18106053600B000200C4
:108E30004A984B9901F006FF434607000C00002BAF
:108E400000DDD5E680231B069C466444E4E62B0047
:108E50003A000D9D2A606B600A000300AA60EB6077
:108E6000320023002A616B6188E6099BDB000093D6
:108E700072AB049332E4A49B022B00DDE8E6002BE6
:108E800000DD92E600D079E6002700246AE600269D
:108E900000246EE70020002198E60026340068E7F1
:108EA000000070410000703EF0B5CE46474680B5E8
:108EB00087B000920193474A4B00814688465B0881
:108EC000934207DC4146484602F020FA4146031E21
:108ED000484666D04A4643464846414601F040FC73
:108EE00004000D0002000B004846414601F038FC2A
:108EF000394A3A4B06000F002000290001F030FCEF
:108F0000374A384B01F09EFE22002B0001F028FC6E
:108F1000354A364B00F0FEFC22002B0001F020FC0D
:108F2000334A344B01F08EFE22002B0001F018FC76
:108F3000314B324A00F0EEFC0E9B02900391002B65
:108F400034D00098019900222D4B01F009FC029ABF
:108F5000039B049005913000390001F001FC0200F0
:108F60000B000498059901F06DFE22002B0001F022
:108F7000F7FB009A019B01F065FE224A04000D00F8
:108F8000214B3000390001F0EBFB02000B00200008
:108F9000290000F0BFFC02000B004846414601F0EA
:108FA00051FE07B00CBC90469946F0BD02000B0084
:108FB0002000290001F0D4FB124A134B01F042FEBD
:108FC00032003B0001F0CCFB4A46434600F0A2FCD5
:108FD000E7E7C046FFFF3F3E7CD5CF5A3AD9E53D93
:108FE000EB9C2B8AE6E55A3E7DFEB157E31DC73E5A
:108FF000D561C119A0012A3F1111813FA6F81011B6
:109000000000E03F495555555555C53F49004B08AF
:1090100019007047474AF0B54F4691464B005B0D2B
:1090200099444646D6464A46C0B505000C000E0097
:1090300088460700132A27DC002A4BDB3E4B1341EE
:109040009A460B0052461340034318D03B4A3C4B10
:109050002800210000F05EFC0022002300F0A0FAAE
:10906000002847D0002C04DA80234A465B031341D2
:1090700098444646534600279E43380031001CBCA6
:1090800090469946A246F0BD332A08DD8023DB00D6
:109090009945F4D102000B0000F03CFCEFE7294AAF
:1090A0009446012263445242DA4092460242E6D09C
:1090B000224A234B2800210000F02CFC0022002330
:1090C00000F06EFA002815D0002C1EDB53464646F1
:1090D0009F430FE0194A1A4B2800210000F01AFCA8
:1090E0000022002300F05CFA002803D0002C04DBEF
:1090F0000027002638003100C1E7640064082543DA
:109100000027002DF6D0104EF4E74B46142B0BD061
:109110003422D21A012393405D19BD4208D20123A3
:109120009C462F00E044D1E7133B9C46E044CDE74A
:109130002F00CBE701FCFFFFFFFF0F009C750088AD
:109140003CE4377EEDFBFFFF0000F0BF00207047DE
:109150004B0070B55B0D14000A00002B1AD14B00B8
:109160005B08034315D0234B002201F0F9FA224B90
:109170009C422DDB0A004B005B0D363B1F4DE31874
:10918000AB422ADC002B0DDD1D4C1B0522401A438F
:10919000110070BD1B4DAB42F0D102000B0000F07E
:1091A000B9FBF6E71D00353519DA174B02009C4272
:1091B00009DD0B001548164900F032F8134A144B2C
:1091C00001F0CEFAE5E70B001248134900F028F849
:1091D000104A114B01F0C4FADBE70200E9E7084C42
:1091E000363322401B051343190000220B4B01F0BC
:1091F000B7FACEE700005043B03CFFFFFE07000087
:10920000FFFF0F80FF07000050C300009C7500881F
:109210003CE4377E59F3F8C21F6EA5010000903C74
:1092200030B54A00DB0FDB0752081A43110030BD8E
:1092300002B4714649084900095C49008E4402BCE9
:109240007047C046002243088B4274D303098B4207
:109250005FD3030A8B4244D3030B8B4228D3030C06
:109260008B420DD3FF22090212BA030C8B4202D3A8
:109270001212090265D0030B8B4219D300E0090AD0
:10928000C30B8B4201D3CB03C01A5241830B8B42D9
:1092900001D38B03C01A5241430B8B4201D34B03C2
:1092A000C01A5241030B8B4201D30B03C01A524127
:1092B000C30A8B4201D3CB02C01A5241830A8B42AC
:1092C00001D38B02C01A5241430A8B4201D34B0295
:1092D000C01A5241030A8B4201D30B02C01A5241F9
:1092E000CDD2C3098B4201D3CB01C01A52418309AD
:1092F0008B4201D38B01C01A524143098B4201D3E7
:109300004B01C01A524103098B4201D30B01C01A11
:109310005241C3088B4201D3CB00C01A524183088B
:109320008B4201D38B00C01A524143088B4201D3B8
:109330004B00C01A5241411A00D201465241104618
:109340007047FFE701B5002000F0F0F802BDC0460D
:109350000029F7D076E7704703460B437FD40022FD
:1093600043088B4274D303098B425FD3030A8B42B9
:1093700044D3030B8B4228D3030C8B420DD3FF2223
:10938000090212BA030C8B4202D31212090265D0F1
:10939000030B8B4219D300E0090AC30B8B4201D3A4
:1093A000CB03C01A5241830B8B4201D38B03C01AEB
:1093B0005241430B8B4201D34B03C01A5241030B62
:1093C0008B4201D30B03C01A5241C30A8B4201D313
:1093D000CB02C01A5241830A8B4201D38B02C01ABE
:1093E0005241430A8B4201D34B02C01A5241030A35
:1093F0008B4201D30B02C01A5241CDD2C3098B421A
:1094000001D3CB01C01A524183098B4201D38B0196
:10941000C01A524143098B4201D34B01C01A524139
:1094200003098B4201D30B01C01A5241C3088B427E
:1094300001D3CB00C01A524183088B4201D38B0069
:10944000C01A524143088B4201D34B00C01A52410B
:10945000411A00D201465241104670475DE0CA0FE2
:1094600000D04942031000D34042534000229C46A2
:1094700003098B422DD3030A8B4212D3FC228901AC
:1094800012BA030A8B420CD3890192118B4208D382
:10949000890192118B4204D389013AD0921100E0E4
:1094A0008909C3098B4201D3CB01C01A52418309F8
:1094B0008B4201D38B01C01A524143098B4201D325
:1094C0004B01C01A524103098B4201D30B01C01A50
:1094D0005241C3088B4201D3CB00C01A52418308CA
:1094E0008B4201D38B00C01A5241D9D243088B4220
:1094F00001D34B00C01A5241411A00D201466346C3
:1095000052415B10104601D34042002B00D5494226
:10951000704763465B1000D3404201B5002000F065
:1095200005F802BD0029F8D016E770477047C0461D
:10953000D0400B1C1141203A03D49C4613411843E0
:1095400063465242934018437047C0468446101CFD
:1095500062468C46191C634600E0C0461FB501F008
:1095600097F8002801D40021C8421FBD10B500F0B3
:10957000EFFF4042013010BD10B501F089F800281E
:1095800001DB002010BD012010BDC04610B501F068
:109590007FF8002801DD002010BD012010BDC0466D
:1095A00010B501F011F8002801DC002010BD0120E9
:1095B00010BDC04610B501F007F8002801DA002000
:1095C00010BD012010BDC046F0B5CE46474615047B
:1095D0002D0C2E0080B50704140C3F0C9946030C8B
:1095E0007E435D43674363437F19340CE4199C4613
:1095F000A54203D980235B029846C4444B464343AB
:109600005143250C36046544360C2404A4195B1917
:10961000591820000CBC90469946F0BDF0B54E4656
:1096200057464546DE46E0B543025B0A450083B037
:109630000F1C99462D0EC60F002D57D0FF2D24D09C
:109640008020DB00C0041843002381469A469B46D5
:109650007F3D7C027A00FB0F640A120E984623D0ED
:10966000FF2A4BD0E30080240020E4047F3A1C430F
:10967000AD186B1C47460193534677403A000F2BB9
:1096800048D87D499B00CB589F46002B00D085E0F1
:1096900008339A46063B9B467C027A00FB0FFF2567
:1096A000640A120E9846DBD1002C00D090E052469E
:1096B00001231A4392460120DBE74C465846170027
:1096C000022824D0032800D1CFE000220023012863
:1096D0004DD15802D205400AFF071043384303B06A
:1096E0003CBC90469946A246AB46F0BD002B5BD1F0
:1096F00004239A46033B00259B46AAE7FF35002C2E
:1097000060D1524602231A4392460220B1E7FF225B
:109710000023DEE74B461B0C9C464B462604360CCA
:10972000180461463300220C6446000C43434E4348
:109730005043544380191A0C1218964203D98021C1
:1097400049028C4664441B041B0C1004C01883019E
:109750005E1EB341800E1843130C1B199B0103437B
:109760001C00230179D5012362081C401443019A8F
:109770007F32002A4DDD630704D00F232340042BE2
:1097800000D00434230103D53C4B019A1C408032A5
:10979000FE2ABCDCA3015B0AD2B29AE70C239A46EC
:1097A000093BFF259B4654E7180001F071FE4A462D
:1097B000431F76259A4000236D4291462D1A9A4602
:1097C0009B4646E7524603231A439246032050E73E
:1097D000200001F05DFE431F2D1A9C40763D0020C5
:1097E00047E780230027DB03FF2272E7424666E754
:1097F0004C463200584662E780234A46DB031A4251
:1098000022D01C4220D123435B025B0A4746FF2241
:109810005FE701239A1A1B2A21DC23000199D34018
:109820009E318C401A0023005C1EA34113435A074B
:1098300004D00F221A40042A00D004335A0111D454
:109840009B015B0A002244E780234A46DB03134363
:109850005B025B0A3700FF223BE7019587E70022A6
:10986000002336E70122002333E78023DB03234371
:109870005B025B0AFF222CE730E20000FFFFFFF7EC
:1098800070B500283DD0C317C5185D40C40F28002F
:1098900001F0FEFD9E22121A962A07DCD2B2082899
:1098A00033DD083885406802400A23E0992A0BDD41
:1098B000052329001B1AD94003001B339D402B00B0
:1098C0005D1EAB4119430D00052801DD431F9D407E
:1098D0002B000F490B406E0709D00F263540042D91
:1098E00005D004335D0102D59F220B40121A9B0163
:1098F000580AD2B24002D205400AE407104320437E
:1099000070BD002400220020F4E76802400AF1E75D
:10991000FFFFFFFBF0B54F464646D6460C00090355
:10992000C0B5490A470F5E0039431F03DB0F9C4651
:1099300065007B0A570F1F436D0DE40F760DA1469E
:10994000C000B846D200AB1B64457BD0002B5FDD66
:10995000002E00D0A4E03E00164300D112E15E1EAE
:10996000002E00D09EE1871A4346B842804101256F
:10997000C91A4042091A0B0200D431E149024E0AC9
:10998000002E00D16EE1300001F082FD0300083BA3
:109990001F2B00DD61E120223900D21A9E40D14008
:1099A0009F400E439D4200DD51E15D1B6B1C1F2B50
:1099B00000DD7CE12021C91A3D0030008F40884045
:1099C000DD40791E8F41310007222843D940002510
:1099D00007433A40002A09D00F233B40042B05D00F
:1099E0003B1DBB42BF417F42C9191F000B0200D47F
:1099F00026E26A1CC64B55056D0D9A4200D106E160
:109A0000C44AFF080A40530752023B43120B8EE040
:109A1000002B00D0B8E06B1C5B055B0D012B00DC5C
:109A200030E1871A4346B842B641CB1A76429E1BB4
:109A3000330200D54CE13B003343A1D10022002486
:109A4000002570E0002B00DCE5E0002E00D183E073
:109A5000AF4EB54260D0802636043743B846382B27
:109A600000DC3EE1434613431F007A1E97413F1836
:109A700087428041404209180B0200D4B0E0A44B59
:109A800001359D4200D1C3E0A24A7B080A40012172
:109A90000F401F435108D30707221F433A4099E75D
:109AA0009B4EB54238D0802636043743B846382B13
:109AB00000DDDCE01F2B00DC30E11E004746203ECD
:109AC000F740BC46202B04D04026F31A46469E4061
:109AD0003243170063467A1E97411F43CCE0002BA8
:109AE00000D104E24346134300D159E14B07C008BB
:109AF00018438023C9081B03194208D04546ED08C6
:109B00001D4204D14346D008590708432900420F9B
:109B1000C9007F4D1143C0004B07CA087C49C008EB
:109B200003438D4268D012036D05120B6D0D0021A9
:109B300012031800130B0A0D12051A43764B2D055C
:109B400013402B435B00E4075B08234319001CBC54
:109B500090469946A246F0BD3E00164312D05E1EC6
:109B6000002E00D000E187188742804141444042E6
:109B7000091801250B0233D5022585E76446330019
:109B8000414610001D00C7E7002D00D0DAE00C00B0
:109B90000443F3D05C1C00D19FE15D4CA64200D190
:109BA0002FE1DB43382B00DD66E11F2B00DD83E175
:109BB00020240500E41A0F00DD40D940A0404346B0
:109BC000A7405B1A441EA04198462F433843171AFA
:109BD000BA42924143465242991A64463500CAE657
:109BE00007223A40002A00D0F6E64B07CA08484947
:109BF000FF083B438D4296D11900114300D19EE1ED
:109C0000802109030A431203120B414D8FE715000F
:109C1000002200238BE7002B00D0C7E06B1C5F0500
:109C20007F0D012F00DCF1E0394DAB4200D1B9E0EE
:109C300085180A0085428941424449425118072249
:109C4000CF076D082F4349083A401D00C2E607229E
:109C50003049ED1A31403A40BCE63E002838864093
:109C600000279FE6380001F013FC20308EE64346C3
:109C700013431F007A1E9741C71BB84280414042E0
:109C8000091A78E60E003B0006431343002D61D10C
:109C9000002E00D0F4E0002B00D11BE16446390017
:109CA000100039E71A4FBB427AD03300FFE630008C
:109CB0001F3DE840202B03D04021CB1A9E40374364
:109CC0007B1E9F41072207433A400021002589E778
:109CD000171A4346BA42B641591A76428E1B644659
:109CE0004EE61F2B00DDADE020264746F61AB740B2
:109CF000B9461700B246DF404E463E43370056464F
:109D0000B240561EB24117434246DA408918AEE6C9
:109D1000FF070000FFFF7FFFFFFF0F802026474661
:109D2000F61AB740B9461700B246DF404E463E43EA
:109D300037005646B240561EB24117434246DA40FB
:109D4000891A99E77F4CA6425BD0802424045B42A9
:109D5000214327E7002E0CD1002B00D1CBE0644635
:109D600039001000774DD7E6764FBB4218D033004C
:109D700075E6002B14D04B07C00818438023C90890
:109D80001B03194207D0FC081C4204D17907D008F4
:109D90000843E14621004C46420FC9001143C00070
:109DA000684DB9E61D0000220023C0E6002D5BD1FE
:109DB0000D00054300D1E2E65D1C00D1B0E0614D2D
:109DC000AE421FD0DB43382B71DC1F2B00DD96E049
:109DD00020250F00ED1AAF40B9460700AA46DF4024
:109DE0004D463D432F005546A840D940451EA84149
:109DF00088440743BF18974292415142414435007D
:109E00003AE6644635004146100085E60B00034300
:109E1000002D00D063E6002BF5D04346134300D15C
:109E20007AE6871887428041072241444042091858
:109E30003A400B0200D4D5E6434B01351940C9E541
:109E4000380069E61E004746203EF740BC46202BFE
:109E500004D04026F31A46469E403243170063461C
:109E60007A1E97411F4302E6364DAE42CAD0802586
:109E70002D045B422943A6E70843411E8841A6E61C
:109E8000002B00D148E6871A4346B842B641CB1AA8
:109E900076429E1B33024BD5171A4346BA42924173
:109EA000591A5242891A072264463A4092E5014300
:109EB0000F00791E8F419DE71C000F00203CE740FA
:109EC000202B03D04024E31A99400843411E8841C7
:109ED00038437CE60022002425E6171A4346BA429E
:109EE0009241591A5242891A6446350043E5414667
:109EF0001000144D10E680220024120380E61D009D
:109F00000F00203DEF40BC46202B03D04025EB1A2C
:109F10009940084307006346781E87411F4369E75D
:109F2000871897429B4141445B42C9183500A3E51D
:109F30003B003343CED0072231003A4052E60023A3
:109F40001A00F4E5FF070000FFFF7FFFF0B557465A
:109F5000DE464E464546E0B5834607000E03480000
:109F600085B092461C00360B400DCD0F002800D165
:109F70009DE0954B984239D08023F6001B041E4388
:109F8000924A7B0F334399469446030063440093FF
:109F900000230026FF00029323031B0B9846630057
:109FA000E40F52465B0D019400D1B3E086498B4229
:109FB00000D19EE04246D100802212040A4351465D
:109FC000490F11438B46814952468C4600996344A0
:109FD000CB1A0021D20000932B0063409A460F2E2B
:109FE00000D905E17A4BB6009B599F465B46334347
:109FF000994600D0B8E0022308260027009002937B
:10A00000CAE7CB463A0002990195019B9A4602297C
:10A0100027D0032900D180E2012944D06D49009B5B
:10A020008C4663441C00002C38DD530700D013E23B
:10A03000D2085B46DB0109D55946674B19408B4670
:10A040008021C9008C46009B63441C00634B9C42EA
:10A0500007DC5B4664055F075B0217431B0B620D61
:10A0600002E000230027584A00211B031C0B0B0DA4
:10A070001B05234314055A4A380013401C4353461A
:10A080006400DB0764081C43210005B03CBC90461B
:10A090009946A246AB46F0BD0122524201231B1B4A
:10A0A000382B00DCADE1002200230027DCE75B4613
:10A0B000334399465ED0002E00D18AE1300001F092
:10A0C000E7F903000B3B1C2B00DD7BE11D22D31ABB
:10A0D0005A460100DA4008398E4013005F46334388
:10A0E00099468F403F4B00261B1A00930023029392
:10A0F00052E7414653460B433B499B468C46009BE7
:10A10000634400935B46002B3BD1022300221E4395
:10A11000022161E7434613439B4637D04346002B59
:10A1200000D162E1404601F0B3F903000B3B1C2B68
:10A1300000DD53E102004146083A914088461D2166
:10A14000CB1A5146D9400B0041460B439B46534620
:10A1500093401A00009B25499C46604403008C46AE
:10A1600063440093002137E70323B14600900C2697
:10A17000029311E700230093013304260027029382
:10A180000AE70323C3461E43032125E701331E4389
:10A190000022012120E700239A46802300271B0389
:10A1A000094A61E7802349461B03194200D1E2E0D6
:10A1B0005946194200D0DEE00B431B0317001B0B6E
:10A1C000A246014A50E7C046FF07000001FCFFFF1E
:10A1D00070E20000FF030000FFFFFFFEFE0700002B
:10A1E000FFFF0F800DFCFFFF01F8FFFFF3030000EE
:10A1F000D94500D9CBE000D1C6E03C004846002755
:10A20000009B013B00935B46160E1B021E4313028C
:10A21000984633041B0C9946310C0191FFF798F8CE
:10A220004A4642430B04210C050019438A4207D9D0
:10A230008919013D8E4203D88A4201D9851E8919A8
:10A24000881A0199FFF784F809048C464A462104CC
:10A2500064464243090C030021438A4204D9891908
:10A26000013B8E4200D8F1E02D041D43AB4643462E
:10A27000891A4246280C12041D0C5B46140C22005D
:10A280001B041B0C5A4303946B43444302956843DD
:10A290001B19150CEB189C4203D980246402A446B8
:10A2A00060441C0C15041B042D0C20185D19814200
:10A2B00077D373D00C1AA24A7D1BAF42BF4194469C
:10A2C000009B7F426344E01B1C00864200D1DBE020
:10A2D0000199FFF73DF84A4642430B04290C070059
:10A2E00019438A4207D98919013F8E4203D88A420D
:10A2F00001D9871E8919881A0199FFF729F80904DD
:10A300004A46894629044D464243090C0300294325
:10A310008A4207D98919013B8E4203D88A4201D962
:10A32000831E89193F04891A3A00039F1A43380093
:10A3300013041B0C584381460298150C6F4343438A
:10A3400045434846000C8446DB1963449F4203D9C9
:10A35000802040028446654448461F0C00041B04CC
:10A36000000C7D191818A94200D284E000D17FE0CA
:10A3700001231A4357E680234A461B0313431B035A
:10A380001B0BAA466F4A6FE6BA4200D935E74B4627
:10A39000DC0758087B081C43FF0734E70024AF4262
:10A3A00089D247444745A4415B466442A4196418D6
:10A3B000013BA6421ED2A0426DD800D1B6E0241ABD
:10A3C0009B4678E703005A46283B9A40002791466F
:10A3D00088E6584601F05CF8203072E603005246E9
:10A3E000283B9A4093460022B4E6504601F050F8CC
:10A3F00020309AE6A642E2D1B845DCD9341A9B4611
:10A4000059E71F2B65DC504C0099A4465C4661441B
:10A4100008008C4011008240D940501E82410C43FC
:10A4200014435A46DA401300620709D00F22224033
:10A43000042A05D02200141D9442894149425B1828
:10A440001A0262D50122002300270DE68A4200D8B5
:10A450000AE7831E891907E70F231340042B00D155
:10A46000E6E5171D9742924153429B44FA08E0E506
:10A47000002800D1D7E57118531EB14227D3A94255
:10A4800015D358D01A0073E7002B00DC04E6012333
:10A4900000229B44CDE502234744474589415B4266
:10A4A0009C46494289190C19E344241A03E74346A0
:10A4B0005F0047459B41B8465B429E19023A8919A5
:10A4C000A94200D054E7404500D051E7ABE51A005F
:10A4D000F6E71F215F4649420C1BE740202B07D0BF
:10A4E0001A49009B8C46634418005B4683401A431C
:10A4F000501E82413A4307270023174009D00F21FD
:10A50000002311401400042995D122005F075B024B
:10A510001B0BD20817430022A6E5802359461B03D4
:10A520000B431B0317001B0B064A9DE5BD42B2D827
:10A530009B460024BFE68045B9D31A00C3E7C04656
:10A54000FF030000FF0700001E0400003E0400009F
:10A55000F0B54F464646D6468446C0B58046194EAD
:10A5600018030F034D00000B5C0082463F0B6D0D7E
:10A57000C90F9146640DDB0F0120B5420AD0B442E9
:10A5800003D0A54201D157450CD01CBC904699463A
:10A59000A246F0BD66463E43F7D1AC42F5D15446E3
:10A5A0001443F2D10120C845EFD1994207D0002DC4
:10A5B000EBD163461F433800471EB841E5E7002052
:10A5C000E3E7C046FF070000F0B54F464646D646D3
:10A5D0004D00C0B50E03C90F8A462C491F035C000D
:10A5E0008046360B6D0D91463F0B640DDB0F8D429F
:10A5F0001ED08C4216D0002D1ED130438446002C34
:10A6000001D13A4323D06246002A1AD09A4529D074
:10A61000514602200139084001381CBC9046994639
:10A62000A246F0BD39001143E5D002204042F4E7D4
:10A630003043FAD1AC420FD0002C0FD13A43E7D0CF
:10A640000CE00122013B934318000130E5E763462B
:10A650000020002BE1D0DBE73A43E6D19A45D7D181
:10A66000A542D5DCA54205DBBE42D1D808D00020EA
:10A67000BE42D2D250460123013898430130CCE784
:10A68000C845C5D80020C845F4D3C6E7FF07000079
:10A69000F0B54F464646D6464D00C0B50E03C90F2D
:10A6A0008A462E491F035C008046360B6D0D91468D
:10A6B0003F0B640DDB0F8D4218D08C4211D0002D62
:10A6C00018D130438446002C1ED13A431CD1634636
:10A6D0000020002B30D051460220013908400138BB
:10A6E0002AE039001143EAD0022025E03043FBD1B3
:10A6F000AC4226D0002C26D13A4324D15146022028
:10A7000001390840013817E06246002A0FD09A4507
:10A71000E1D1A54205DBBE42DDD819D00020BE4202
:10A720000AD25046012301389843013004E0012247
:10A73000013B9343180001301CBC90469946A24649
:10A74000F0BD3A43D0D19A45C5D1A542C3DCE0E77C
:10A75000C845C0D80020C845E3D3EDE7FF07000097
:10A76000F0B55746DE464E464546E0B58346060000
:10A770000F03480087B092461D003F0B400DCC0FE1
:10A78000002800D16FE0DE4B984238D08023FF00D4
:10A790001B041F43730F3B430193DA4B0027994679
:10A7A00000239B46F60081442B0369001B0B524695
:10A7B0009846490DED0F002900D185E0D04B994214
:10A7C00000D173E04346DA0080231B041343524652
:10A7D000CC48520F84461343524600206144D200B5
:10A7E00089442100694000918C46012149448A46F0
:10A7F0000F2F00D990E0C449BF00CF59BF465B4638
:10A800003B43019300D06AE10223082700268146DA
:10A810009B46C9E732005846019B614600910228D9
:10A8200000D175E0032800D1FEE1012800D02CE121
:10A8300000230027002600253F032A0D3F0BB348C5
:10A8400012053A4302401B051343009A5B00D107EF
:10A850005B080B433000190007B03CBC904699469A
:10A86000A246AB46F0BD5B463B43019300D12FE1CE
:10A87000002F00D1A5E1380000F00AFE03000B3BD9
:10A880001C2B00DD96E11D22D31A5A460100DA4046
:10A890005E4608398F4013008E403B4301939C4B2A
:10A8A00000271B1A994600239B467DE741465346E5
:10A8B0000B4393498C46E144002B00D01AE102225D
:10A8C0000220174300228CE7134300D10DE14346D9
:10A8D000002B00D181E1404600F0DAFD02000B3A86
:10A8E0001C2A00DD72E10100434608398B4098467E
:10A8F0001D239A1A5346D3401A0043461343524627
:10A900008A404946081A824989468144002068E7FE
:10A910007B4B002700268EE7140C1204120C11004A
:10A92000370C3604350C794328008C462E006043E2
:10A930006044834656432100300C80465846794394
:10A9400040440291844506D98846802149028C46BC
:10A95000E044414602913604010C360C00048B465B
:10A9600081191E0C1B041B0C0391190079438C46A2
:10A97000280075436544A8465843050C4544774371
:10A98000A94203D9802149028C466744290C8C4690
:10A9900039000004000C2D042D186144AB440591CE
:10A9A0005946049101990F043F0C080C390051439A
:10A9B0004243904602008C46090C8B4662437C431E
:10A9C00044445C44A04503D980214902884642445E
:10A9D000210C884661460904090C8C46390059430C
:10A9E000434370437E430F0CF6182404BE1964449D
:10A9F00042448C46B34203D980235B0298464044CC
:10AA0000029B61469846049B370443449B46AB45F2
:10AA1000AD416B420D0405992D0C8C467F1967449E
:10AA2000FD18A8465D462D19A542A44193466442EF
:10AA3000A446C344DC448F42BF4198459B419345A3
:10AA40009241A445A4415B427F421F43360C5242CF
:10AA50006442BF192243BF18624638184302D20D20
:10AA6000039913436A020A43501E82416146ED0D69
:10AA70002A434E023243D90100D4B3E001265008E4
:10AA800032400243DE0732435B08224C5444002C20
:10AA900062DD510709D00F201040042805D0101D99
:10AAA0009042924152429B180200D90104D5802461
:10AAB0001948E400034054441848844200DD27E765
:10AAC0005E075B02D2081F0B630516435B0DB2E6FF
:10AAD000002399460133042700269B4664E603239E
:10AAE000019781460C279B465EE601220120174311
:10AAF000002276E6032303201F43434671E6C04647
:10AB0000FF07000001FCFFFFB0E20000FFFF0F8025
:10AB10000DFCFFFFFF030000FFFFFFFEFE0700002C
:10AB20000023802700933F030026434B83E6019BCD
:10AB30003200A446584670E6AC466EE6802701997E
:10AB40003F0339422DD03B422BD11F433F033F0BE4
:10AB500000951600384B6EE601252D1B382D00DDC3
:10AB600066E61F2D40DC35481C005044160082402C
:10AB70008440EE40501E824134431443EB40620750
:10AB800009D00F222240042A05D02200141D94422D
:10AB9000804140421B181A023ED50123002700269F
:10ABA00049E68027019B3F031F433F033F0B00946F
:10ABB000214B40E603005A46283B9A40002601926A
:10ABC0006DE6584600F064FC203057E6030052461C
:10ABD000283B9A401300002293E6504600F058FCB0
:10ABE00020307BE6CA4650E71F201E004042041B6F
:10ABF000E640202D03D0124C5444A3401A43501E6B
:10AC00008241324307260027164009D00F20002337
:10AC1000104014000428B9D122005E075B021F0B0C
:10AC2000D2081643002306E680273F031F433F0355
:10AC30003F0B1600004BFEE5FF0700001E0400005E
:10AC40003E040000F8B557464E464546DE460C0029
:10AC50000903E0B5490A460F5F0031431E03DB0FCD
:10AC6000760A9B46530F3343C84E6500C000E40F7D
:10AC7000D2006D0DA24681467F0D9C469046B7429C
:10AC800000D1B9E05B46012673409B46EE1BA3450D
:10AC900000D183E0002E63DD002F00D0B1E06346D9
:10ACA000134300D123E1731E002B00D0BAE1861AB2
:10ACB0006346B04280410125C91A4042091A0B027D
:10ACC00000D447E149024B0A98464346002B00D185
:10ACD00089E1404600F0DCFB0300083B1F2B00DD50
:10ACE0007CE120223000D21A4146D0409940020037
:10ACF0009E400A439D4200DD6AE15D1B6B1C1F2BD9
:10AD000000DD94E1202110003500C91A8E40DA40A0
:10AD10008840DD40711E8E41110007222843002526
:10AD200006433240002A09D00F233340042B05D0BC
:10AD3000331DB342B641764289191E000B0200D47E
:10AD40003DE26A1C914B55056D0D9A4200D119E107
:10AD50008F4AF6080A40570752023743120B9BE00E
:10AD6000002E00D0C5E06E1C7605760D012E00DCAD
:10AD700048E16746861ACB1BB042BF417F42B846C6
:10AD80001F004346FF1A3B00B8461B0200D55FE197
:10AD900037439AD100220024002579E0002E00DC00
:10ADA000FAE0002F00D18DE0784B9D4267D08023E0
:10ADB00067461B041F43BC46382E00DC52E1634645
:10ADC00013435A1E93411E1886428041404209187F
:10ADD0000B0200D4BEE06D4B01359D4200D1D2E0A4
:10ADE0006B4A73080A4001210E401E435108D307E5
:10ADF00007221E43324095E71E00164300D045E768
:10AE000040E7624B9D423AD0802367461B041F43B4
:10AE1000BC46382E00DDEBE01F2E00DC3AE13300AB
:10AE20006746203BDF403B00202E05D04027BF1B5C
:10AE30006646BE40324390464646721E96413343B4
:10AE4000DAE0002B00D114E26346134300D168E13D
:10AE500080234E07C008C9081B030643194208D0C7
:10AE60006046C008184204D163460100D2085E075C
:10AE70001643F3009946C900720F444D11434B46E7
:10AE8000DE08424B4F073743CA089D4200D16EE0AF
:10AE900012036D05120B6D0D00211203130B0A0D29
:10AEA00012051A433B4B2D0513402B435B00E4076F
:10AEB0005B082343380019003CBC90469946A246E3
:10AEC000AB46F8BD6346134311D0731E002B00D070
:10AED00007E18618864280416144404209180125F5
:10AEE0000B0237D502257BE73E00614691463500CF
:10AEF000C5E75C46002D00D0E1E00B000343F3D032
:10AF0000731C00D1ACE1214B9F4200D13AE1F343E5
:10AF1000382B00DD6FE11F2B00DD8CE120250E00BA
:10AF2000ED1AAE40B0460600AA46DE40454635431F
:10AF30002E005546D940A8406346451EA8415B1ADD
:10AF40009C463043161AB242924163465242991AC5
:10AF50003D00B4E607223240002A00D0E4E60B4B65
:10AF6000F6084F073743CA089D4200D090E73B00E0
:10AF7000134300D1A6E180231B031A431203120BD3
:10AF8000024D89E715000022002785E7FF07000032
:10AF9000FFFF7FFFFFFF0F80002E00D0C7E06B1C7C
:10AFA0005E05760D012E00DCF0E0C84DAB4200D10D
:10AFB000B9E085180A008542894162444942511826
:10AFC0000722CE076D082E43490832401D00A9E62E
:10AFD000BF49ED1A114007223240A3E6320028385B
:10AFE0008240002686E6300000F052FA203073E6F8
:10AFF000634613435A1E9341C61AB04280414042F1
:10B00000091A5CE60E00674606431743002D5ED121
:10B01000002E00D0F3E0002F00D11EE15C46614617
:10B0200091462CE7A94FBE427BD01E00F1E61000EE
:10B030001F3DE840202B03D04021CB1A9A401643F5
:10B04000731E9E410722064332400021002583E7FC
:10B05000161A6346B2428041591A40420B1A98466A
:10B060005C4632E61F2E00DDABE02027BB1B9A4674
:10B0700063465746BB40994613004F46F3401F4373
:10B080003B005746BA40571EBA4113436246F2404E
:10B09000891898E62027BB1B9A4663465746BB4053
:10B0A000994613004F46F3401F433B005746BA40B2
:10B0B000571EBA4113436246F240891A9CE7834BFC
:10B0C0009F425FD080252D047342294320E7002E44
:10B0D0000CD1002F00D1D0E05C46614691467B4DFB
:10B0E000CDE67A4FBE421CD01E0065E6002F18D078
:10B0F000C0084E0706438020C9080003014208D05B
:10B100006346DC08044204D12100DA46D2085E0717
:10B110001643F300994601245346C900720F1143A8
:10B120001C406A4DABE61D0000220027B4E6002D4E
:10B1300059D10B00034300D1D6E6731C00D1B2E015
:10B14000624B9F421ED0F343382B6FDC1F2B00DD78
:10B1500097E020250E00ED1AAE40B0460600AA4644
:10B16000DE40454635432E005546A840D940451E91
:10B17000A8418C440643B61896429241514261441C
:10B180003D0025E63D006146914678E60B0003430D
:10B19000002D00D055E6002BF5D06346134300D1B7
:10B1A0006DE68618864280416144404209180022BB
:10B1B0000B0200D4D0E6464B01351940B2E5B1464A
:10B1C0005DE633006746203BDF403B00202E05D084
:10B1D0004027BF1B6646BE40324390464646721E1D
:10B1E00096413343EFE5394B9F42CBD080252D0468
:10B1F00073422943A8E70843411E8841A2E6002F75
:10B2000000D13CE66346861ACF1AB0429B415B42AE
:10B21000FB1A98461B024ED5161A6346B24292415B
:10B22000591A5242891A5C4600227BE501430E00FE
:10B23000711E8E419FE71D000E00203DEE40B0467E
:10B24000202B04D04025EB1A9940084381464846FC
:10B250004346411E8841184374E60022002417E645
:10B26000161A6346B2429241591A5242891A3D0057
:10B2700025E561469146154D01E680220024120322
:10B2800079E61D000E00203DEE40B046202B04D094
:10B290004025EB1A9940084381464E464346711EAD
:10B2A0008E411E4367E7861896429B4161445B428C
:10B2B000C9183D008CE547463743CED007224146AA
:10B2C000324049E600273A00E6E5C046FF070000A5
:10B2D000FFFF7FFF70B50C4E0D031C0349005B00A0
:10B2E0002D0B490D240B5B0DB14208D006490020FF
:10B2F0008B4203D114432000441EA04170BD05437E
:10B300000120002DFAD1F1E7FF07000030B5144D00
:10B310000A034B00120B5B0DC90F0024AB4211DD79
:10B32000104CA34210DC8024640322430E4CE41A28
:10B330001F2C0CDD0D48C31ADA4013005C420029B3
:10B3400000D11C00200030BD094BCC18FAE7094D94
:10B35000E040AC4663449A4013000343EEE7C04626
:10B36000FE0300001D04000033040000130400006D
:10B37000FFFFFF7FEDFBFFFF70B500282DD0C31747
:10B38000C5185D40C40F280000F082F8154B1B1A49
:10B390005B055B0D0A2815DD0B38854000222D0367
:10B3A0002D0B002110002D030A0D2D0B12052A4331
:10B3B0000D4D1B052A4013435B00E4075B08234344
:10B3C000190070BD02002900153291400A000B21BE
:10B3D000081AC5402D032D0BE3E7002400230025A8
:10B3E0000022DEE71E040000FFFF0F804100090E6F
:10B3F0004B1C70B5DBB24602750AC40F012B14DD7D
:10B40000E0239B006D07360BCB1800210A0D2800A6
:10B4100012051C4D32435B052A405B0813435B0059
:10B42000E4075B082343190070BD002914D1002DE7
:10B430001ED0280000F02CF80A281CDC0B232A0060
:10B440001B1ADA40030015339D400F4B12031B1AE1
:10B450005B05160B5B0DD8E7002D06D0320B80265E
:10B4600036036D071643094BCFE7084B0026CCE7A0
:10B4700000230026C9E703002A000B3B9A40002561
:10B48000E3E7C046FFFF0F8089030000FF070000CD
:10B490001C2101231B04984201D3000C10391B0A04
:10B4A000984201D3000A08391B09984201D30009C8
:10B4B000043902A2105C40187047C046040302021F
:10B4C00001010101000000000000000030B51C0077
:10B4D000094B05001B6885B0D868084B002A01D1CC
:10B4E000074B1A000292019300912B00220005499C
:10B4F00000F026F800F0A6FD84000020F0E2000035
:10B5000014D10000FDE20000014B18687047C046EE
:10B5100084000020084B10B50400002B02D000214D
:10B5200000E000BF054B1868836A002B00D09847E5
:10B53000200001F05DFBC046000000002CE300008D
:10B540000EB403B5010003AB044804CB00680193BB
:10B5500000F076F802B008BC03B018478400002061
:10B5600070B500260C4D0D4C641BA410A64209D1E9
:10B57000002601F03FFB0A4D0A4C641BA410A642B2
:10B5800005D170BDB300EB5898470136EEE7B30024
:10B59000EB5898470136F2E754020020540200208D
:10B5A0005402002064020020002310B59A4200D10A
:10B5B00010BDCC5CC4540133F8E710B5884202D901
:10B5C0008B18984203D3002307E08B5C8354013A25
:10B5D000FBD210BDCC5CC45401339A42FAD1F8E7D7
:10B5E00003001218934200D1704719700133F9E734
:10B5F000936810B5013B9360002B04DA9469A34271
:10B6000007DB0A2905D01368581C10601970080060
:10B6100010BD00F04BFC0100F9E7F8B506000F0083
:10B620001400D518AC4201D1002007E021783A007F
:10B630003000FFF7DDFF0134431CF3D1F8BD0000FB
:10B64000F0B59FB002900F0016000593002805D0BA
:10B6500083690493002B01D100F0F4FD7B4B9F42E2
:10B660005BD1029B5F68BB891B0762D53B69002BDE
:10B670005FD0002306AC6361203363761033A3767A
:10B6800035002B78002B01D0252B5CD1AB1B04930C
:10B690000CD0320039000298FFF7BFFF431C00D1E5
:10B6A000C4E06269049B9446634463612B78002B79
:10B6B00000D1BBE0012200235242626002A9543251
:10B6C00052186E1C2360E360A3601370A365317889
:10B6D00005225F4800F0D4FE751C002835D1226891
:10B6E000D30604D5532302A95B1820211970130730
:10B6F00004D5532302A95B182B21197033782A2B08
:10B700002CD0350000210A20E3682A786E1C303ADC
:10B71000092A64D900292ED026E04E4B9F4202D13F
:10B72000029B9F689FE74C4B9F429CD1029BDF6826
:10B7300099E73900029800F00FFC002899D0012009
:10B7400040421FB0F0BD01359BE7414B2268C01A53
:10B7500001238340134323602E00B8E7059B191D86
:10B760001B680591002B01DB099304E05B42E36059
:10B770000223134323602B782E2B0AD16B782A2BBC
:10B7800035D1059B02351A1D1B680592002B2BDB5A
:10B790000793324E29780322300000F071FE002812
:10B7A00006D04023801B8340226801351343236069
:10B7B000297806222A486E1C217600F061FE0028B6
:10B7C0003AD0284B002B25D10722059B0733934302
:10B7D000083305936369039A9B18636150E74343F9
:10B7E00001219B18350090E701235B42D0E700233D
:10B7F0000A201A000135636029786E1C3039092946
:10B8000003D9002BC5D00792C3E742430123521846
:10B810003500F1E705AB00933A00134B2100029885
:10B8200000E000BF0390039B0133D3D1BB895B06CB
:10B8300000D584E70B9884E705AB00933A000A4BE8
:10B840002100029800F080F8ECE7C04684E3000095
:10B8500030E30000A4E3000064E3000036E30000EE
:10B860003AE30000000000001BB60000F7B5150029
:10B8700001938A680B6900900C00934200DA130070
:10B8800022002B6043321278002A01D001332B6052
:10B8900023689B0602D52B6802332B60062723689A
:10B8A0001F4027D0230043331B785A1E9341226840
:10B8B000920630D42200019943320098089EB04786
:10B8C000431C25D0062320682A68E1680340002530
:10B8D000042B03D18D1AEB43DB171D40A3682269AB
:10B8E000934201DD9B1AED180027BD4220D10020B4
:10B8F00010E00137E3682A689B1ABB42D2DD2200C0
:10B900000123193201990098089EB047431CF0D1D9
:10B9100001204042FEBD3020E11843310870210073
:10B920005A1C45310978A218433202331170C1E71D
:10B93000220001231A3201990098089EB047431C47
:10B94000E6D00137D1E70000F0B589B004920A00D3
:10B9500043320593039002920A7E0C000E9B6E2ADE
:10B9600000D186E01FD8632A33D008D8002A00D13E
:10B970008CE0582A4DD0250042352A7030E0642AE8
:10B9800001D0692AF7D1196825680A1D280629D52A
:10B9900008681A60002803DA2D23029A40421370C7
:10B9A0006B4E0A274FE0732A74D008D86F2A1FD035
:10B9B000702AE0D1202209680A43226003E0752A38
:10B9C00016D0782AD7D12200782145321170614EE5
:10B9D00022E025001A684235111D196013682B708A
:10B9E000012365E008681A606906D3D500B2D1E783
:10B9F00019682568081D186008682E0605D5544E7C
:10BA000008276F2A1BD00A2719E06D06F7D580B2E8
:10BA1000F5E745314E4E0A7018682268011D00682E
:10BA20001960150621D5D30702D520231A432260B9
:10BA30001027002803D1202322689A432260230084
:10BA4000002243331A706368A360002B58DB042282
:10BA5000216891432160002854D1029D002B5AD0C7
:10BA60002500337842352B7055E05506DBD580B282
:10BA7000D9E71A680D68101D4969186013682E0609
:10BA800001D5196002E06D06FBD519800023029DE7
:10BA900023614FE01A68111D196015680021626862
:10BAA000280000F0EDFC002801D0401B60606368B6
:10BAB00023610023029A13703CE023692A00049951
:10BAC0000398059DA847431C3ED023689B0715D4C7
:10BAD000079BE068984239DA180037E0220001231A
:10BAE000193204990398059EB047431C2CD00135A8
:10BAF000E368079A9B1AAB42F0DCE9E70025F7E719
:10BB00000028ADD0029D3900FDF722FC735C013D99
:10BB10002B700028F7D1082F09D12368DB0706D541
:10BB200063682269934202DC3023013D2B70029B43
:10BB30005B1B2361059B07AA00932100049B0398CC
:10BB4000FFF794FE431CB8D10120404209B0F0BD7C
:10BB500041E3000052E300000D4B70B51C68050086
:10BB6000A36B002B0FD1182000F06EFC094BA063D3
:10BB70000360094B01224360084B83600B238381E0
:10BB80000023026143610022A36B1D615A6170BDF5
:10BB9000840000200E33CDAB34126DE6ECDE0500E0
:10BBA000124B10B51C68A36B002B0FD1182000F0AE
:10BBB0004BFC0F4BA06303600E4B012243600E4B06
:10BBC00083600B238381002302614361A46B0B4AD2
:10BBD000206961690A4BFDF7F7FC012200238018F8
:10BBE0005941206161614800400810BD8400002077
:10BBF0000E33CDAB34126DE6ECDE05002D7F954C97
:10BC00002DF451580CB430B5164B9DB00C1E1D6868
:10BC100008DA8B2301202B6040421DB030BC08BCE9
:10BC200002B01847822302A99B008B810023029057
:10BC300008619C4200D0631E8B604B6101235B4214
:10BC4000CB81209A21AB2800019300F055FD431CC5
:10BC500001DA8B232B60002CDFD00023029A1370B3
:10BC6000DBE7C046840000200EB400B50B499CB051
:10BC70001DAB02900690079104910948094904CB35
:10BC80000591006802A9019300F036FD0023029A95
:10BC900013701CB008BC03B01847C046FFFFFF7FFD
:10BCA000840000200802FFFF020010B51378541C26
:10BCB000002B05D1CC5CD4540133002CFAD110BD3B
:10BCC0002200F3E7C9B20378002B04D08B4200D1E5
:10BCD00070470130F7E74B42594149420840F7E7C6
:10BCE00002780B78002A03D0013001319A42F7D054
:10BCF000D01A70470023C25C0133002AFBD1581EC2
:10BD00007047002330B59A420AD0013AC45CCD5C3A
:10BD1000AC4204D1934202D00133002CF6D1631B14
:10BD2000180030BD30B50500002A00D130BD0C78B8
:10BD3000013A6B1C2C700131002C05D19A189A42E3
:10BD4000F4D01C700133FAE71D00EDE710B503785D
:10BD5000002B0FD10B785A4253415B42184010BD63
:10BD60000023CA5C002AFAD0C45C944201D101339A
:10BD7000F7E701300378002BF2D11800EFE700005D
:10BD8000F0B51F000E0087B00590019102920C984B
:10BD9000347800F0EAFA082200194378751C134041
:10BDA00036D12D2C36D1B51C74780126002F62D0E7
:10BDB000102F09D1302C07D120222B789343582BF8
:10BDC00054D110276C7802352D4B3900F318180028
:10BDD0000393FDF7BDFA04910121002349420200BB
:10BDE0008C4618002100303909291AD80C00A742C6
:10BDF00023DD591C09D06346824206D302D104993F
:10BE0000A14202DB0123784320182C780135E9E7B1
:10BE10002E00BCE72B2C01D01E00C7E7B51C7478A0
:10BE2000FAE721004139192901D8373CDFE7210021
:10BE30006139192901D8573CD9E75A1C08D1059A0C
:10BE400023331360029B0398002B09D107B0F0BD88
:10BE5000002E00D04042029A002AF7D0002B01D0D9
:10BE60006B1E0193029B019A1A60EFE73024002FAA
:10BE7000AAD10827A8E7302C9ED00A27A4E7C046FD
:10BE8000FFFFFF7F37B51300064A05001068046AFC
:10BE9000002C00D1044C0A0000942900FFF770FF29
:10BEA0003EBDC04684000020E8000020F8B5050033
:10BEB0000E001400002804D08369002B01D100F08B
:10BEC000C1F9224B9C422DD16C68A369A360A38960
:10BED0001B0731D52369002B2ED023682269F7B2C6
:10BEE000981A6369F6B2834205DC2100280000F04D
:10BEF0003BF9002826D1A3680130013BA3602368E9
:10BF00005A1C22601F706369834204D0A389DB0737
:10BF10001AD50A2E18D12100280000F025F9002892
:10BF200012D00FE00A4B9C4201D1AC68CDE7094B1F
:10BF30009C42CAD1EC68C8E72100280000F00CF848
:10BF40000028CAD0012676423000F8BD84E3000004
:10BF5000A4E3000064E30000364B70B51D680600E2
:10BF60000C00002D05D0AB69002B02D1280000F099
:10BF700069F9314B9C420FD16C680C23E25E93B29D
:10BF800019072DD4D90611D4092301203360373382
:10BF90001343A381404270BD284B9C4201D1AC6841
:10BFA000EBE7274B9C42E8D1EC68E6E75B0713D54B
:10BFB000616B002908D023004433994202D030003D
:10BFC00000F06AFA002363632422A3899343A381C8
:10BFD00000236360236923600823A2891343A3819C
:10BFE0002369002B0BD1A0218022A3898900920014
:10BFF0000B40934203D02100300000F0E1F901230F
:10C00000A289134011D00023A36063695B42A3613E
:10C01000002023698342BED10C23E25E1306BAD509
:10C0200040231343A3810138B5E7920700D4636925
:10C03000A360EDE78400002084E30000A4E3000097
:10C0400064E3000010B5062000F090FC012000F031
:10C05000CFFD0000F7B58A8905000C00130760D4F6
:10C060004B68002B04DC0B6C002B01DC0020FEBDB8
:10C07000E76A002FFAD000232E682B6080235B0133
:10C08000216A1A4034D0606DA3895B0706D56368C6
:10C09000C01A636B002B01D0236CC01A0200216A06
:10C0A00000232800E76AB847A189431C06D12B6802
:10C0B0001D2B30D82B4ADA40D3072CD500236360E0
:10C0C00023692360CB0405D5431C02D12B68002BC8
:10C0D00000D16065616B2E600029C7D02300443316
:10C0E000994202D0280000F0D7F900206063BEE733
:10C0F00001232800B847431CC6D12B68002BC3D0AE
:10C100001D2B01D0162B01D12E60AFE74023A28951
:10C110001343A381ABE740230B430120A38140429B
:10C12000A5E70F69002FA1D00B680F60DB1B0193FF
:10C130000023920700D14B69A360019B002B00DC18
:10C1400094E7019B3A00216A2800A66AB0470028BC
:10C1500003DC4023A2891343DFE7019B3F181B1A2E
:10C160000193EAE7010040200B6970B505000C005F
:10C17000002B01D1002070BD002804D08369002B62
:10C1800001D100F05FF80B4B9C4209D16C680C2286
:10C19000A35E002BEED021002800FFF75BFFEAE74B
:10C1A000054B9C4201D1AC68F1E7044B9C42EED1B7
:10C1B000EC68ECE784E30000A4E3000064E3000023
:10C1C000002310B5040003604360836081814366EF
:10C1D000C281036143618361190008225C30FFF76B
:10C1E000FFF9054B24626362044BA362044BE362D4
:10C1F000044B236310BDC046ADC90000D5C9000083
:10C200000DCA000039CA000010B5024900F08CF8D0
:10C2100010BDC04669C1000070B568254A1E55436F
:10C220000E002900743100F081F9041E08D00021AD
:10C230002A00016046600C30A0606832FFF7D0F938
:10C24000200070BD836913B50400002B28D18364DE
:10C25000C3640365134B144A1B68826201939842BE
:10C2600001D101238361200000F020F860602000EC
:10C2700000F01CF8A060200000F018F80022E06038
:10C2800004216068FFF79CFF01220921A068FFF7E5
:10C2900097FF02221221E068FFF792FF0123A361BA
:10C2A00013BDC0462CE3000009C20000F8B51C4BCA
:10C2B00007001E68B369002B02D13000FFF7C2FFF0
:10C2C0004836B4687368013B04D53368002B07D047
:10C2D0003668F6E70C22A55E002D0DD06834F2E733
:10C2E00004213800FFF798FF30600028F0D10C23BC
:10C2F00004003B602000F8BD20000A4B6566256005
:10C300006560A560E36025616561A561082229007B
:10C310005C30FFF765F96563A563A564E564E9E74B
:10C320002CE300000100FFFFF7B504000700002622
:10C3300001914834002C01D13000FEBD6368A5682E
:10C340000093009B013B009301D52468F2E7AB8981
:10C35000012B08D90E22AB5E013304D0290038002E
:10C36000019B984706436835EBE7EC30006870475F
:10C3700070B50E001D000E23C95E96B01400002992
:10C3800007DA00232B60B3891B0611D48023DB005E
:10C390000FE06A4600F088FB0028F2DBF022019BE8
:10C3A00012021340054A9B185A4253412B60EDE795
:10C3B00040230020236016B070BDC04600E0FFFFA0
:10C3C000F7B502268B8905000C00334206D0230006
:10C3D00047332360236101236361F7BD01AB6A46E4
:10C3E000FFF7C6FF00990700280000F09FF800281B
:10C3F00008D10C22A35E9A05EFD4032293431E4377
:10C40000A681E4E70F4BAB628023A289206013432F
:10C41000A381009B20616361019B002B0DD00E2343
:10C42000E15E280000F052FB002806D00322A38919
:10C4300093431A0001231343A381A0893843A081A9
:10C44000CBE7C04609C2000010B5034B01001868D5
:10C4500000F06CF810BDC0468400002082B00029B6
:10C4600000D101A9101E06D0002B06D013780B6056
:10C470001078431E984102B0704702204042FAE70C
:10C48000C9B28218904201D10020704703788B42D4
:10C49000FBD00130F6E7000070B50500002910D090
:10C4A0000C1F2368002B00DAE418280000F034FB8E
:10C4B0001D4A1368002B05D163601460280000F04A
:10C4C0002CFB70BDA34209D9216860188342F3D1C7
:10C4D00018685B6841182160EEE713005A68002A6B
:10C4E00001D0A242F9D919685818A0420BD120688E
:10C4F0000918581819608242E0D110685268411832
:10C5000019605A60DAE7A04202D90C232B60D5E704
:10C5100021686018824203D1106852684118216076
:10C5200062605C60CAE7C046301C0020032370B51F
:10C53000CD1C9D43083506000C2D1ED20C25A942AA
:10C540001DD8300000F0E8FA254A146821000029BF
:10C5500019D1244C2368002B03D1300000F0CAF914
:10C5600020602900300000F0C5F9431C2BD10C23BA
:10C570003000336000F0D1FA03E0002DDFDA0C2345
:10C580003360002070BD0B685B1B19D40B2B03D9E3
:10C590000B60CC18256003E04B688C420DD1136012
:10C5A000300000F0BAFA200007220B30231D904320
:10C5B000C31AE7D05A42E250E4E763600C00EFE7A9
:10C5C0000C004968C3E70323C41C9C43A042E1D08C
:10C5D000211A300000F08EF9431CDBD1C7E7C046BA
:10C5E000301C0020341C0020F8B507000D00160098
:10C5F000002905D11100FFF799FF04002000F8BDC4
:10C60000002A03D1FFF748FF3400F7E700F086FA6D
:10C610002C00B042F2D231003800FFF787FF041E31
:10C62000ECD029003200FEF7BFFF29003800FFF7E9
:10C6300033FFE3E7F0B58E6885B007000C00039286
:10C6400001939E423CD890238A89DB001A4234D061
:10C650000325096923685B1A0293636902985D43A5
:10C66000EB0F5D19019B6D1001331B18AB4200D914
:10C670001D00530532D529003800FFF757FF061E6D
:10C6800009D10C233B6040230120A289404213437F
:10C69000A38105B0F0BD029A2169FEF785FFA38949
:10C6A000144A1A4080231343A381029B2661F61883
:10C6B00026606561019EED1AA560019B9E4200D92E
:10C6C000019E320003992068FEF777FFA3680020DF
:10C6D0009B1BA36023689E192660DAE72A003800B6
:10C6E000FFF782FF061EE0D121693800FFF7D4FE74
:10C6F000C7E7C0467FFBFFFFF0B59FB002900593F0
:10C700008B890F0016001B0611D50B69002B0ED16B
:10C710004021FFF70BFF38603861002805D10C235A
:10C72000029A013813601FB0F0BD40237B610023E3
:10C7300006AC6361203363761033A37635002B7823
:10C74000002B01D0252B46D1AB1B04930CD032001B
:10C7500039000298FFF76EFF431C00D1AEE062691A
:10C76000049B9446634463612B78002B00D1A5E0C1
:10C77000012200235242626002A9543252186E1CF8
:10C780002360E360A3601370A365317805225448E9
:10C79000FFF776FE751C00281FD12268D30604D54A
:10C7A000532302A95B1820211970130704D55323C2
:10C7B00002A95B182B21197033782A2B16D035006B
:10C7C00000210A20E3682A786E1C303A092A4ED9E3
:10C7D000002918D010E00135B1E7414B2268C01A9A
:10C7E00001238340134323602E00CEE7059B191DD0
:10C7F0001B680591002B01DB099304E05B42E360B9
:10C800000223134323602B782E2B0AD16B782A2B1B
:10C8100035D1059B02351A1D1B680592002B2BDBB9
:10C820000793304E297803223000FFF729FE0028B5
:10C8300006D04023801B83402268013513432360C8
:10C840002978062228486E1C2176FFF719FE002859
:10C850003CD0264B002B25D10722059B0733934361
:10C86000083305936369039A9B18636166E7434342
:10C8700001219B183500A6E701235B42D0E7002386
:10C880000A201A000135636029786E1C30390929A5
:10C8900003D9002BC5D00792C3E7424301235218A6
:10C8A0003500F1E705AB00933A00114B21000298E7
:10C8B00000E000BF0390039B0133D3D1BB890B98E9
:10C8C0005B0600D42FE7012040422CE705AB009324
:10C8D0003A00074B21000298FFF736F8EAE7C04616
:10C8E00030E3000036E300003AE3000000000000FF
:10C8F00035C60000002370B5064C05000800236013
:10C9000000F060F9431C03D12368002B00D02B609A
:10C9100070BDC046C42F002070B504000D001F2953
:10C9200004D9162303600120404270BD436C002BE4
:10C9300004D08A009B181A68002A08D1200000F051
:10C9400031F82A000100200000F01AF8EDE700207D
:10C95000012AEAD0511C03D1162301302360E4E7F9
:10C96000002428001C6090472000DEE710B5034B30
:10C9700001001868FFF7D0FF10BDC04684000020FA
:10C98000002370B5064C050008001100236000F07C
:10C9900001F9431C03D12368002B00D02B6070BD2C
:10C9A000C42F002010B500F0E5F810BD70B50C00E4
:10C9B0000E25495F00F0BAF8002803DB636D1B18F1
:10C9C000636570BDA389024A1340A381F9E7C0469D
:10C9D000FFEFFFFFF8B51F008B8905000C00160064
:10C9E000DB0505D50E23C95E0022022300F080F886
:10C9F000A389054A28001340A38132000E23E15E7B
:10CA00003B0000F02BF8F8BDFFEFFFFF70B50C0006
:10CA10000E25495F00F06CF8A389421C03D1054A3A
:10CA20001340A38170BD802252011343A38160652E
:10CA3000F8E7C046FFEFFFFF10B50E23C95E00F018
:10CA400021F810BD0B1E04D0FF2A04D98A230360ED
:10CA50008B3B180070470A700123FAE770B5050098
:10CA6000080011000022064C22601A0000F0B8F8FD
:10CA7000431C03D12368002B00D02B6070BDC0463F
:10CA8000C42F0020002370B5064C05000800236069
:10CA900000F060F8431C03D12368002B00D02B600A
:10CAA00070BDC046C42F0020002370B5064C0500A1
:10CAB00008001100236000F055F8431C03D12368DF
:10CAC000002B00D02B6070BDC42F0020002370B558
:10CAD000064C05000800236000F054F8431C03D105
:10CAE0002368002B00D02B6070BDC046C42F0020EF
:10CAF00070B50500080011000022064C22601A00E3
:10CB000000F050F8431C03D12368002B00D02B60A9
:10CB100070BDC046C42F0020704770470B1F1B68B4
:10CB2000181F002B01DA0B58C018704770B50500AC
:10CB3000080011000022064C22601A0000F03AF8AA
:10CB4000431C03D12368002B00D02B6070BDC0466E
:10CB5000C42F002058220120014B40421A60704728
:10CB6000C42F002058220120014B40421A60704718
:10CB7000C42F002058220120014B40421A60704708
:10CB8000C42F00205822024B00201A607047C04674
:10CB9000C42F002058220120014B40421A607047E8
:10CBA000C42F002058220120014B40421A607047D8
:10CBB000C42F002058220120014B40421A607047C8
:10CBC000C42F0020044A1368002B00D1034B18180F
:10CBD000106018007047C046381C0020C82F002085
:10CBE00058220120014B40421A607047C42F002098
:10CBF000FEE7C046F8B5C046F8BC08BC9E46704784
:10CC0000F8B5C046F8BC08BC9E46704764617461C4
:10CC10000000000090CC0000EF01000099CC000063
:10CC2000E3020000A1CC000005090000A8CC000030
:10CC3000150A0000ADCC00002D050000B8CC0000A6
:10CC400053030000BDCC00006D0C0000C9CC0000F7
:10CC50001F020000D3CC00000D080000E1CC000052
:10CC6000B9060000EECC0000EF04000072616E64B3
:10CC70006F6D00616C6C006C6173740066616C7345
:10CC800065007472756500252E3135732E2E2E00C9
:10CC90006D616B654C697374006164644C6173749D
:10CCA0000064656C657465006A6F696E00636F701F
:10CCB0007946726F6D546F0066696E64006A6F69C1
:10CCC0006E537472696E677300756E69636F646525
:10CCD000417400756E69636F6465537472696E6741
:10CCE000006E65774279746541727261790066728F
:10CCF00065654D656D6F72790000000061CD0000C3
:10CD0000D510000066CD0000F3100000A1CC00009B
:10CD1000F71000006CCD0000D910000076CD0000A7
:10CD2000FB1000007FCD0000FF10000089CD000047
:10CD30000311000094CD000007110000A0CD0000F9
:10CD4000DD100000A9CD0000EB100000B3CD000005
:10CD5000E1100000BECD0000EF10000066696C65B8
:10CD6000006F70656E00636C6F736500656E644F75
:10CD70006646696C6500726561644C696E65007237
:10CD8000656164427974657300617070656E644CAE
:10CD9000696E6500617070656E64427974657300D8
:10CDA00066696C6553697A650073746172744C6965
:10CDB0007374006E657874496E4C6973740073798E
:10CDC0007374656D496E666F0000000034130000D7
:10CDD000441300005E130000DC1300001414000074
:10CDE0004A14000082140000A8140000E41400009B
:10CDF000261500007C150000C01500002C16000050
:10CE0000741600009A160000D216000018170000D1
:10CE10003E1700006C1700009A170000D2170000A0
:10CE2000561800001E19000094190000021A000094
:10CE30004E1A00006E1A0000901A0000421B0000FB
:10CE4000881B0000001C00002E1C00005E1C00005F
:10CE5000941C0000FC1C00007C1D0000C21D000092
:10CE60000A1E0000801E0000F61E00003E1F00008B
:10CE7000841F0000BA1F00000020000046200000B0
:10CE80008E200000E2200000402100007E210000F2
:10CE9000E82100001E22000066220000AE220000F1
:10CEA000F62200003023000078230000C023000099
:10CEB0002C2500006C170000D2160000282400006A
:10CEC000341300005E2400008A240000C024000007
:10CED000EC2400003413000034130000341300006D
:10CEE00034130000A6250000E82500002E260000CF
:10CEF0007E260000AA260000FA2600002027000057
:10CF00004E27000034130000341300007227000085
:10CF1000A2270000D22700000828000032280000C5
:10CF20006828000092280000BA280000E2280000CB
:10CF30004829000078290000A2290000CC2900001F
:10CF4000FC290000262A00003413000034130000DE
:10CF5000341300003413000034130000562A00007C
:10CF6000822A0000AE2A0000DA2A0000062B000008
:10CF70003C2B0000722B0000A82B0000DE2B0000D1
:10CF80000A2C0000362C00006C2C0000341300002A
:10CF90003413000034130000341300003413000075
:10CFA0003413000034130000341300003413000065
:10CFB0003413000034130000341300003413000055
:10CFC00034130000982C0000CE2C00005B25642058
:10CFD0006974656D206C6973745D00282564206236
:10CFE000797465732900286F626A656374207479A7
:10CFF00070653A2025642900537461636B20756E57
:10D00000646572666C6F7700626F6F6C65616E004D
:10D010006E756D62657200737472696E67006C691B
:10D020007374006279746520617272617900000026
:10D0300007000000030000008AD00000F12D00006E
:10D0400092D00000A12E00009BD000004B2F0000CA
:10D05000A4D00000F52D0000ADD000004F2F00003F
:10D06000B5D00000392F00000000000001000000D2
:10D070000200000003000000040000000A0000009D
:10D080006D6963726F3A62697400686173546F6EA0
:10D090006500706C6179546F6E65006861735365EB
:10D0A00072766F00736574536572766F00646163A6
:10D0B000496E69740064616357726974650047431F
:10D0C00020746F6F6B2025642075736563733B203C
:10D0D0006672656520256420776F726473003C4931
:10D0E0006E74656765723E003C4C6973743E003C2B
:10D0F0004F626A6563743E003C42797465417272A6
:10D1000061793E000D0A564D2050616E69633A20E8
:10D1100025730D0A006D69736300000051D1000092
:10D120000D3C00005AD100009D3B00005ED1000084
:10D13000F13A000066D10000973A000070D100007B
:10D140002D3A00007CD100002F3900006E756C6C08
:10D1500000686578546F496E740073696E006A7375
:10D160006F6E476574006A736F6E436F756E7400FF
:10D170006A736F6E56616C75654174006A736F6E89
:10D180004B65794174000000E4D10000793C000057
:10D19000ECD100007D3C0000F6D100009B3C00007B
:10D1A000FFD10000A53C00000AD20000AF3C000007
:10D1B00016D20000B93C00002BD20000C33C000096
:10D1C00040D20000CD3C00004CD20000D73C000013
:10D1D0005CD20000873C000068D20000913C000057
:10D1E0006E65740068617357694669007374617293
:10D1F00074576946690073746F70576946690077A0
:10D20000696669537461747573006D79495041643E
:10D2100064726573730068747470536572766572B6
:10D220004765745265717565737400726573706FCC
:10D230006E64546F487474705265717565737400D0
:10D2400068747470436F6E6E656374006874747094
:10D250004973436F6E6E65637465640068747470BF
:10D26000526571756573740068747470526573707B
:10D270006F6E7365001A1B1C03040607090A171852
:10D2800019000000000008080800080A4A400000D1
:10D290000A5FEA5FEA0ED92ED36E19324489330C45
:10D2A000924C924D08080000000488080804080405
:10D2B000848488000A448A4000048EC480000000F0
:10D2C000048800000EC0000000000800012244880D
:10D2D000100C9252524C048C84848E1C824C901EF2
:10D2E0001EC244924C06CA525FE21FF01EC13E02AB
:10D2F000448ED12E1FE24488100ED12ED12E0ED195
:10D300002EC48800080008000004800488024488B5
:10D310000482000EC00EC008048244880ED126C0CC
:10D32000040ED135B36C0C925ED2521C925C925CAE
:10D330000ED010100E1C9252525C1ED01C901E1E5D
:10D34000D01C90100ED013712E12525ED2521C8837
:10D3500008081C1FE242524C1254981492101010EC
:10D36000101E113B75B131113935B3710C92525207
:10D370004C1C925C90100C92524C861C925C925108
:10D380000ED00C825C1FE4848484125252524C11E1
:10D3900031312A44113135BB7112524C9252112A4B
:10D3A0004484841EC488101E0EC808080E10080489
:10D3B00082410EC242424E048A400000000000003A
:10D3C0001F0804800000000ED2524F10101C925C07
:10D3D000000ED0100E02424ED24E0C925C900E0601
:10D3E000C81C88080ED24EC24C10101C9252080065
:10D3F000080808024002424C1014981492080808C9
:10D400000806001B75B131001C925252000C92525A
:10D410004C001C925C90000ED24EC2000ED0101038
:10D420000006C8049808080EC807001252524F00A0
:10D4300011312A4400113135BB00124C8C9200117D
:10D440002A4498001EC4881E06C48C8486080808D6
:10D45000080818080C881800000C83600000000001
:10D4600001000000020000000300000004000000B2
:10D470000500000006000000070000000800000092
:10D48000090000000A0000000B0000000C00000072
:10D490000D0000000E0000000F0000001000000052
:10D4A0001200000014000000160000001800000028
:10D4B0001A0000001C0000001E00000020000000F8
:10D4C0002300000026000000290000002C000000BE
:10D4D0002F00000032000000360000003A0000007B
:10D4E0003E00000042000000460000004B0000002B
:10D4F00050000000550000005A00000061000000CC
:10D50000680000006F000000760000007D00000051
:10D51000840000008B0000009200000099000000D1
:10D52000A0000000A7000000AE000000B500000051
:10D53000BC000000C3000000CA000000D1000000D1
:10D54000D8000000DF000000E6000000ED00000051
:10D55000F4000000FB000000FF000000ACD500005C
:10D56000F93C0000B7D500008D420000C1D5000095
:10D57000B53E0000CED50000FD400000D5D500002E
:10D580004D410000DED500009D410000EAD50000BD
:10D5900095400000FBD50000253F000008D60000A4
:10D5A00025400000646973706C6179006C6967687C
:10D5B000744C6576656C006D62446973706C61795A
:10D5C000006D62446973706C61794F6666006D62CC
:10D5D000506C6F74006D62556E706C6F74006D628C
:10D5E000447261775368617065006D625368617061
:10D5F00065466F724C6574746572006E656F506934
:10D6000078656C53656E64006E656F506978656C03
:10D6100053657450696E004E6F7420656E6F756748
:10D620006820726F6F6D206576656E206166746527
:10D630007220636F6D70616374696F6E00436F6D0C
:10D6400070616374656420466C61736820636F6405
:10D65000652073746F72650A25642062797465733E
:10D66000207573656420282564252529206F662090
:10D67000256400426164207265636F726420666F86
:10D68000756E6420647572696E6720696E6974696D
:10D69000616C697A6174696F6E002564202564206D
:10D6A00025642028256420776F726473290025641F
:10D6B000207265636F7264732C20256420776F720B
:10D6C00064732C206D617849442025642C20636F9D
:10D6D0006D70616374696F6E206379636C6573202C
:10D6E000256400526573746F72656420256420732D
:10D6F000637269707473005374617274656400724C
:10D700006164696F0000000098D700005D4C000064
:10D71000A5D70000F94E0000B5D70000794E0000F3
:10D72000C3D700008D500000CED70000854C00000C
:10D73000DED700000D4D0000F2D70000F54C0000D0
:10D7400001D800006F5200000DD80000ED5100001C
:10D7500016D800009151000021D80000D9500000D7
:10D760002CD800001551000035D8000049510000A8
:10D770003ED80000954C00004DD80000754C0000CC
:10D7800056D80000A54C00006E6F6E65006F74687F
:10D79000657200706169720064697361626C6552E0
:10D7A0006164696F006D6573736167655265636578
:10D7B00069766564007061636B6574526563656961
:10D7C0007665007061636B657453656E64007265A5
:10D7D000636569766564496E746567657200726534
:10D7E0006365697665644D657373616765547970C7
:10D7F00065007265636569766564537472696E6706
:10D800000073656E64496E74656765720073656E5A
:10D8100064506169720073656E64537472696E67F7
:10D82000007365744368616E6E656C007365744760
:10D83000726F757000736574506F776572007369ED
:10D84000676E616C537472656E67746800646576A8
:10D850006963654944006C6173744D6573736167F6
:10D8600065494400556E6B6E6F776E207072696DFE
:10D870006974697665205B25733A25735D00000045
:10D8800000000000963007772C610EEEBA5109991E
:10D8900019C46D078FF46A7035A563E9A395649E7A
:10D8A0003288DB0EA4B8DC791EE9D5E088D9D2979E
:10D8B0002B4CB609BD7CB17E072DB8E7911DBF90FA
:10D8C0006410B71DF220B06A4871B9F3DE41BE841E
:10D8D0007DD4DA1AEBE4DD6D51B5D4F4C785D3837A
:10D8E00056986C13C0A86B647AF962FDECC9658A1E
:10D8F0004F5C0114D96C0663633D0FFAF50D088D7A
:10D90000C8206E3B5E10694CE44160D5727167A21D
:10D91000D1E4033C47D4044BFD850DD26BB50AA579
:10D92000FAA8B5356C98B242D6C9BBDB40F9BCAC9D
:10D93000E36CD832755CDF45CF0DD6DC593DD1ABF9
:10D94000AC30D9263A00DE518051D7C81661D0BF1D
:10D95000B5F4B42123C4B3569995BACF0FA5BDB879
:10D960009EB802280888055FB2D90CC624E90BB11D
:10D97000877C6F2F114C6858AB1D61C13D2D66B679
:10D980009041DC760671DB01BC20D2982A10D5EFDD
:10D990008985B1711FB5B606A5E4BF9F33D4B8E839
:10D9A000A2C9077834F9000F8EA8099618980EE1DD
:10D9B000BB0D6A7F2D3D6D08976C6491015C63E639
:10D9C000F4516B6B62616C1CD83065854E0062F25D
:10D9D000ED95066C7BA5011BC1F4088257C40FF5B9
:10D9E000C6D9B06550E9B712EAB8BE8B7C88B9FCDD
:10D9F000DF1DDD62492DDA15F37CD38C654CD4FB39
:10DA00005861B24DCE51B53A7400BCA3E230BBD4DC
:10DA100041A5DF4AD795D83D6DC4D1A4FBF4D6D338
:10DA20006AE96943FCD96E34468867ADD0B860DADC
:10DA3000732D0444E51D03335F4C0AAAC97C0DDD38
:10DA40003C710550AA41022710100BBE86200CC95C
:10DA500025B56857B3856F2009D466B99FE461CEB8
:10DA60000EF9DE5E98C9D9292298D0B0B4A8D7C7DC
:10DA7000173DB359810DB42E3B5CBDB7AD6CBAC038
:10DA80002083B8EDB6B3BF9A0CE2B6039AD2B17454
:10DA90003947D5EAAF77D29D1526DB048316DC73B0
:10DAA000120B63E3843B64943E6A6D0DA85A6A7A54
:10DAB0000BCF0EE49DFF099327AE000AB19E077DB0
:10DAC00044930FF0D2A3088768F2011EFEC20669D4
:10DAD0005D5762F7CB67658071366C19E7066B6E30
:10DAE000761BD4FEE02BD3895A7ADA10CC4ADD6754
:10DAF0006FDFB9F9F9EFBE8E43BEB717D58EB060B0
:10DB0000E8A3D6D67E93D1A1C4C2D83852F2DF4F53
:10DB1000F167BBD16757BCA6DD06B53F4B36B248AF
:10DB2000DA2B0DD84C1B0AAFF64A0336607A044153
:10DB3000C3EF60DF55DF67A8EF8E6E3179BE6946AF
:10DB40008CB361CB1A8366BCA0D26F2536E26852D3
:10DB500095770CCC03470BBBB91602222F2605552F
:10DB6000BE3BBAC5280BBDB2925AB42B046AB35C53
:10DB7000A7FFD7C231CFD0B58B9ED92C1DAEDE5BAF
:10DB8000B0C2649B26F263EC9CA36A750A936D0293
:10DB9000A906099C3F360EEB8567077213570005EF
:10DBA000824ABF95147AB8E2AE2BB17B381BB60C13
:10DBB0009B8ED2920DBED5E5B7EFDC7C21DFDB0B6F
:10DBC000D4D2D38642E2D4F1F8B3DD686E83DA1F93
:10DBD000CD16BE815B26B9F6E177B06F7747B718EF
:10DBE000E65A0888706A0FFFCA3B06665C0B011193
:10DBF000FF9E658F69AE62F8D3FF6B6145CF6C16EF
:10DC000078E20AA0EED20DD75483044EC2B3033992
:10DC1000612667A7F71660D04D476949DB776E3EEE
:10DC20004A6AD1AEDC5AD6D9660BDF40F03BD83712
:10DC300053AEBCA9C59EBBDE7FCFB247E9FFB5306E
:10DC40001CF2BDBD8AC2BACA3093B353A6A3B42492
:10DC50000536D0BA9306D7CD2957DE54BF67D923EE
:10DC60002E7A66B3B84A61C4021B685D942B6F2A92
:10DC700037BE0BB4A18E0CC31BDF055A8DEF022DEE
:10DC8000416C6C207461736B732073746F7070657A
:10DC900064007631303100202573202573004D65F6
:10DCA0006D6F727920636C6561726564004E6F20E0
:10DCB00066726565207461736B20656E7472696548
:10DCC0007300000014DD00000166000021DD00008B
:10DCD000A56100002DDD0000D165000033DD0000EE
:10DCE000E165000039DD0000F16500003FDD000066
:10DCF000D961000049DD00005D66000051DD0000D3
:10DD0000B16300005ADD00003562000073656E7378
:10DD10006F727300616363656C65726174696F6EC5
:10DD20000074656D70657261747572650074696CFC
:10DD300074580074696C74590074696C745A007476
:10DD40006F7563685265616400693263526561642E
:10DD50000069326357726974650072656164444892
:10DD600054000000D8DD0000E9660000E6DD000098
:10DD7000ED660000EFDD0000F9660000F9DD00004F
:10DD8000FD66000002DE00000167000007DE000003
:10DD9000056700000CDE00000967000018DE0000C7
:10DDA0000D6700001FDE00001167000028DE000084
:10DDB000156700002DDE00001967000038DE000046
:10DDC0001D67000042DE0000F16600004CDE00002E
:10DDD000F566000074667400656E61626C65446986
:10DDE00073706C6179006765745769647468006763
:10DDF000657448656967687400736574506978650F
:10DE00006C006C696E65007265637400726F756E8C
:10DE10006465645265637400636972636C65007461
:10DE20007269616E676C65007465787400746674FD
:10DE3000546F756368656400746674546F756368C5
:10DE40005800746674546F7563685900746674542E
:10DE50006F75636850726573737572650076617271
:10DE60007300000084DE0000AD6B00008EDE000059
:10DE70008D6B000097DE0000696B0000A3DE0000E0
:10DE8000F56A000076617245786973747300766193
:10DE9000724E616D6564007365745661724E616D9A
:10DEA0006564007661724E616D65466F72496E649D
:10DEB00065780057656C636F6D6520746F204D69E0
:10DEC00063726F426C6F636B732100705F73706974
:10DED00020213D204E554C4C002F686F6D652F67FB
:10DEE00069742F2E706C6174666F726D696F2F701C
:10DEF00061636B616765732F6672616D65776F72C1
:10DF00006B2D61726475696E6F6E6F726469636E9A
:10DF10007266352F6C69627261726965732F535036
:10DF2000492F5350492E63707000535049436C6120
:10DF300073733A3A535049436C617373284E524697
:10DF40005F5350495F547970652A2C2075696E744F
:10DF5000385F742C2075696E74385F742C20756975
:10DF60006E74385F7429000000000000000000009B
:10DF7000B96D0000756D00009B6D0000A56D00007F
:10DF8000AF6D0000996D000003000000020000006A
:10DF90000100000004000000050000001100000066
:10DFA0000C0000000B000000120000000A0000003E
:10DFB000060000001A000000140000001700000016
:10DFC000160000001500000010000000FFFFFFFF1A
:10DFD000FFFFFFFF000000001E000000190000000E
:10DFE0001800000007000000080000000900000001
:10DFF0000D0000000E0000000F0000001C000000DB
:10E000001B0000001D0000001300000000000000C5
:10E0100000000000697200009D7A0000E9720000B3
:10E02000FD720000F372000065720000597200007A
:10E0300009730000857200005572000000000000A6
:10E04000000000000000304300000000000030C36A
:10E050007371727400000000FB21F93FFB2109403D
:10E060007CD91240FB2119407A6A1F407CD922409A
:10E07000BBFD2540FB2129403A462C407A6A2F40BF
:10E080005C4731407CD932409C6B3440BBFD35400D
:10E09000DB8F3740FB2139401BB43A403A463C40C5
:10E0A0005AD83D407A6A3F404C7E40405C474140F0
:10E0B0006C1042407CD942408CA243409C6B44404F
:10E0C000AC344540BBFD4540CBC64640DB8F4740A6
:10E0D000EB584840FB21494083F9A200444E6E00B2
:10E0E000FC291500D1572700DD34F50062DBC000A4
:10E0F0003C999500419043006351FE00BBDEAB00AC
:10E10000B761C5003A6E2400D24D42004906E000D6
:10E1100009EA2E001C92D100EB1DFE0029B11C0063
:10E12000E83EA700F535820044BB2E009CE9840040
:10E13000B4267000417E5F00D691390053833900C8
:10E140009CF439008B5F840028F9BD00F81F3B0068
:10E15000DEFF97000F980500112FEF000A5A8B0081
:10E160006D1F6D00CF7E360009CB2700464FB700EC
:10E170009E663F002DEA5F00BA277500E5EBC700F9
:10E180003D7BF100F739070092528A00FB6BEA00F1
:10E190001FB15F00085D8D00300356007BFC460018
:10E1A000F0AB6B0020BCCF0036F49A00E3A91D0051
:10E1B0005E619100081BE60085996500A0145F0070
:10E1C0008D40680080D8FF0027734D00060631009F
:10E1D000CA561500C9A873007BE260006B8CC000B2
:10E1E00000000040FB21F93F000000002D44743E78
:10E1F000000000809846F83C0000006051CC783B5D
:10E2000000000080831BF0390000004020257A3890
:10E21000000000802282E336000000001DF3693513
:10E2200002000000030000000400000006000000DF
:10E2300014970000BE960000BE960000EC97000008
:10E24000BA960000BA960000E2970000EC97000032
:10E25000BA960000E2970000BA960000EC97000022
:10E26000F0970000F0970000F0970000F89700008A
:10E27000F0A1000062A00000A6A000000AA000001B
:10E28000A6A0000096A10000A6A000000AA0000021
:10E2900062A0000062A0000096A100000AA0000099
:10E2A00002A0000002A0000002A00000A4A1000043
:10E2B00018A900001AA800001AA8000038AB000036
:10E2C00014A8000014A8000020AB000038AB000028
:10E2D00014A8000020AB000014A8000038AB000018
:10E2E0002EAB00002EAB00002EAB00003CAB0000BC
:10E2F0002C2066756E6374696F6E3A2000617373CB
:10E30000657274696F6E2022257322206661696CC4
:10E3100065643A2066696C6520222573222C206C86
:10E32000696E65202564257325730A008800002026
:10E33000232D302B2000686C4C00656667454647EE
:10E340000030313233343536373839414243444571
:10E3500046003031323334353637383961626364E0
:10E3600065660000000000000000000000000000E2
:10E37000000000000000000000000000000000009D
:10E38000000000000000000000000000000000008D
:10E39000000000000000000000000000000000007D
:10E3A000000000000000000000000000000000006D
:10E3B000000000000000000000000000000000005D
:10E3C000000000004300504F534958000020202017
:10E3D0002020202020202828282828202020202015
:10E3E00020202020202020202020202020881010E5
:10E3F0001010101010101010101010101004040441
:10E4000004040404040404101010101010104141FE
:10E4100041414141010101010101010101010101EC
:10E420000101010101010101101010101010424200
:10E4300042424242020202020202020202020202BC
:10E44000020202020202020210101010200000005C
:10E4500000000000000000000000000000000000BC
:10E4600000000000000000000000000000000000AC
:10E47000000000000000000000000000000000009C
:10E48000000000000000000000000000000000008C
:10E49000000000000000000000000000000000007C
:10E4A000000000000000000000000000000000006C
:10E4B000000000000000000000000000000000005C
:10E4C000000000000000000000000000000000004C
:04E4D0000000000048
:08E4D400341CFF7F0100000071
:10E4DC00FFFFFFFFD007000001000000E803DC0590
:10E4EC00DC05DC05DC050000FFFFFFFFFFFFFFFF85
:10E4FC001800000019FCFFFFFFFFFFFFFF000000EA
:10E50C000024F4000200000003000000FFFFFFFFE6
:10E51C0000000000010000000000020001000000EB
:10E52C00FFFFFFFF000000000200000000000400DD
:10E53C0002000000FFFFFFFF0000000003000000CE
:10E54C0000000800030000000A00000008000000A2
:10E55C0001000000880000200000000084E300009F
:10E56C00A4E3000064E300000000000000000000D1
:10E57C00000000000000000000000000000000008F
:10E58C00000000000000000000000000000000007F
:10E59C00000000000000000000000000000000006F
:10E5AC00000000000000000000000000000000005F
:10E5BC00000000000000000043000000000000000C
:10E5CC00000000000000000000000000000000003F
:10E5DC0000000000000000004300000000000000EC
:10E5EC00000000000000000000000000000000001F
:10E5FC0000000000000000004300000000000000CC
:10E60C0000000000000000000000000000000000FE
:10E61C0000000000000000004300000000000000AB
:10E62C0000000000000000000000000000000000DE
:10E63C00000000000000000043000000000000008B
:10E64C0000000000000000000000000000000000BE
:10E65C00000000000000000043000000000000006B
:10E66C00000000000000000000000000000000009E
:10E67C00000000000000000043000000000000004B
:10E68C00000000000000000000000000000000007E
:10E69C00000000000000000045CA00005DC400003E
:10E6AC0000000000CCE300008ECC000014D1000070
:10E6BC0014D1000014D1000014D1000014D10000BA
:10E6CC0014D1000014D1000014D1000014D10000AA
:10E6DC00FFFFFFFFFFFFFFFFFFFFFFFFFFFF00003C
:10E6EC0001004153434949000000000000000000B4
:10E6FC00000000000000000000000000000000000E
:10E70C000000415343494900000000000000000094
:10E71C0000000000000000000000000000000000ED
:10E72C0000000000E9000000456D00008D70000045
:08E73C00B5750000C1000000EA
:04000003000071295F
:00000001FF
